:020000040000FA
:080000000002040000000000F2
:04000C00823300003B
:10001000823300008233000082330000823300000C
:1000200082330000823300008233000082330000FC
:1000300082330000823300008233000082330000EC
:1000400082330000823300008233000082330000DC
:1000500082330000823300008233000082330000CC
:1000600082330000823300008233000082330000BC
:1000700082330000823300008233000082330000AC
:10008000823300008233000082330000823300009C
:10009000823300008233000082330000823300008C
:1000A000B833000082330000823300008233000046
:1000B000823300008233000082330000823300006C
:1000C000823300008233000082330000823300005C
:1000D000823300008233000082330000823300004C
:1000E000823300008233000082330000823300003C
:1000F000823300008233000082330000823300002C
:10010000823300008233000082330000823300001B
:10011000823300008233000082330000823300000B
:1001200082330000823300008233000082330000FB
:1001300082330000823300008233000082330000EB
:1001400082330000823300008233000082330000DB
:1001500082330000823300008233000082330000CB
:1001600082330000823300008233000082330000BB
:1001700082330000823300008233000082330000AB
:10018000823300008233000082330000823300009B
:10019000823300008233000082330000823300008B
:1001A000823300008233000082330000823300007B
:1001B000823300008233000082330000823300006B
:1001C000823300008233000082330000823300005B
:1001D000823300008233000082330000823300004B
:1001E000823300008233000082330000823300003B
:1001F000823300008233000082330000823300002B
:1004000000802000E1FF2100018009000018EB00BE
:100410002060EF00040028008411880004402000C0
:1004200094118800A4002000C41188002CA3EF00C0
:100430002AA3EF006CA3EF006AA3EF000FF82300DC
:10044000F0FF230020A0B700000000000028EF000C
:100450003868EF003968EF00E439EF0097C0A90071
:10046000040E2000140288002CA3EF002AA3EF0042
:100470002400240034168800CA62A800C662A900BD
:10048000CA82A800C682A900A00020006E33020024
:10049000000000000408200064168800047020009A
:1004A0009416880044052000F416880004282100D2
:1004B00024178800CA02A900C602A90040A7A90003
:1004C0003D68A9003D88A9003DA8A90001002000C1
:1004D00001007800282E0200000000008100E800E2
:1004E0003322AF00FEFF3700A011880090022000E9
:1004F0000008E600F6FF3700010020000100780048
:10050000622E0200000000008100E8003322AF00EC
:10051000FEFF3700A0118800E00020000008E60080
:10052000F6FF370000C4B3002DEBB70048340200DB
:1005300000000000C435020000000000D762A800DF
:1005400060C0B30096FCB70010C0B30097FCB700C2
:10055000063402000000000010C0B3001DEBB7001D
:1005600010C0B30025EBB700907CEF00917CEF004A
:100570004636020000000000F4FF200024638800DB
:10058000622CEF0005002000050078007E2E02009E
:10059000000000000040B3004220AF00050037001B
:1005A0008502E8008EFCB700B03A020000000000AF
:1005B000F5FF370040C1B30090FCB700A0C0B30006
:1005C00091FCB7004636020000000000642CEF00EA
:1005D00004FF200014638800050020000500780057
:1005E000A62E0200000000000040B3004220AF0031
:1005F000050037008502E8008EFCB700B03A020023
:1006000000000000F5FF3700A0C5B30090FCB70064
:10061000A0C0B30091FCB700463602000000000005
:10062000642CEF0004F02000146388000500200013
:1006300005007800BE2E0200000000000040B3005C
:100640004220AF00050037008502E8008EFCB700AD
:10065000B03A020000000000F5FF370020C3B300ED
:1006600090FCB70040C1B30091FCB70046360200D1
:1006700000000000642CEF00F400200014638800E8
:100680000500200005007800D62E020000000000C2
:100690000040B3004220AF00050037008502E800AB
:1006A0008EFCB700B03A020000000000F5FF3700F2
:1006B0002A3D020000000000010020000100780037
:1006C000F22E0200000000008100E8003322AF009B
:1006D000FEFF3700A0118800100120000008E6008E
:1006E000F6FF3700F0420200000000000100200089
:1006F00001007800122F0200000000008100E800D5
:100700003322AF00FEFF3700A011880080012000D7
:100710000008E600F6FF3700866D020000000000CA
:10072000648D210084C58800050020000500780044
:10073000382F0200000000000040B3004220AF004C
:10074000040037008502E800664C0200000000004B
:10075000F6FF37008C91020000000000648D21003C
:1007600084C5880005002000050078004C2F020099
:10077000000000000040B3004220AF00040037003A
:100780008502E800664C020000000000F6FF37001A
:100790008C9102000000000097C0A8004220EF00EA
:1007A00038C8BF003948E30004003200D09202008C
:1007B00000000000D0030400000000000200200040
:1007C000E183200002007800B42502000000000050
:1007D000805878000201E8000004E0004220AE00EA
:1007E000F8FF37003C68EF003868EF003968EF0029
:1007F00038C8BF003948E30004003200D09202003C
:1008000000000000F803040000000000F8030400EA
:08081000000000000040FE00A2
:0C4004003220EF00030A2000830150006E
:1040100005003100E3012200008041001040BA0099
:104020000160EF0000000600F001220083814100E2
:10403000808141001380BA000000060000003200B9
:104040000000490000007900005F410000003E00D0
:1040500000077E0000071100001411007F141100FA
:104060007F147E00242A7F007F2A49001223490002
:10407000130849006462360036493E00552241006B
:10408000500041000503410000002200001C7F0099
:104090002241410000004100412222001C001C007E
:1040A00014087F003E08490014084900083E4900F2
:1040B0000808410000507F00300009000008090096
:1040C000080809000808010000603E006000410087
:1040D000002049001008490004027A003E517F0088
:1040E000494508003E000800427F080040007F006C
:1040F000426100005149410046217F004145410095
:104100004B31000018142000127F4000102741009E
:1041100045453F00453901003C4A7F0049490800B8
:1041200030011400710922000503410036497F0067
:10413000494940003606400049494000291E4000D8
:1041400000367F003600020000000C0056360200E8
:1041500000007F0008147F002241040000140800C2
:104160001414100014147F0000413E00221441007A
:10417000080241000151410009063E003220EF00D3
:10418000030A20008301500005003100A30D220026
:10419000008041001040BA000160EF0000000600FE
:1041A000B00D220083814100808141001380BA005C
:1041B000000006007F097C0009091400063E140077
:1041C00041511400215E08007F09080019291400DC
:1041D000464614004949180049317C0001017C0021
:1041E0007F010800013F040040400400403F0800F8
:1041F0001F204800402054001F3F54004038540006
:10420000403F20006314040008143F00630744008B
:10421000087040000807200061513C0049454000FB
:10422000430040007F41200041007C0002041C004C
:104230000810200020004000414120007F001C00A9
:1042400004023C00010240000440300040404000B5
:1042500040403C00000144000204280000201000FF
:1042600054542800547844007F480C0044445000C3
:10427000383850004444500044203C003844440046
:10428000444864007F38540054544C00541844008F
:10429000087E000009010800020C3600525241005D
:1042A000523E00007F0800000404000078007F00F8
:1042B000447D00004000000020400000443D4100DB
:1042C000007F360010280800440000000041100064
:1042D0007F400800007C08000418100004780800E3
:1042E0007C087800040446007838410044444600C5
:1042F000443878003220EF0023082000830150006A
:104300000500310063192200008041001040BA000E
:104310000160EF0000000600701922008381410057
:10432000808141001380BA00000006001E213C007D
:1043300061214100123C400041404100217C3C0091
:104340003854000056550000182000005555000054
:1043500055780000205520005455480078203E0034
:10436000555649005478620020540000555400000E
:10437000781C000022620000221000003855000066
:10438000555500001838000055540000551800001D
:10439000385440005556680018003E00457C09001E
:1043A00041000200004520007D41540000005600FD
:1043B000457E550040007800781500001415440033
:1043C00078787E0014154100147800007C54380081
:1043D000565544004424460054784500544838005B
:1043E0007E093C007E494000493842004545210095
:1043F00045387C0038457C004445090038380500C4
:1044000045460500443878003C417C0041210900C4
:104410007C3C110041422100207C7C000C517E003C
:10442000505125003C3825004544260045381800E9
:104430003220EF0043222200008041001040BA00E9
:104440000160EF00000006002063000061720000C0
:10445000643F00003F200000000000003220EF0019
:10446000A3232200008041001040BA000160EF0049
:10447000000006004361000072640000203F00005D
:10448000202000002020000020200000200000004C
:104490003220EF0043252200008041001040BA0086
:1044A0000160EF0000000600616300006D64000021
:1044B000383D000025780000200000003220EF0089
:1044C000A3262200008041001040BA000160EF00E6
:1044D00000000600436100007264000020420000FA
:1044E0006F6F0000742E00002E2E000000000000F0
:1044F0003220EF0043282200008041001040BA0023
:104500000160EF0000000600737400006174000099
:10451000313D0000202500004C7800002000000004
:104520003220EF00C3292200008041001040BA0071
:104530000160EF0000000600737400006174000069
:10454000323D0000202500004C78000020000000D3
:104550003220EF00432B2200008041001040BA00BF
:104560000160EF00000006005344000048430000D3
:104570003D20000025780000200000003220EF00E0
:10458000A32C2200008041001040BA000160EF001F
:1045900000000600202000005344000020420000DC
:1045A0006F6F0000742E00002E2E0000000000002F
:1045B0003220EF00432E2200008041001040BA005C
:1045C0000160EF0000000600534400004843000073
:1045D000204200006F6F0000742E00002E2E00009D
:1045E000000000003220EF00E32F22000080410095
:1045F0001040BA000160EF00000006007374000074
:1046000061740000333D0000202500006C7800003C
:10461000200000003220EF006331220000804100C2
:104620001040BA000160EF00000006006163000066
:104630006D640000343100003D200000257800004A
:10464000200000003220EF00E33222000080410011
:104650001040BA000160EF00000006004D4D000060
:10466000432000004D4F00004445000020000000A2
:104670003220EF0043342200008041001040BA0095
:104680000160EF0000000600204D00004D430000D7
:10469000204200006F6F0000740000003220EF0025
:1046A000A3352200008041001040BA000160EF00F5
:1046B000000006000A0D0000207200006561000085
:1046C000645F0000626F00006F74000020730000E0
:1046D0007461000072740000696E000067200000C1
:1046E0000A0D0000000000003220EF000338220015
:1046F000008041001040BA000160EF000000060099
:104700005365000063560000423D0000254C000048
:10471000782000000A0D0000000000003220EF00A9
:10472000A3392200008041001040BA000160EF0070
:10473000000006004270000053650000633D000069
:10474000202500004C780000200A00000D00000029
:104750003220EF00433B2200008041001040BA00AD
:104760000160EF0000000600536500006370000068
:10477000436C0000753D0000202500004C780000CF
:10478000200A00000D0000003220EF00033D22004F
:10479000008041001040BA000160EF0000000600F8
:1047A00052530000656300003D200000254C0000CE
:1047B000782000000A0D0000000000003220EF0009
:1047C000A33E2200008041001040BA000160EF00CB
:1047D0000000060046610000744E00003D2000000D
:1047E000254C0000782000000A0D000000000000A9
:1047F0003220EF0043402200008041001040BA0008
:104800000160EF00000006005365000063460000F1
:1048100061740000313D0000202500004C7800004C
:10482000200A00000D0000003220EF0003422200A9
:10483000008041001040BA000160EF000000060057
:1048400046410000543100005F6C000062610000CE
:104850005F73000074610000727400003D2000006E
:10486000254C0000782000000A0D00000000000028
:104870003220EF0043442200008041001040BA0083
:104880000160EF0000000600537000004661000068
:10489000743D0000202500004C780000200A000034
:1048A0000D0000003220EF00E345220000804100AF
:1048B0001040BA000160EF00000006005244000002
:1048C00069720000456E0000744E00003D2000003B
:1048D000254C0000782000000A0D000000000000B8
:1048E0003220EF00C3472200008041001040BA0090
:1048F0000160EF0000000600204600004154000067
:10490000313600002C200000000000003220EF00B3
:1049100023492200008041001040BA000160EF00EE
:104920000000060053650000635200006F6F000036
:1049300074440000697200003D2500004C780000BE
:10494000200A00000D0000003220EF00034B22007F
:10495000008041001040BA000160EF000000060036
:10496000456E00006453000065630000526F000054
:104970006F74000044690000723D0000254C000087
:10498000782000000A0D0000000000003220EF0037
:10499000234D2200008041001040BA000160EF006A
:1049A00000000600536500006370000046410000EF
:1049B00054330000323D0000254C000078200000F8
:1049C0000A0D0000000000003220EF00034F22001B
:1049D000008041001040BA000160EF0000000600B6
:1049E000436C0000755200006F6F000074440000BB
:1049F000697200005F46000041540000333200003D
:104A00003D2500004C780000200A00000D00000049
:104A10003220EF0043512200008041001040BA00D4
:104A20000160EF00000006006C62000061520000AF
:104A30006F6F000074440000697200003D250000A3
:104A40004C780000200A00000D0000003220EF002A
:104A500023532200008041001040BA000160EF00A3
:104A600000000600212100002042000070530000D9
:104A70006563000020690000732000006E6F000075
:104A80007420000035310000322000002121000098
:104A9000200A00000D0000003220EF0083552200A4
:104AA000008041001040BA000160EF0000000600E5
:104AB00053630000616E00006E6900006E670000C5
:104AC0002E2E00002E0000003220EF00035722009F
:104AD000008041001040BA000160EF0000000600B5
:104AE000444500004C2000000A0D000000000000BA
:104AF0003220EF0043582200008041001040BA00ED
:104B00000160EF00000006004C4600004E2000004F
:104B10000A0D0000000000003220EF00835922003F
:104B2000008041001040BA000160EF000000060064
:104B3000454E000044310000200A00000D00000036
:104B40003220EF00C35A2200008041001040BA001A
:104B50000160EF0000000600454E000044320000F6
:104B6000200A00000D0000003220EF00035C22004C
:104B7000008041001040BA000160EF000000060014
:104B8000000000003220EF00E35C220000804100C2
:104B90001040BA000160EF000000060064690000E8
:104BA000725F0000703D00002575000020200000AD
:104BB000000000003220EF00635E22000080410010
:104BC0001040BA000160EF0000000600202A00003B
:104BD000303100002A200000000000003220EF00E9
:104BE000A35F2200008041001040BA000160EF0086
:104BF00000000600202A0000303300002A200000B8
:104C0000000000003220EF00E3602200008041003D
:104C10001040BA000160EF0000000600726F000053
:104C20006F740000200000003220EF0003622200B9
:104C3000008041001040BA000160EF000000060053
:104C4000202A0000303400002A200000000000006C
:104C50003220EF0043632200008041001040BA0080
:104C60000160EF0000000600202A0000303500003F
:104C70002A200000000000003220EF0083642200A0
:104C8000008041001040BA000160EF000000060003
:104C90002A2A00002A460000494C0000453D000039
:104CA000200000003220EF00E36522000080410078
:104CB0001040BA000160EF000000060064690000C7
:104CC000725F00006E7500006D620000657200008A
:104CD0003D2500006C750000200000003220EF0030
:104CE000A3672200008041001040BA000160EF007D
:104CF0000000060025730000200A00000D200000BF
:104D0000000000003220EF00E36822000080410034
:104D10001040BA000160EF00000006006E65000060
:104D200078740000436C0000757300007465000027
:104D3000723D0000254C0000782000000A0D0000A4
:104D4000000000003220EF00E36A220000804100F2
:104D50001040BA000160EF0000000600204600008D
:104D600041540000333200002C20000000000000FD
:104D70003220EF00436C2200008041001040BA0056
:104D80000160EF0000000600202A000066720000AB
:104D9000616700003D200000257800002A20000007
:104DA0000A0D0000000000003220EF00036E220018
:104DB000008041001040BA000160EF0000000600D2
:104DC0006C620000615F000073740000617200009B
:104DD000743D0000254C0000782000000000000019
:104DE0003220EF00C36F2200008041001040BA0063
:104DF0000160EF0000000600616400006430000004
:104E000031200000000000003220EF00037122007A
:104E1000008041001040BA000160EF000000060071
:104E20007730000031200000000000003220EF0049
:104E300023722200008041001040BA000160EF00A0
:104E40000000060020730000746F00007030000046
:104E500031200000000000003220EF0083732200A8
:104E6000008041001040BA000160EF000000060021
:104E70002C2E00003B3F0000213A000020200000C3
:104E8000000000003220EF00E374220000804100A7
:104E90001040BA000160EF000000060063790000D6
:104EA000636C000065320000200A00000D00000065
:104EB0003220EF0043762200008041001040BA000B
:104EC0000160EF00000006000A0D00000A0D00005E
:104ED00025730000000000003220EF0083772200DD
:104EE000008041001040BA000160EF0000000600A1
:104EF0000A0D00002A2A0000204900006E6400000C
:104F00006578000020730000656100007263000096
:104F1000682000000A0D0000000000003220EF00B1
:104F2000A3792200008041001040BA000160EF0028
:104F3000000006002023000023230000257300004A
:104F400020230000232300000A0D000000000000C1
:104F50003220EF00437B2200008041001040BA0065
:104F60000160EF00000006000A0D00002A2A000080
:104F7000205700004F520000442000004E4F000018
:104F800054200000464F0000554E00004420000011
:104F90002A20000021210000200A00000D0000004E
:104FA0003220EF00C37D2200008041001040BA0093
:104FB0000160EF00000006000A0D00002A2A000030
:104FC000204600006173000074200000736500003B
:104FD0006172000063680000200A00000D200000DC
:104FE000000000003220EF00E37F2200008041003B
:104FF0001040BA000160EF00000006000A0D00003A
:105000002A2A0000204E00006F7200006D6100002F
:105010006C2000007365000061720000636800008E
:10502000200A00000D200000000000003220EF00E8
:1050300023822200008041001040BA000160EF008E
:1050400000000600206D000032200000000000007B
:105050003220EF0043832200008041001040BA005C
:105060000160EF0000000600206D0000312000000C
:10507000000000003220EF00638422000080410025
:105080001040BA000160EF0000000600202A000076
:10509000636C0000755F0000736B000069700000B6
:1050A0003D2500006C750000200000003220EF005C
:1050B00023862200008041001040BA000160EF000A
:1050C00000000600202A000073650000635F0000F6
:1050D000736B0000697000003D2500006C750000D6
:1050E000200000003220EF00E38722000080410012
:1050F0001040BA000160EF000000060020660000CA
:10510000736300003D2500006C7500002000000066
:105110003220EF0043892200008041001040BA0095
:105120000160EF00000006002066000073730000BD
:105130003D2500006C750000200000003220EF00CB
:10514000A38A2200008041001040BA000160EF00F5
:1051500000000600206600006C6C00003D25000089
:105160006C750000200000003220EF00038C22004C
:10517000008041001040BA000160EF00000006000E
:1051800020660000663D0000256C000075200000D0
:10519000000000003220EF00638D220000804100FB
:1051A0001040BA000160EF0000000600202A000055
:1051B00066630000633D0000256C00007520000060
:1051C000000000003220EF00E38E2200008041004A
:1051D0001040BA000160EF0000000600202A000025
:1051E00066740000633D0000256C0000752000001F
:1051F000000000003220EF00639022000080410098
:105200001040BA000160EF00000006006C61000071
:10521000737400005F6C000062610000733D000069
:10522000256C0000752000002A0A00000D00000017
:105230003220EF0043922200008041001040BA006B
:105240000160EF0000000600202B00002B2D000065
:105250002D2B00002B310000200000003220EF0039
:10526000A3932200008041001040BA000160EF00CB
:1052700000000600202B00002B2D00002D2B00002D
:105280002B320000200000003220EF0003952200A6
:10529000008041001040BA000160EF0000000600ED
:1052A000202B00002B2D00002D2B00002B330000A5
:1052B000200000003220EF006396220000804100B1
:1052C0001040BA000160EF0000000600202A000034
:1052D0002A2D00002D4200002D2D00002A2A00005A
:1052E000200000003220EF00E39722000080410000
:1052F0001040BA000160EF000000060020700000BE
:105300007265000030330000200000003220EF0002
:1053100023992200008041001040BA000160EF0094
:105320000000060020730000747200006561000038
:105330006D200000000000003220EF00839A220060
:10534000008041001040BA000160EF00000006003C
:10535000202B00002B2D00002D2B00002B370000F0
:10536000200000003220EF00E39B2200008041007B
:105370001040BA000160EF0000000600202B000082
:105380002B2D00002D2B00002B38000020000000EA
:105390003220EF00439D2200008041001040BA00FF
:1053A0000160EF000000060061640000643200004C
:1053B000200000003220EF00639E220000804100A8
:1053C0001040BA000160EF000000060077300000D6
:1053D00032200000000000003220EF00839F2200F6
:1053E000008041001040BA000160EF00000006009C
:1053F0000A0D00002A2A0000205700004F5200002A
:10540000442000004E4F000054200000464F000092
:10541000554E0000442000002A2A000020540000BD
:10542000414B0000494E0000472000004E4500005F
:105430005854000020210000212000000A0D000027
:10544000000000003220EF00E3A2220000804100B3
:105450001040BA000160EF00000006005374000025
:105460006172000074200000706800006F6E000020
:10547000656D000065200000696E00006465000035
:10548000786900006E670000200A00000D0000002F
:105490003220EF0043A52200008041001040BA00F6
:1054A0000160EF0000000600546F0000746100000E
:1054B0006C200000466900006C650000732000004D
:1054C0003D200000256C0000752000000A0D000042
:1054D000000000003220EF0063A72200008041009E
:1054E0001040BA000160EF0000000600546F000099
:1054F000746100006C2000004469000072650000C7
:10550000637400006F720000696500007320000082
:105510003D200000256C0000752000000A0D0000F1
:10552000000000003220EF00E3A9220000804100CB
:105530001040BA000160EF0000000600526F00004A
:105540006F7400003A200000636F00006E7400006A
:10555000616900006E730000200000003220EF003F
:10556000A3AB2200008041001040BA000160EF00B0
:1055700000000600446900007265000063740000CA
:105580006F72000079200000256C0000753A000061
:10559000200000003220EF0063AD220000804100B7
:1055A0001040BA000160EF0000000600256C00000A
:1055B00075200000666900006C6500007320000023
:1055C0000A0D0000000000003220EF0003AF2200AF
:1055D000008041001040BA000160EF0000000600AA
:1055E000204C000069730000746900006E670000C1
:1055F000206600006F7500006E64000020660000E9
:10560000696C0000657300002E2E00002E20000043
:105610000A0D0000000000003220EF0083B12200DC
:10562000008041001040BA000160EF000000060059
:105630000A0D0000202A00002A200000666E0000EB
:105640006E3D0000253400006C7500002000000055
:105650003220EF0043B32200008041001040BA0026
:105660000160EF0000000600206600007363000088
:105670003D250000386C000075200000000000008F
:105680003220EF00C3B42200008041001040BA0075
:105690000160EF0000000600206600007373000048
:1056A0003D250000386C000075200000000000005F
:1056B0003220EF0043B62200008041001040BA00C3
:1056C0000160EF0000000600206600006C6C000026
:1056D0003D250000386C000075200000000000002F
:1056E0003220EF00C3B72200008041001040BA0012
:1056F0000160EF00000006002066000072610000FB
:10570000673D000025750000200000003220EF00FA
:1057100023B92200008041001040BA000160EF0070
:1057200000000600202C00003B20000000000000CC
:105730003220EF0043BA2200008041001040BA003E
:105740000160EF0000000600414100000000000081
:105750003220EF0043BB2200008041001040BA001D
:105760000160EF000000060041450000000000005D
:105770003220EF0043BC2200008041001040BA00FC
:105780000160EF000000060041480000000000003A
:105790003220EF0043BD2200008041001040BA00DB
:1057A0000160EF0000000600414F00000000000013
:1057B0003220EF0043BE2200008041001040BA00BA
:1057C0000160EF00000006004157000000000000EB
:1057D0003220EF0043BF2200008041001040BA0099
:1057E0000160EF00000006004158000000000000CA
:1057F0003220EF0043C02200008041001040BA0078
:105800000160EF00000006004159000000000000A8
:105810003220EF0043C12200008041001040BA0056
:105820000160EF0000000600420000003220EF009F
:1058300023C22200008041001040BA000160EF0046
:105840000000060043480000000000003220EF0086
:1058500023C32200008041001040BA000160EF0025
:105860000000060044480000000000003220EF0065
:1058700023C42200008041001040BA000160EF0004
:1058800000000600440000003220EF0003C52200A3
:10589000008041001040BA000160EF0000000600E7
:1058A00045480000000000003220EF0003C622003F
:1058B000008041001040BA000160EF0000000600C7
:1058C00045520000000000003220EF0003C7220014
:1058D000008041001040BA000160EF0000000600A7
:1058E00045590000000000003220EF0003C82200EC
:1058F000008041001040BA000160EF000000060087
:10590000460000003220EF00E3C822000080410082
:105910001040BA000160EF000000060047000000E0
:105920003220EF00C3C92200008041001040BA00BD
:105930000160EF0000000600484800000000000081
:105940003220EF00C3CA2200008041001040BA009C
:105950000160EF0000000600494800000000000060
:105960003220EF00C3CB2200008041001040BA007B
:105970000160EF000000060049590000000000002F
:105980003220EF00C3CC2200008041001040BA005A
:105990000160EF00000006004A480000000000001F
:1059A0003220EF00C3CD2200008041001040BA0039
:1059B0000160EF00000006004B0000003220EF0005
:1059C000A3CE2200008041001040BA000160EF0029
:1059D000000006004C0000003220EF0083CF2200C0
:1059E000008041001040BA000160EF000000060096
:1059F0004D0000003220EF0063D022000080410003
:105A00001040BA000160EF00000006004E470000A1
:105A1000000000003220EF0063D12200008041002E
:105A20001040BA000160EF00000006004E000000C8
:105A30003220EF0043D22200008041001040BA0023
:105A40000160EF00000006004F570000000000005A
:105A50003220EF0043D32200008041001040BA0002
:105A60000160EF00000006004F5900000000000038
:105A70003220EF0043D42200008041001040BA00E1
:105A80000160EF00000006005041000055000000DA
:105A90003220EF0043D52200008041001040BA00C0
:105AA0000160EF0000000600500000003220EF000F
:105AB00023D62200008041001040BA000160EF00B0
:105AC00000000600520000003220EF0003D7220041
:105AD000008041001040BA000160EF0000000600A5
:105AE00053480000000000003220EF0003D82200DD
:105AF000008041001040BA000160EF000000060085
:105B0000530000003220EF00E3D822000080410063
:105B10001040BA000160EF00000006005448000089
:105B2000000000003220EF00E3D922000080410095
:105B30001040BA000160EF000000060054000000B1
:105B40003220EF00C3DA2200008041001040BA008A
:105B50000160EF0000000600554800000000000052
:105B60003220EF00C3DB2200008041001040BA0069
:105B70000160EF0000000600555700000000000023
:105B80003220EF00C3DC2200008041001040BA0048
:105B90000160EF0000000600560000003220EF0018
:105BA000A3DD2200008041001040BA000160EF0038
:105BB00000000600570000003220EF0083DE2200C4
:105BC000008041001040BA000160EF0000000600B4
:105BD000590000003220EF0063DF22000080410006
:105BE0001040BA000160EF00000006005A480000B3
:105BF000000000003220EF0063E02200008041003E
:105C00001040BA000160EF00000006005A000000DA
:105C10003220EF0043E12200008041001040BA0032
:105C20000160EF00000006004465000066610000AE
:105C3000756C000074200000696E0000746500003F
:105C40007272000075700000740D00000A00000000
:105C50003220EF00E30120008301500005003100F5
:105C600043E42200008041001040BA000160EF00D0
:105C70000000060050E42200838141008081410041
:105C80001380BA00000006000A0D70000A0D6500BE
:105C90000A0D65002030630035366800202D200095
:105CA00020544D00442D6F00535064003031750076
:105CB00020546C0065786500742D0000546F00005E
:105CC0002D5300003220EF00E3E622000080410067
:105CD0001040BA000160EF00000006000A0D00004D
:105CE000206200006F6F0000746900006E670000A2
:105CF0002E2E00002E0A00000D0000003220EF00C2
:105D0000A3E82200008041001040BA000160EF00CB
:105D100000000600204F00004C4500004420000019
:105D200031360000302000007820000031320000C1
:105D300038200000646F00007473000020520000DF
:105D40004742000020210000200000003220EF0028
:105D500023EB2200008041001040BA000160EF00F8
:105D60000000060054650000636800004465000000
:105D700073690000676E0000200000003220EF0011
:105D8000A3EC2200008041001040BA000160EF0047
:105D900000000600456C000065630000747200009E
:105DA0006F6E000069630000730000003220EF0096
:105DB00023EE2200008041001040BA000160EF0095
:105DC000000006002030000035360000202D0000C5
:105DD000205700004156000020540000545300009A
:105DE000200000003220EF00E3EF2200008041009D
:105DF0001040BA000160EF0000000600204D0000D6
:105E00004D4300002F53000044200000696E000045
:105E100069740000206400006F6E000065200000BF
:105E2000000000003220EF00E3F12200008041007A
:105E30001040BA000160EF0000000600204D000095
:105E40004D4300002F530000442000007265000005
:105E500061640000206200006F6F00007420000089
:105E6000646F00006E6500000A0D00002000000055
:105E70003220EF0043F42200008041001040BA00BD
:105E80000160EF00000006004D4F00004455000087
:105E90004C450000000000003220EF0083F5220096
:105EA000008041001040BA000160EF0000000600D1
:105EB0005245000041440000590000003220EF002C
:105EC000A3F62200008041001040BA000160EF00FC
:105ED00000000600434D0000554500004E470000FD
:105EE0007E3100002E5400005854000000000000D5
:105EF0003220EF0043F82200008041001040BA0039
:105F00000160EF0000000600434D0000554900000D
:105F10004E4400007E3100002E5400005854000012
:105F2000000000003220EF00E3F922000080410071
:105F30001040BA000160EF0000000600414100007F
:105F40002E57000041560000000000003220EF00F4
:105F500023FB2200008041001040BA000160EF00E6
:105F600000000600414500002E5700004156000089
:105F7000000000003220EF0063FC2200008041009E
:105F80001040BA000160EF00000006004148000028
:105F90002E57000041560000000000003220EF00A4
:105FA000A3FD2200008041001040BA000160EF0014
:105FB00000000600414F00002E570000415600002F
:105FC000000000003220EF00E3FE220000804100CC
:105FD0001040BA000160EF000000060041570000C9
:105FE0002E57000041560000000000003220EF0054
:105FF00023002300008041001040BA000160EF0040
:1060000000000600415800002E57000041560000D5
:10601000000000003220EF006301230000804100F7
:106020001040BA000160EF00000006004159000076
:106030002E57000041560000000000003220EF0003
:10604000A3022300008041001040BA000160EF006D
:1060500000000600422E00005741000056000000DC
:106060003220EF00C3032300008041001040BA003B
:106070000160EF0000000600434800002E570000BA
:1060800041560000000000003220EF00030523000D
:10609000008041001040BA000160EF0000000600DF
:1060A000442E000057410000560000003220EF004F
:1060B00023062300008041001040BA000160EF0079
:1060C00000000600444800002E5700004156000022
:1060D000000000003220EF00630723000080410031
:1060E0001040BA000160EF000000060045480000C3
:1060F0002E57000041560000000000003220EF0043
:10610000A3082300008041001040BA000160EF00A6
:1061100000000600455200002E57000041560000C6
:10612000000000003220EF00E3092300008041005E
:106130001040BA000160EF00000006004559000061
:106140002E57000041560000000000003220EF00F2
:10615000230B2300008041001040BA000160EF00D3
:1061600000000600462E00005741000056000000C7
:106170003220EF00430C2300008041001040BA00A1
:106180000160EF0000000600472E000057410000AC
:10619000560000003220EF00630D23000080410014
:1061A0001040BA000160EF000000060048480000FF
:1061B0002E57000041560000000000003220EF0082
:1061C000A30E2300008041001040BA000160EF00E0
:1061D00000000600494800002E570000415600000C
:1061E000000000003220EF00E30F23000080410098
:1061F0001040BA000160EF0000000600495900009D
:106200002E57000041560000000000003220EF0031
:1062100023112300008041001040BA000160EF000C
:10622000000006004A4800002E57000041560000BA
:10623000000000003220EF006312230000804100C4
:106240001040BA000160EF00000006004B2E000075
:1062500057410000560000003220EF008313230056
:10626000008041001040BA000160EF00000006000D
:106270004C2E000057410000560000003220EF0075
:10628000A3142300008041001040BA000160EF0019
:10629000000006004D2E000057410000560000008F
:1062A0003220EF00C3152300008041001040BA00E7
:1062B0000160EF00000006004E2E00005741000074
:1062C000560000003220EF00E3162300008041005A
:1062D0001040BA000160EF00000006004E470000C9
:1062E0002E57000041560000000000003220EF0051
:1062F00023182300008041001040BA000160EF0025
:10630000000006004F5700002E57000041560000C5
:10631000000000003220EF006319230000804100DC
:106320001040BA000160EF00000006004F59000065
:106330002E57000041560000000000003220EF0000
:10634000A31A2300008041001040BA000160EF0052
:1063500000000600502E00005741000056000000CB
:106360003220EF00C31B2300008041001040BA0020
:106370000160EF000000060050410000552E0000B3
:1063800057410000560000003220EF00031D23009B
:10639000008041001040BA000160EF0000000600DC
:1063A000522E000057410000560000003220EF003E
:1063B000231E2300008041001040BA000160EF005E
:1063C00000000600532E0000574100005600000058
:1063D0003220EF00431F2300008041001040BA002C
:1063E0000160EF0000000600534800002E57000037
:1063F00041560000000000003220EF0083202300FF
:10640000008041001040BA000160EF00000006006B
:10641000542E000057410000560000003220EF00CB
:10642000A3212300008041001040BA000160EF006A
:1064300000000600544800002E570000415600009E
:10644000000000003220EF00E32223000080410022
:106450001040BA000160EF0000000600554800003F
:106460002E57000041560000000000003220EF00CF
:1064700023242300008041001040BA000160EF0097
:1064800000000600555700002E570000415600003E
:10649000000000003220EF0063252300008041004F
:1064A0001040BA000160EF0000000600562E000008
:1064B00057410000560000003220EF0083262300E1
:1064C000008041001040BA000160EF0000000600AB
:1064D000572E000057410000560000003220EF0008
:1064E000A3272300008041001040BA000160EF00A4
:1064F00000000600592E0000574100005600000021
:106500003220EF00C3282300008041001040BA0071
:106510000160EF00000006005A2E00005741000005
:10652000560000003220EF00E329230000804100E4
:106530001040BA000160EF00000006005A48000059
:106540002E57000041560000000000003220EF00EE
:10655000232B2300008041001040BA000160EF00AF
:1065600000000600706800006F6E00005F540000BD
:106570006F5F0000506C0000617900003D25000055
:106580006C750000200000003220EF00032D230076
:10659000008041001040BA000160EF0000000600DA
:1065A000666900006C6500005F6C000062610000BD
:1065B0005F6C0000656E000067740000683D0000BD
:1065C000254C0000782000000A0D000000000000AB
:1065D0003220EF00432F2300008041001040BA001A
:1065E0000160EF0000000600666900006C650000B5
:1065F0005F7400006F740000616C0000636C000049
:10660000757300007465000072730000206900005B
:10661000733D0000202500006C7800002000000081
:106620003220EF00C3312300008041001040BA0047
:106630000160EF00000006006C6100007374000050
:106640005F6C000062610000733D0000256C00007B
:1066500078200000000000003220EF008333230088
:10666000008041001040BA000160EF000000060009
:10667000737400006172000074200000706C0000F0
:1066800061790000696E0000672E00002E0A00008C
:106690000D0000003220EF00633523000080410030
:1066A0001040BA000160EF0000000600200000006A
:1066B0003220EF0043362300008041001040BA0032
:1066C0000160EF0000000600200A00000D0A000033
:1066D0000D25000073200000000000000000E00015
:1066E0004220AF0006003700190E0900000000002C
:1066F000FF3F0900000000000000E900F7FF37003D
:10670000000006004200F8003600F800801F780004
:10671000200020000C000900B01F780001002000BC
:1067200001007800082E0200000000008100E8004F
:106730003322AF00FEFF3700A011880020012000A7
:106740000008E600F6FF3700803E20006E330200AE
:1067500000000000A00120000C0009004F1078008C
:106760004F0078003600F9004200F90000400600B2
:106770004200F8003600F800801F7800200020005A
:106780000C000900B01F7800C44180000960EF00D0
:1067900063802000830242003202AE00FEFF370019
:1067A000B0118000804A780038C8BF003AE8B700CE
:1067B000C4418000614242000440780000E0B7001C
:1067C0000160EF0024032000110009000480D800BC
:1067D0000140780038E8B70038C8BF003948E30006
:1067E00002003A003AC8BF0038E8B70087C0A900E5
:1067F000A00120000C0009004F1078004F00780025
:106800003600F9004200F90000400600851F7800BC
:10681000E822A900CB62A900C762A900CB82A80028
:10682000C782A900CBA2A900C7A2A900B4E4800036
:106830000960EF000380200083024200B516880043
:10684000CBA2A800C7A2A900E822A800E822A900BC
:10685000CB62A800C762A900CB82A800C782A900AA
:10686000CBA2A900C7A2A900B4E480004822DE00A0
:106870000380200083024200B5168800CBA2A80046
:10688000C7A2A900E822A800CF02780000000600F5
:10689000E822A800E9E2A900A00020006E3302006F
:1068A00000000000E9E2A8001E0E09000000000040
:1068B000FF3F090000000000400620006E33020088
:1068C0000000000040C0B30096FCB70010C0B30049
:1068D00097FCB70006340200000000001E0E0900FD
:1068E00000000000FF3F09000000000040C0B300AE
:1068F00096FCB70040C0B30097FCB7000634020016
:10690000000000001E0E090000000000FF3F09000B
:106910000000000060C1B30096FCB70050C4B30093
:1069200097FCB700063402000000000020C0B3004E
:1069300096FCB70010C4B30097FCB7000634020001
:106940000000000080C0B30096FCB70030C0B30068
:1069500097FCB700063402000000000090C0B300AE
:1069600096FCB70050C0B30097FCB7000634020095
:1069700000000000A0C0B30096FCB70050C0B300F8
:1069800097FCB7000634020000000000B0C0B3005E
:1069900096FCB70080C4B30097FCB7000634020031
:1069A00000000000C0C0B30096FCB700D0C4B30024
:1069B00097FCB7000634020000000000D0C0B3000E
:1069C00096FCB70060C4B30097FCB7000634020021
:1069D0000000000000C1B30096FCB7002DCBBF0043
:1069E00097FCB700063402000000000010C1B3009D
:1069F00096FCB7002DCBBF0097FCB7000634020011
:106A00000000000020C1B30096FCB7002DCBBF00F2
:106A100097FCB700063402000000000040C0B3003D
:106A200096FCB700977CEF000634020000000000DF
:106A30001E0E090000000000FF3F090000000000DA
:106A40001E0E090000000000FF3F090000000000CA
:106A5000B0C3B30096FCB700977CEF000634020089
:106A60000000000000000600851F7800D5E48000CB
:106A7000C22ADD009BDCBF000160EF004400DE00A5
:106A80009DFCB700054078009D7CB7009F1CA900C5
:106A90009B7CAF009F1CA800D5E48000C82ADE00C4
:106AA000C52ADD009CDCBF000160EF004100DE0074
:106AB0009EFCB700054078009E7CB7009F3CA90073
:106AC0009C1CAF009F3CA800E822A900CB62A80054
:106AD000C762A900CB82A800C782A900CBA2A900E7
:106AE000C7A2A900E4E480004822DE000380200061
:106AF00083024200B51688009F1CAF0002003700D9
:106B0000CB02A90001003700CB02A800C702A900F0
:106B1000CBA2A800C7A2A900CB62A900C762A900A6
:106B2000E822A800E822A900CB62A800C762A90059
:106B3000CB82A800C782A900CBA2A900C7A2A90046
:106B4000F4E480000960EF0003802000830242002B
:106B5000B51688009F3CAF0002003700CB02A900A9
:106B600001003700CB02A800C702A900CBA2A800F1
:106B7000C7A2A900CB62A900C762A900E822A800A9
:106B8000CF027800000006000470200094168800F0
:106B900070C1B30096FCB700977CEF00063402008A
:106BA0000000000080C1B30096FCB700F0C9B3003C
:106BB00097FCB700063402000000000090C1B3004B
:106BC00096FCB700977CEF0006340200000000003E
:106BD000A0C1B30096FCB700F0C7B30097FCB700A4
:106BE000063402000000000000C2B30096FCB700AB
:106BF000977CEF00063402000000000010C2B300D2
:106C000096FCB700F0C7B30097FCB700063402004B
:106C1000000000000470200094168800E822A900FB
:106C2000CB62A900C762A900CB82A800C782A900D5
:106C3000CBA2A900C7A2A90024822000B416880014
:106C4000CBA2A800C7A2A900CB62A800C762A90076
:106C5000E822A800E639EF0034CF800003002500C9
:106C60000418E100080032009A7CEF009B7CEF00E2
:106C70009C7CEF003435020000000000E639EC0097
:106C80002C360400000000000000060070C1B300B4
:106C900096FCB700977CEF0006340200000000006D
:106CA00080C1B30096FCB700F0C9B30097FCB700F1
:106CB000063402000000000090C1B30096FCB7004B
:106CC000977CEF000634020000000000A0C1B30072
:106CD00096FCB700F0C7B30097FCB700063402007B
:106CE0000000000000C2B30096FCB70090DCBF00BB
:106CF00097FCB700063402000000000010C2B30089
:106D000096FCB70091DCBF0097FCB7000634020088
:106D10000000000090DCBF005EECB7005F6CEF008D
:106D200091DCBF0060ECB700616CEF0004702000E4
:106D300094168800E822A900CB62A900C762A900C6
:106D4000CB82A800C782A900CBA2A900C7A2A90034
:106D500024822000B4168800CBA2A800C7A2A900F4
:106D6000CB62A800C762A900E822A80000000600C4
:106D7000F45580004822DE0074CCB20004003A00D2
:106D800000C8B300BFEAB7002439040000000000C7
:106D9000F45580004822DE00C4CFB20004003A005F
:106DA00010C8B300BFEAB700243904000000000097
:106DB000F45580004822DE0094CEB20004003A0070
:106DC00020C8B300BFEAB700243904000000000067
:106DD000F45580004822DE0024CEB20004003A00C0
:106DE00030C8B300BFEAB700243904000000000037
:106DF000F45580004822DE0044CEB20004003A0080
:106E000040C8B300BFEAB700243904000000000006
:106E1000F45580004822DE0004CEB20004003A009F
:106E200050C8B300BFEAB7002439040000000000D6
:106E3000F45580004822DE0054CEB20004003A002F
:106E400060C8B300BFEAB7002439040000000000A6
:106E5000F45580004822DE0074CEB20004003A00EF
:106E600070C8B300BFEAB700243904000000000076
:106E7000F45580004822DE00A4CEB20004003A009F
:106E800080C8B300BFEAB700243904000000000046
:106E9000F45580004822DE00B4CEB20004003A006F
:106EA00090C8B300BFEAB700243904000000000016
:106EB000F45580004822DE0084CEB20004003A007F
:106EC000A0C8B300BFEAB7002439040000000000E6
:106ED000F45580004822DE00F4CEB20004003A00EF
:106EE000B0C8B300BFEAB7002439040000000000B6
:106EF000F45580004822DE00E4CEB20004003A00DF
:106F0000C0C8B300BFEAB700243904000000000085
:106F1000F45580004822DE00C4CEB20004003A00DE
:106F2000D0C8B300BFEAB700243904000000000055
:106F3000F45580004822DE0044CCB20004003A0040
:106F4000E0C8B300BFEAB700243904000000000025
:106F5000F45580004822DE0054CCB20004003A0010
:106F6000F0C8B300BFEAB7002439040000000000F5
:106F7000F45580004822DE0094CCB20004003A00B0
:106F800000C9B300BFEAB7002439040000000000C4
:106F9000F45580004822DE0064CEB20004003A00BE
:106FA00010C9B300BFEAB700243904000000000094
:106FB000F45580004822DE0064CCB20004003A00A0
:106FC00020C9B300BFEAB700243904000000000064
:106FD000F45580004822DE0044CFB20004003A009D
:106FE00030C9B300BFEAB700243904000000000034
:106FF000F45580004822DE0064CFB20004003A005D
:1070000040C9B300BFEAB700243904000000000003
:10701000F45580004822DE0024CFB20004003A007C
:1070200050C9B300BFEAB7002439040000000000D3
:10703000F45580004822DE00B4CFB20004003A00CC
:1070400060C9B300BFEAB7002439040000000000A3
:10705000F45580004822DE0094CFB20004003A00CC
:1070600070C9B300BFEAB700243904000000000073
:10707000F45580004822DE00F4CFB20004003A004C
:1070800080C9B300BFEAB700243904000000000043
:10709000F45580004822DE0064CDB20004003A00BE
:1070A00090C9B300BFEAB700243904000000000013
:1070B000F45580004822DE00C4CDB20004003A003E
:1070C000A0C9B300BFEAB7002439040000000000E3
:1070D000F45580004822DE0084CFB20004003A005C
:1070E000B0C9B300BFEAB7002439040000000000B3
:1070F000F45580004822DE0034CAB20004003A0091
:10710000C0C9B300BFEAB700243904000000000082
:10711000F45580004822DE0084CDB20004003A001D
:10712000D0C9B300BFEAB700243904000000000052
:10713000F45580004822DE0074CDB20004003A000D
:10714000E0C9B300BFEAB700243904000000000022
:10715000F45580004822DE0034C8B20004003A0032
:10716000F0C9B300BFEAB7002439040000000000F2
:10717000F45580004822DE0014CEB20004003A002C
:1071800000CAB300BFEAB7002439040000000000C1
:10719000F45580004822DE00D4CEB20004003A004C
:1071A00010CAB300BFEAB700243904000000000091
:1071B000F45580004822DE0034CFB20004003A00CB
:1071C00020CAB300BFEAB700243904000000000061
:1071D000F45580004822DE00A4CFB20004003A003B
:1071E00030CAB300BFEAB700243904000000000031
:1071F000F45580004822DE0014CFB20004003A00AB
:1072000040CAB300BFEAB700243904000000000000
:10721000F45580004822DE0014CDB20004003A008C
:1072200050CAB300BFEAB7002439040000000000D0
:10723000F45580004822DE00F4CDB20002003A008E
:1072400060CAB300BFEAB70000000600851F7800DF
:10725000861F7800F45580004822DE0003022000DB
:10726000041CE10003003600BA003700483904006E
:1072700000000000F45580004822DE00F3072000E3
:10728000041CE10002003100B836020000000000DA
:10729000F45580004822DE00630A2000041CE1004F
:1072A00001003100AB003700C76AEF0034568000A0
:1072B0004822DE006524E1007A003100F4558000A8
:1072C0004822DE0003052000041CE1000D0036000A
:1072D000BFCABF000042B100004278000960EF0061
:1072E0006520B80007EBB70007CBBF00C74AB40062
:1072F000022002000000000015EBB700C6390400B0
:1073000000000000F45580004822DE000308200041
:10731000041CE1000D003600BFCABF000045B100EB
:10732000004278000960EF006520B80007EBB70065
:1073300007CBBF00C74AB400BE2002000000000017
:1073400015EBB700C639040000000000F4558000BA
:107350004822DE00730A2000041CE1000B00360006
:10736000BFCABF000048B100004278000960EF00CA
:107370006520B80007EBB70007CBBF00C74AB400D1
:107380007A2102000000000015EBB700917CEF00AD
:1073900091DCBF001D4BE3003F00320070C0B30022
:1073A00090FCB70084E48000F4CFB20037003200D4
:1073B00000F02000640CB600800278004628DE0051
:1073C000A0E4880025638000050FB200B5E48800C2
:1073D000963CD500963CD50020638000EF0260000B
:1073E000C5E48800983CD400983CD40015CBBF007D
:1073F0008000780090DCBF000100A5000F0039007C
:1074000000F02000620CB600800278004628DE0002
:10741000A0E4880015638000050FB200B5E4880081
:10742000963CD500963CD50010638000EF026000CA
:10743000C5E48800983CD400983CD400927CEF00CE
:1074400092DCBF00254BE3000B00320094DCBF0050
:107450009AFCB70096DCBF009BFCB70098DCBF002D
:107460009CFCB7003435020000000000927CEC0068
:10747000203A04000000000084E4800061405200D3
:1074800090FCB700D239040000000000917CEC00B1
:10749000C839040000000000C76AEC005639040037
:1074A0000000000000F02000640CB60080027800AC
:1074B0004628DE00A0E4880025638000050FB200A6
:1074C000B5E48800963CD500963CD500206380004A
:1074D000EF026000C5E48800983CD400983CD400DA
:1074E000917CEF0091DCBF001D4BE30019003200DE
:1074F000907CEF0084E480006824E10012003200F8
:10750000927CEF0092DCBF00254BE3000B003200C1
:1075100094DCBF009AFCB70096DCBF009BFCB70070
:1075200098DCBF009CFCB70034350200000000006E
:10753000927CEC00823A040000000000907CEC0099
:107540007A3A040000000000917CEC00723A0400DA
:10755000000000004F037800CF0278000000060012
:10756000851F7800861F780070C1B30096FCB700B5
:107570005ECCBF0097FCB70006340200000000009C
:10758000E45880004822DE006620B8000080FB003E
:10759000F462800084024000801F780080C1B30044
:1075A00096FCB7004F007800961CF800F5FF9F008E
:1075B000961CF900063402000000000090C1B300E0
:1075C00096FCB70060CCBF0097FCB7000634020001
:1075D0000000000025CBBF004300DD000080FB0061
:1075E000046380008402400061835200A0C1B300A4
:1075F00096FCB7000640780097FCB70006340200FE
:107600000000000000C2B30096FCB7005ECCBF00D3
:1076100097FCB700063402000000000025CBBF0035
:107620004300DD000080FB00046380008402400012
:107630006183520010C2B30096FCB7000640780088
:1076400097FCB70006340200000000000470200020
:1076500094168800E822A900CB62A900C762A9009D
:10766000CB82A800C782A900CBA2A900C7A2A9000B
:1076700024822000B4168800CBA2A800C7A2A900CB
:10768000CB62A800C762A900E822A8008EDCBF0078
:10769000BFEAB7002639020000000000E45880006D
:1076A0004822DE006620B8000080FB005E2CB4009B
:1076B0004F037800CF02780000000600E902A8001E
:1076C00070C0B300F0F9B70084CF8000F4CFB200EF
:1076D00009003200E8C2A90000000000000000001C
:1076E000E8C2A8000000000000000000F079ED00F2
:1076F000643B0400000000000060EF000000060092
:10770000E70160004300DE00010040000000A70028
:10771000E88141000000A1000204E0001098AD00E3
:1077200000000600851F7800C57EEF0070C0B30022
:10773000C6FEB70034F68000F4CFB2001700320066
:1077400021F68000C6DEBF000100A5000200310066
:10775000E902A90001003700E902A80000000000CA
:10776000E8C2A900E8C2A800E6E2AE0008003700BF
:1077700051EC2100C6DEBF000160EF0012002000C6
:10778000821F78004F017800803B0200000000005B
:10779000C67EED009A3B040000000000C5DEBF007D
:1077A000CF02780000000600851F7800C4FEEF00BD
:1077B000923B020000000000B6DEBF00C4FEB7002E
:1077C000923B020000000000B9DEBF00800278009A
:1077D0000B60EF00C41EF800E5FF9F00C41EF90017
:1077E000923B020000000000B8DEBF00C4FEB700FC
:1077F000923B020000000000BBDEBF008002780068
:107800000B60EF00C41EF800E5FF9F00C41EF900E6
:10781000923B020000000000BADEBF00C4FEB700C9
:10782000923B020000000000B7DEBF00C4FEB700BC
:10783000923B020000000000C4FEEF00923B0200F9
:1078400000000000C4FEEF00923B020000000000B8
:1078500035EBB70035CBBF00CF0278000000060043
:10786000851F7800861F78000001EB000103780077
:1078700064C110004211DD000200DD0080027800CA
:107880000C60EC000C60ED000D003200050078008B
:10789000C42ADD004C00DE00F000B2000003B0009E
:1078A000A20320000200E100010039000D40B400F5
:1078B0003322AF00FEFF3700A0118800F1FF370030
:1078C0004F037800CF027800000006006E2CEF0016
:1078D000702CEF00C4FEEF00923B0200000000009D
:1078E000F0D9BF00C4FEB700923B020000000000C8
:1078F000C4FEEF00923B020000000000C4FEEF0057
:10790000923B020000000000C4FEEF00923B020028
:1079100000000000C4FEEF00923B020000000000E7
:10792000C4FEEF00923B020000000000C4FEEF0026
:10793000923B020000000000C4FEEF00923B0200F8
:1079400000000000C4FEEF00923B020000000000B7
:10795000F1F9B700F1D9BF006EECB7006F6CEF0022
:10796000702CEF0070CCBF0071ECB7006FCCBF0083
:1079700070ECB7006ECCBF006FECB7006E6CEF0020
:10798000C4FEEF00923B020000000000F2F9B700D5
:1079900094CF80000960EF00736380000480410091
:1079A0007063880083638000E081490083638800FE
:1079B00070CCBF0071ECB7006FCCBF0070ECB700AB
:1079C0006ECCBF006FECB7006E6CEF00C4FEEF0032
:1079D000923B020000000000F3F9B70094CF800052
:1079E0004822DE00736380000480410070638800D9
:1079F00083638000E08149008363880070CCBF000E
:107A000071ECB7006FCCBF0070ECB7006ECCBF005C
:107A10006FECB7006E6CEF00C4FEEF00923B02000B
:107A200000000000F4F9B700A4CF80000960EF0067
:107A3000736380000480410070638800836380006A
:107A4000E081490083638800706380008163800067
:107A500000000600851F7800861F7800CA62A90012
:107A6000C662A9003D68AE000B003700010020008F
:107A70000100780018220200000000008100E800E8
:107A80003322AF00FEFF3700A011880070002000F5
:107A90000008E600F6FF3700907CEF0000C2B3005C
:107AA00091FCB7004636020000000000642CEF0095
:107AB000F4FF200014638800050020000500780012
:107AC0002E220200000000000040B3004220AF0060
:107AD000050037008502E8008EFCB700B03A0200CE
:107AE00000000000F5FF3700A00F20006E330200F9
:107AF00000000000CA82A800C682A900A0C0B3008E
:107B0000E6F9B70034CF8000F4CFB20005003200B0
:107B10005E3B020000000000E679ED00823D0400BB
:107B200000000000CA82A900C682A90000C4B300F8
:107B3000B6FEB700B83EEF00BA3EEF0050C9B30042
:107B4000B7FEB700D43B020000000000E7F9B70021
:107B50003D68AE0009003700E7D9BF000160EF00C3
:107B600021702200303C0200000000003322AF00F0
:107B7000FEFF370004022000A411880034CF8000EB
:107B80004822DE006124E10007003200CA62A8003A
:107B9000C662A900401F20006E33020000000000F2
:107BA0002E3D04000000000080C4B300B6FEB70004
:107BB000B83EEF0070C8B300B7FEB700A41A2000AB
:107BC000D4F58800D43B020000000000E7F9B700BC
:107BD0003D68AE001400370001002000010078006D
:107BE00048220200000000008100E8003322AF00BC
:107BF000FEFF3700A0118800500020000008E600BA
:107C0000F6FF3700E7D9BF000160EF0021702200C6
:107C1000303C0200000000003322AF00FEFF3700BE
:107C200004022000A411880034CF80004822DE0026
:107C30006124E1002F003A00C4FEEF00923B0200F5
:107C400000000000E7F9B700C4FEEF00923B02001D
:107C500000000000E7F9B700C4FEEF00923B02000D
:107C600000000000E9F9B7003D68AE0009003700E8
:107C7000E9D9BF000160EF0021702200303C020012
:107C8000000000003322AF00FEFF37000402200096
:107C9000A4118800C4FEEF00923B02000000000027
:107CA000EAF9B7003D68AE0009003700EAD9BF0025
:107CB0000160EF0021702200303C02000000000053
:107CC0003322AF00FEFF370004022000A411880019
:107CD00044CF80004822DE006124E10005003A0024
:107CE00054CF8000A4CAB20002003A0010C0B30012
:107CF000E8F9B700E859E20013003A00907CEF0081
:107D000000C2B30091FCB70046360200000000003C
:107D100005002000050078005E220200000000003F
:107D20000040B3004220AF00050037008502E800A4
:107D30008EFCB700B03A020000000000F5FF3700EB
:107D40002440040000000000A0C7B300F0F9B70011
:107D5000663C02000000000060CF880071CF880000
:107D60003D68AE00170037000100200001007800D8
:107D700078220200000000008100E8003322AF00FA
:107D8000FEFF3700A0118800600020000008E60018
:107D9000F6FF370070CF800041702200303C0200B7
:107DA0000000000060CF800041702200303C0200E3
:107DB000000000003322AF00FEFF37000402200065
:107DC000A411880000F02F00EC19B60080027800A2
:107DD00076CF8000F60FB200040028000520E100F5
:107DE00003003A00F40F20000620E10002003200F8
:107DF000A43E04000000000070C7B300B6FEB70048
:107E0000B83EEF00BA3EEF00F0CFB300B7FEB700C8
:107E1000D43B020000000000E9F9B70090C6B300AF
:107E2000B6FEB700BA3EEF00F0CFB300B7FEB70022
:107E300004002400C4F58800D43B020000000000C8
:107E4000EAF9B70044CF80004822DE006224E10056
:107E500004003900EA59E20002003200FC3E04004E
:107E600000000000A0C7B300F0F9B700663C0200B4
:107E70000000000060CF880071CF88003D68AE0030
:107E80001700370001002000010078009022020056
:107E9000000000008100E8003322AF00FEFF370041
:107EA000A0118800600020000008E600F6FF3700FF
:107EB00070CF800041702200303C020000000000C2
:107EC00060CF800041702200303C020000000000C2
:107ED0003322AF00FEFF370004022000A411880007
:107EE0004D6BEF00EFD9AF004D6BEC0000F02F00B1
:107EF000EC19B6008002780076CF8000F60FB20051
:107F0000040028000520E10003003A00F40F2000DF
:107F10000620E10002003200323F040000000000B1
:107F20003D68AE0014003700010020000100780019
:107F3000A8220200000000008100E8003322AF0008
:107F4000FEFF3700A0118800500020000008E60066
:107F5000F6FF37004DCBBF000160EF00217022001B
:107F6000303C0200000000003322AF00FEFF37006B
:107F700004022000A41188004D4BE2001B003A00CF
:107F800054CF80004822DE0043062000041CE1009C
:107F900016003900EB79EC00907CEF0000C2B300D2
:107FA00091FCB700463602000000000005002000EA
:107FB00005007800BE220200000000000040B3006F
:107FC0004220AF00050037008502E8008EFCB700B4
:107FD000B03A020000000000F5FF3700FC3E04004C
:107FE000000000002040040000000000645A8000EF
:107FF0004822DE006124E10011003A00907CEF008D
:1080000000C2B30091FCB700463602000000000039
:108010000500200005007800D822020000000000C2
:108020000040B3004220AF00050037008502E800A1
:108030008EFCB700B03A020000000000F5FF3700E8
:108040007C40040000000000A0C7B300F0F9B700B6
:10805000663C02000000000060CF880071CF8800FD
:108060003D68AE00170037000100200001007800D5
:10807000F2220200000000008100E8003322AF007D
:10808000FEFF3700A0118800600020000008E60015
:10809000F6FF370070CF800041702200303C0200B4
:1080A0000000000060CF800041702200303C0200E0
:1080B000000000003322AF00FEFF37000402200062
:1080C000A411880000F02F00EC19B600800278009F
:1080D00076CF8000F60FB200040028000520E100F2
:1080E00003003A00F40F20000620E10002003200F5
:1080F0002440040000000000907CEF0050C0B3005A
:1081000091FCB700463602000000000070C7B300C3
:10811000B6FEB700B83EEF00BA3EEF00F0CFB300B6
:10812000B7FEB700D43B020000000000E7F9B7003B
:1081300090C6B300B6FEB700BA3EEF00F0CFB30072
:10814000B7FEB70004002400C4F58800D43B020049
:1081500000000000E7F9B7003D68AE0014003700EA
:1081600001002000010078000A2302000000000046
:108170008100E8003322AF00FEFF3700A011880025
:10818000700020000008E600F6FF3700E7D9BF00C6
:108190000160EF0021702200303C0200000000006E
:1081A0003322AF00FEFF370004022000A411880034
:1081B00034CF80004822DE006524E10004003A004C
:1081C000F440040000000000F04004000000000043
:1081D000E759E200020032007C4004000000000089
:1081E0000060EF00370037003D68AE000B0037003D
:1081F000010020000100780022230200000000009E
:108200008100E8003322AF00FEFF3700A011880094
:10821000800020000008E600F6FF3700C4FEEF00F3
:10822000923B02000000000010C4B300B6FEB7008D
:10823000B83EEF00BA3EEF00F0CFB300B7FEB70094
:10824000D43B0200000000000004E00018003200EF
:10825000907CEF0000C2B30091FCB70046360200EC
:10826000000000000500200005007800382302000F
:10827000000000000040B3004220AF0005003700BE
:108280008502E8008EFCB700B03A02000000000052
:10829000F5FF3700907CEF0080C2B30091FCB7007F
:1082A0004636020000000000F44004000000000018
:1082B000C4FEEF00923B02000000000010C0B300BB
:1082C00000E0B7004F037800CF02780000000600FE
:1082D000851F7800B6DEBF00C4FEB700923B0200E7
:1082E00000000000B9DEBF00800278000B60EF00E4
:1082F000C41EF800E5FF9F00C41EF900923B020077
:1083000000000000B8DEBF00C4FEB700923B0200D0
:1083100000000000BBDEBF00800278000B60EF00B1
:10832000C41EF800E5FF9F00C41EF900923B020046
:1083300000000000BADEBF00C4FEB700923B02009E
:1083400000000000B7DEBF00C4FEB700923B020091
:1083500000000000C4FEEF00923B0200000000009D
:10836000CF02780000000600851F78004D4BE20028
:1083700007003A00940020000402E8000402E9002B
:1083800003003200A23ED400A4BED600FBFF37009B
:10839000A21EF800AC1EF900A41EF800A21EF900EF
:1083A000A43EEF00A21EF800AA1EF900CA82A9008E
:1083B000C682A900C4FEEF00923B0200000000004C
:1083C00000C5B300B6FEB700B83EEF00F0CFB30073
:1083D000B7FEB70004202000D4F58800D43B02008B
:1083E000000000000004E00002003200DA41040056
:1083F00000000000C4FEEF00923B020000000000FD
:10840000C4FEEF00923B020000000000CA82A800F8
:10841000C682A900CA82A900C682A90010C5B300FD
:10842000B6FEB700F0CFB300B7FEB700AA1EF80043
:10843000B81EF900AC1EF800BA1EF900684102002F
:1084400000000000C4FEEF00923B020000000000AC
:10845000AEFEB700AE5EE20002003200224204002F
:1084600000000000C4FEEF00923B0200000000008C
:10847000E40F20000024E100FAFF3A00A83EEF00DC
:1084800044F58000032020000418E1000A003600B3
:1084900030F58000A63EEC0080027800C4FEEF00BC
:1084A000923B020000000000804A7800A83EEC00E9
:1084B0004042040000000000C4FEEF00923B0200B6
:1084C00000000000CA82A800C682A9000060EF0078
:1084D000CF02780000000600851F7800C50020004C
:1084E00003000900B51F78000202B8000303B800BA
:1084F0004200A9008502430060844B00020BB800D3
:1085000085024B0008844B00030BB80008044300AD
:108510000780B000870178000801780085007800A6
:10852000040078002501200003000900CF12780024
:10853000CF02780000000600851F7800C5002000EB
:1085400003000900B51F7800090020004300AF00B8
:1085500019002000891F78000002EB008002EB0068
:108560000003EB008003EB000304690011003200FC
:10857000080220004200A9000080D2008180D200C1
:108580000482D2008582D2000328E10001003A0073
:1085900002A0E100030039000202520083825A0067
:1085A0004200A8000683D2008783D2000804E900B5
:1085B000F0FF3A008700780006007800CF047800CA
:1085C0000900E000010032000400BE002501200087
:1085D00003000900CF127800CF02780000000600E7
:1085E000851F780001002000010078004E23020062
:1085F000000000008100E8003322AF00FEFF3700DA
:10860000A0118800700120000008E600F6FF370086
:10861000CA82A900C682A900C4FEEF00923B0200F4
:108620000000000000C5B300B6FEB700B83EEF0082
:10863000F0CFB300B7FEB70004202000D4F58800C7
:10864000D43B0200000000000004E0000200320001
:108650000C43040000000000C4FEEF00923B020047
:1086600000000000C4FEEF00923B0200000000008A
:10867000CA82A800C682A900A23EEF00A43EEF0075
:10868000A49E210034F58800B441020000000000DF
:10869000B3DBBF00E6F9B700E6D9BF0072ECB70064
:1086A000736CEF00742CEF0074CCBF0075ECB70056
:1086B00073CCBF0074ECB70072CCBF0073ECB70092
:1086C000726CEF00B2DBBF00E7F9B70034CF800077
:1086D0004822DE009363800004804100906388009C
:1086E000A3638000E0814900A363880074CCBF00CD
:1086F00075ECB70073CCBF0074ECB70072CCBF0050
:1087000073ECB700726CEF00B1DBBF00E8F9B700A3
:1087100044CF80000960EF00936380000480410033
:1087200090638800A3638000E0814900A363880010
:1087300074CCBF0075ECB70073CCBF0074ECB7000D
:1087400072CCBF0073ECB700726CEF00B0DBBF00FF
:10875000E9F9B70044CF80004822DE00936380002F
:108760000480410090638800A3638000E081490099
:10877000A36388003D88AE001F0037000100200081
:108780000100780074230200000000008100E8006E
:108790003322AF00FEFF3700A011880050002000F8
:1087A0000008E600F6FF3700A06380004170220059
:1087B000303C020000000000906380004170220005
:1087C000303C0200000000003322AF00FEFF370003
:1087D00004022000A41188003322AF00FEFF3700FE
:1087E000A4002000A41188003322AF00FEFF370050
:1087F000D4002000A4118800720CF800A21EF90019
:10880000740CF800A41EF900A49E210034F5880021
:10881000B441020000000000F6D9BF00E6F9B7003D
:10882000E6D9BF007AECB7007B6CEF007C2CEF0040
:108830007CCCBF007DECB7007BCCBF007CECB700EC
:108840007ACCBF007BECB7007A6CEF00F5D9BF00A3
:10885000E7F9B70034CF80004822DE00D363800000
:1088600004804100D0638800E3638000E081490018
:10887000E36388003D68AE001F0037000100200060
:10888000010078008E230200000000008100E80053
:108890003322AF00FEFF3700A011880060002000E7
:1088A0000008E600F6FF3700E06380004170220018
:1088B000303C020000000000D063800041702200C4
:1088C000303C0200000000003322AF00FEFF370002
:1088D00004022000A41188003322AF00FEFF3700FD
:1088E000A4002000A41188003322AF00FEFF37004F
:1088F000D4002000A4118800F7D9BF003DEBB700D9
:108900003D68AE001C003700010020000100780027
:10891000A8230200000000008100E8003322AF001D
:10892000FEFF3700A0118800800020000008E6004C
:10893000F6FF37003DCBBF000160EF002170220041
:10894000303C0200000000003322AF00FEFF370081
:1089500004022000A41188003322AF00FEFF37007C
:10896000A4002000A41188003322AF00FEFF3700CE
:10897000D4002000A4118800F9D9BF00E6F9B7009F
:10898000E6D9BF0068ECB700696CEF0068CCBF00A7
:1089900069ECB700686CEF00F8D9BF00E7F9B700E1
:1089A00034CF80004822DE00436380000480410011
:1089B000406388003D68AE001B00370001002000C6
:1089C00001007800C4230200000000008100E800DC
:1089D0003322AF00FEFF3700A011880050002000B6
:1089E0000008E600F6FF3700406380004170220077
:1089F000303C0200000000003322AF00FEFF3700D1
:108A000004022000A41188003322AF00FEFF3700CB
:108A1000A4002000A41188003322AF00FEFF37001D
:108A2000D4002000A4118800FAD9BF0045EBB7009C
:108A30003D68AE001C0037000100200001007800F6
:108A4000DE230200000000008100E8003322AF00B6
:108A5000FEFF3700A0118800500020000008E6004B
:108A6000F6FF370045CBBF000160EF002170220008
:108A7000303C0200000000003322AF00FEFF370050
:108A800004022000A41188003322AF00FEFF37004B
:108A9000A4002000A41188003322AF00FEFF37009D
:108AA000D4002000A411880090638000680CB400FA
:108AB000B0638800A463800060024A00C463880039
:108AC0003D68AE001F003700010020000100780063
:108AD000F8230200000000008100E8003322AF000C
:108AE000FEFF3700A0118800800020000008E6008B
:108AF000F6FF3700C063800041702200303C020066
:108B000000000000B063800041702200303C020091
:108B1000000000003322AF00FEFF370004022000F7
:108B2000A41188003322AF00FEFF3700A40020000C
:108B3000A41188003322AF00FEFF3700D4002000CC
:108B4000A4118800B0638000C1638000D2638000FC
:108B5000E36380006C420200000000003064880083
:108B6000416488003D68AE001F003700010020000E
:108B70000100780014240200000000008100E800D9
:108B80003322AF00FEFF3700A0118800F000200064
:108B90000008E600F6FF37004064800041702200C4
:108BA000303C020000000000306480004170220070
:108BB000303C0200000000003322AF00FEFF37000F
:108BC00004022000A41188003322AF00FEFF37000A
:108BD000A4002000A41188003322AF00FEFF37005C
:108BE000D4002000A411880001DABF00E6F9B70024
:108BF000E6D9BF006AECB7006B6CEF006ACCBF002F
:108C00006BECB7006A6CEF0000DABF00E7F9B70061
:108C100034CF80004822DE0053638000048041008E
:108C2000506388003D68AE001B0037000100200043
:108C30000100780038240200000000008100E800F4
:108C40003322AF00FEFF3700A01188006000200033
:108C50000008E600F6FF37005063800041702200F4
:108C6000303C0200000000003322AF00FEFF37005E
:108C700004022000A41188003322AF00FEFF370059
:108C8000A4002000A41188003322AF00FEFF3700AB
:108C9000D4002000A4118800FCD9BF00E6F9B70079
:108CA000E6D9BF006CECB7006D6CEF006CCCBF0078
:108CB0006DECB7006C6CEF00FBD9BF00E7F9B700B3
:108CC00034CF80004822DE006363800004804100CE
:108CD000606388003D68AE001B0037000100200083
:108CE0000100780052240200000000008100E8002A
:108CF0003322AF00FEFF3700A01188009000200053
:108D00000008E600F6FF3700606380004170220033
:108D1000303C0200000000003322AF00FEFF3700AD
:108D200004022000A41188003322AF00FEFF3700A8
:108D3000A4002000A41188003322AF00FEFF3700FA
:108D4000D4002000A41188003DCBBF000160EF00DB
:108D500001002000D2638000E36380006C420200C7
:108D60000000000050648800616488006C0CE20020
:108D70006C0032006A0CE2006A0032000100200040
:108D80000100780070240200000000008100E8006B
:108D90003322AF00FEFF3700A011880070002000D2
:108DA0000008E600F6FF37007068A90054638000F1
:108DB000235A8000C819DE000320B800B463800085
:108DC0000400400090648800C46380000300200019
:108DD00004804900A06488003D68AE001F00370091
:108DE000010020000100780086240200000000003D
:108DF0008100E8003322AF00FEFF3700A011880099
:108E0000A00020000008E600F6FF3700A064800004
:108E100041702200303C020000000000906480009D
:108E200041702200303C0200000000003322AF00FD
:108E3000FEFF370004022000A41188003322AF0097
:108E4000FEFF3700A4002000A41188003322AF00E9
:108E5000FEFF3700D4002000A41188006563800065
:108E6000C52ADD004300A9000500780001002000AC
:108E7000D2638000E36380009C4202000000000097
:108E80009464800004004000B0648800A464800002
:108E900004804800C06488003D68AE001F003700B1
:108EA0000100200001007800A4240200000000005E
:108EB0008100E8003322AF00FEFF3700A0118800D8
:108EC000D00020000008E600F6FF3700C0648000F4
:108ED00041702200303C020000000000B0648000BD
:108EE00041702200303C0200000000003322AF003D
:108EF000FEFF370004022000A41188003322AF00D7
:108F0000FEFF3700A4002000A41188003322AF0028
:108F1000FEFF3700D4002000A4118800064A040098
:108F2000000000007068A80011DABF00E6F9B70081
:108F3000E6D9BF007EECB7007F6CEF00802CEF001D
:108F400080CCBF0081ECB7007FCCBF0080ECB700C5
:108F50007ECCBF007FECB7007E6CEF0010DABF0064
:108F6000E7F9B70034CF80004822DE00F3638000C9
:108F700004804100F063880003648000E0814900C0
:108F80000364880080CCBF0081ECB7007FCCBF00B9
:108F900080ECB7007ECCBF007FECB7007E6CEF00AA
:108FA0000FDABF00E8F9B70044CF80000960EF0096
:108FB000F363800004804100F06388000364800054
:108FC000E08149000364880080CCBF0081ECB700D9
:108FD0007FCCBF0080ECB7007ECCBF007FECB70039
:108FE0007E6CEF000EDABF00E9F9B70044CF8000D5
:108FF0004822DE00F363800004804100F0638800B3
:1090000003648000E0814900036488003D68AE008D
:109010001F0037000100200001007800C624020074
:10902000000000008100E8003322AF00FEFF37009F
:10903000A0118800900020000008E600F6FF37002D
:109040000064800041702200303C020000000000FB
:10905000F063800041702200303C020000000000FC
:109060003322AF00FEFF370004022000A411880065
:109070003322AF00FEFF3700A4002000A4118800B7
:109080003322AF00FEFF3700D4002000A411880077
:1090900019DABF00E6F9B700E6D9BF0082ECB700E5
:1090A000836CEF00842CEF0084CCBF0085ECB7000C
:1090B00083CCBF0084ECB70082CCBF0083ECB70048
:1090C000826CEF0018DABF00E7F9B70034CF8000F8
:1090D0004822DE0013648000048041001064880090
:1090E00023648000E08149002364880084CCBF00B1
:1090F00085ECB70083CCBF0084ECB70082CCBF0006
:1091000083ECB700826CEF0017DABF00E8F9B70014
:1091100044CF80000960EF001364800004804100A8
:109120001064880023648000E08149002364880083
:1091300084CCBF0085ECB70083CCBF0084ECB700C3
:1091400082CCBF0083ECB700826CEF0016DABF0060
:10915000E9F9B70044CF80004822DE0013648000A4
:10916000048041001064880023648000E08149008D
:10917000236488003D68AE001F0037000100200016
:1091800001007800E4240200000000008100E800F3
:109190003322AF00FEFF3700A0118800000120003D
:1091A0000008E600F6FF37002064800041702200CE
:1091B000303C02000000000010648000417022007A
:1091C000303C0200000000003322AF00FEFF3700F9
:1091D00004022000A41188003322AF00FEFF3700F4
:1091E000A4002000A41188003322AF00FEFF370046
:1091F000D4002000A411880045CBBF000160EF001F
:10920000010020000001780081017800F0638000F7
:10921000016480006C42020000000000906488003D
:10922000A164880090648000760CB400906488008B
:10923000C4638000A364800004804900A0648800A7
:109240003D68AE001F0037000100200001007800DB
:1092500086240200000000008100E8003322AF00F5
:10926000FEFF3700A0118800A00020000008E600E3
:10927000F6FF3700A064800041702200303C0200FD
:10928000000000009064800041702200303C020029
:10929000000000003322AF00FEFF37000402200070
:1092A000A41188003322AF00FEFF3700A400200085
:1092B000A41188003322AF00FEFF3700D400200045
:1092C000A411880090648000A1648000D2638000B3
:1092D000E36380006C42020000000000D06488005C
:1092E000E16488003D68AE001F00370001002000E7
:1092F0000100780008250200000000008100E8005D
:109300003322AF00FEFF3700A0118800A00020002C
:109310000008E600F6FF3700E0648000417022009C
:10932000303C020000000000D06480004170220048
:10933000303C0200000000003322AF00FEFF370087
:1093400004022000A41188003322AF00FEFF370082
:10935000A4002000A41188003322AF00FEFF3700D4
:10936000D4002000A4118800E45980004822DE00C7
:109370009364800004804100B0648800A36480008E
:10938000E0814900C36488003D68AE001F003700DB
:109390000100200001007800A42402000000000069
:1093A0008100E8003322AF00FEFF3700A0118800E3
:1093B000D00020000008E600F6FF3700C0648000FF
:1093C00041702200303C020000000000B0648000C8
:1093D00041702200303C0200000000003322AF0048
:1093E000FEFF370004022000A41188003322AF00E2
:1093F000FEFF3700A4002000A41188003322AF0034
:10940000FEFF3700D4002000A4118800920CF80061
:109410008E0CF900940CF800900CF900D4638000D5
:1094200004A0B20002003A007C0CE2000C00320002
:109430000100200001007800262502000000000045
:109440008100E8003322AF00FEFF3700A011880042
:10945000800120000008E600F6FF37000000FE0053
:10946000CF02780000000600851F780055E48000D8
:10947000C32ADD00907CEF000540780091FCB70026
:1094800046360200000000008B7CEF0054E48000B0
:109490004822DE007B24E1000700320000C2B30056
:1094A0008EFCB700B03A0200000000008B7CEC009C
:1094B000464A040000000000CF02780000000600C9
:1094C000851F7800C500200003000900B51F780043
:1094D000800378008404780004F0A1000400E00018
:1094E00006003A0009F0A70002003700050020003E
:1094F0000F003700050020000D003700E642520043
:109500000A0039000003200009F0A6000002200034
:109510003322AF00FEFF3700A01188008502E9006A
:10952000FBFF3B005500200001003700840278005B
:109530006400200005E0A00009F0A70005F0A000ED
:1095400008712200110009008883D800DA4A02005D
:109550000000000081037800883E2000110009000F
:109560008883D800DA4A02000000000081037800F6
:1095700048062000110009008883D800DA4A02005A
:109580000000000081037800A800200011000900FD
:109590008883D800DA4A020000000000000320009F
:1095A00000C040003322AF00FEFF3700A01188004A
:1095B00017003700060320000000E0000E003A000C
:1095C00005E0A6000D0037000402E9000524E100D3
:1095D000020032004200AF00000006000000E00080
:1095E00005003A0005E0A6000400370005F0A600DB
:1095F000060220000100370005E0A1000040430002
:109600003322AF00FEFF3700A011880000000600E3
:109610002501200003000900CF127800CF02780056
:1096200000000600851F7800861F78000001EB000F
:109630000103780064C110004211DD000200DD006A
:10964000800278000C60EC000C60ED000D00320030
:1096500005007800C42ADD004C00DE00F000B200F6
:109660000003B000A20320000200E1000100390065
:109670000D40B4008EFCB700B03A020000000000BC
:10968000F1FF37004F037800CF027800000006009A
:10969000861F7800871F7800881F7800891F780050
:1096A0000002EB008002EB000003EB008003EB0004
:1096B0000304690011003200080220004200A900E2
:1096C0000080D2008180D2000482D2008582D20044
:1096D0000328E10001003A0002A0E1000300390084
:1096E0000202520083825A004200A8000683D20080
:1096F0008783D2000804E900F0FF3A008700780071
:1097000006007800CF0478004F047800CF0378007B
:109710004F03780000000600851F7800C500200078
:1097200003000900B51F780000037800810378006A
:109730000406780004F0A1000400E00006003A00EE
:1097400009F0A700020037000500200013003700D1
:109750000500200011003700EB4252000E003900D6
:109760000003200009F0A600000220003322AF0011
:10977000FEFF3700A011880041E0AF00FBFF37007B
:10978000801088001162EF008502E900F7FF3B00BE
:1097900055002000010037008402780008012000F5
:1097A000090020001000FA000C377C000884E90052
:1097B000FDFF3B00B400200005E0A0000CF0A70076
:1097C00005F0A000040F7800150798000600780047
:1097D0008700780002A02C00A3B9230008712200A2
:1097E0000DF0A1000DF0A200484B020000000000A7
:1097F0000DF0A700070037004007980051079800B8
:1098000000017800810178002E009000BE009000D9
:10981000F4FF370042079800530798002407980088
:10982000350798001E0278009E0290000603200073
:109830000000E00012003A0005E0A6001200370028
:109840000402E900040F78000400E0000E0032007A
:109850000524E100020032004200AF000E00370094
:10986000060320000000E00005003A0005E0A60025
:109870000500370005F0A6000602200002003700B0
:1098800005E0A10015079800004043003322AF0017
:10989000FEFF3700A01188004E009000DE0090000F
:1098A000A20020008001EB006100E1000100320015
:1098B000CCFF37000080FA002501200003000900DA
:1098C000CF127800CF02780000000600811F7800D8
:1098D00081C58000805878008048EB00CF00780078
:1098E000B038EC0000000600851F7800A81CF800C6
:1098F000AC1CF90060E580001004E00014003200A8
:10990000AA1CF800AE1CF90070E580001004E0000D
:109910000C00320060E580009042780070E5800025
:1099200010407800002CE10003003A00AC1CF80065
:109930000000F90007003700AE3CEC00844C040046
:1099400000000000AC3CEC007A4C04000000000079
:109950000020EF00CF02780000000600851F78008D
:109960000200200001CA2100020078004A330200F0
:1099700000000000805878000201E8000004E000C8
:109980004220AE00F8FF37009E1CF800A41CF9002E
:109990009E1CF800A81CF90004CA210054E58800A8
:1099A000744C02000000000010E5880010E5800003
:1099B0009E1CE30003003A009E3CEC002E4D040088
:1099C00000000000A21CE20019003A00F0E4800050
:1099D0001004E0000800320020E58000A43CEC0008
:1099E00080027800F0E480009E3CEC00904A780011
:1099F000E64C040000000000A43CED0020E58000DF
:109A00001042780004C2B20004003A0025E580004C
:109A1000804AEB00144D040000000000A43CEC0060
:109A200025E58000804AEB002E4D04000000000078
:109A300010E580009E1CE3000800320020E5800055
:109A4000A43CEC0080027800F0E480009E3CEC0036
:109A5000904A7800184D040000000000A21CE200AB
:109A6000CBFF3A00A41CF8009E1CF900CF0278003E
:109A700000000600851F7800A25CE2001F00320093
:109A8000F0E480009042780000E58000104078000B
:109A9000002CE1000D003200F0E4800090427800DC
:109AA00000E5800010407800002CE1000300310048
:109AB00000C0EB00604D04000000000010C0B300C7
:109AC0000F003700704D040000000000F0E480003B
:109AD0001004E00002003A000060EF0008003700C8
:109AE000F0E480009E3CEC0000E58000A03CEC002F
:109AF000A27CED003C4D0400000000000060EF007F
:109B0000CF02780000000600851F78009E1CF80038
:109B1000A41CF900A25CE2000C00320000E5800009
:109B20001004E0000900320020E58000A43CEC00B5
:109B30008002780000E58000A03CEC00904A7800AC
:109B4000A27CED008A4D040000000000A25CE2004F
:109B50000700320020E58000A43CEC008002780081
:109B6000804AEB00A27CED00A64D0400000000003E
:109B70009E1CF8000000F900CF02780000000600EB
:109B8000851F7800861F7800A63CEF00A23CEF00FE
:109B9000A400200024E58800A03CEF009E1CE20009
:109BA00002003A000020EF00C400370030E58000DA
:109BB000A63CEC0080027800050078009E1CB400F2
:109BC00044E580000042900044E5880044E58000C0
:109BD000D4C2B2000C003A001400200014E5880042
:109BE00030E58000A63CEC0080027800050078009B
:109BF0009E1CB40044E580000042900044E58800CB
:109C00001A4E04000000000044E58000B4C2B20017
:109C100008003A0030E58000A63CEC0080027800A5
:109C2000050078009E1CB40044E5800000429000CE
:109C300044E5880044E5800003032000041CE100A3
:109C400092003E0044E5800093032000041CE100E4
:109C50008E00390044E5800004C3B20015003A00CC
:109C600030E580009E1CB4001042780084C7B2002A
:109C70000500320030E580009E1CB40010427800E0
:109C800084C5B2000B003A000401200024E58800DE
:109C9000A63CEC0030E58000A63CEC008002780099
:109CA000050078009E1CB40044E58000004290004E
:109CB00044E5880024E580006A20E1001E003A00A7
:109CC00044E5800003032000041CE10018003E006E
:109CD00044E5800093032000041CE10014003900D7
:109CE00004E580006A20B8008002780044E5800026
:109CF0000443B1000440780000E0B7000080FB009E
:109D00000500400000E5880030E58000A63CEC003E
:109D100080027800050078009E1CB40044E58000B5
:109D20000042900044E58800604E040000000000FE
:109D3000464F04000000000024E580007020E10090
:109D400052003A0044E5800013062000041CE100A4
:109D500007003E0044E58000A3072000041CE1004A
:109D600003003900A8DCBF00F04DB200010037004D
:109D7000A8DCBF00A8FCB70044E580000303200076
:109D8000041CE10005003E0044E580009303200030
:109D9000041CE100010039000800370044E58000A0
:109DA00013042000041CE10038003E0044E580005C
:109DB00063042000041CE1003400390044E5800005
:109DC00003032000041CE1000F003E0044E5800076
:109DD00093032000041CE1000B00390005E580001E
:109DE000C42ADD0044E580000443B100044078004B
:109DF00000E0B7000080FB000500400000E588009F
:109E0000184F04000000000005E58000C42ADD00B2
:109E100044E580001444B1000440780000E0B7003D
:109E20006A4040000080FB000500400000E588001B
:109E300030E58000A63CEC00800278000500780048
:109E40009E1CB40044E580000042900044E5880078
:109E500044E5800013062000041CE10007003E00DA
:109E600044E58000A3072000041CE1000300390042
:109E7000A8DCBF00F04DB20001003700A8DCBF0035
:109E8000A8FCB700BC4E04000000000014E58000F0
:109E90006120E10007003A0024E580006A20E1002B
:109EA00004003A000400200003E580000300520093
:109EB00000E58800A01CF8000000F9004F037800BE
:109EC000CF02780000000600C1C8210002AC2000CB
:109ED000B24878003104E0004220AE00FCFF3700B9
:109EE000C4C82100F4E48800AE4C02000000000069
:109EF00002002000A1AF2000020078005E2F0200C7
:109F000000000000805878000201E8000004E00032
:109F10004220AE00F8FF3700C0C0B300A2FCB7007B
:109F2000C4C82100F4E48800A4AF200004E5880040
:109F30003A4D0200000000008AFCB7008A5CE20093
:109F400002003A000060EF000A043700020020001F
:109F5000A1AF200002007800782F0200000000006E
:109F6000805878000201E8000004E0004220AE00C2
:109F7000F8FF3700C0C0B300A2FCB700C4C821007E
:109F8000F4E48800A4AF200004E588003A4D020004
:109F9000000000008AFCB7008A5CE20003003A007F
:109FA00010C0B30000E0B700F20337000200200049
:109FB00061B1200002007800922F02000000000032
:109FC000805878000201E8000004E0004220AE0062
:109FD000F8FF370060C0B300A2FCB70064B12000F6
:109FE000F4E48800C4C8210004E588003A4D02006A
:109FF000000000008AFCB7008A5CE20003003A001F
:10A0000020C0B30000E0B700DA03370002002000F0
:10A0100061B1200002007800A62F020000000000BD
:10A02000805878000201E8000004E0004220AE0001
:10A03000F8FF370060C0B300A2FCB70064B1200095
:10A04000F4E48800C4C8210004E588003A4D020009
:10A05000000000008AFCB7008A5CE20003003A00BE
:10A0600030C0B30000E0B700C20337000200200098
:10A0700061B1200002007800BA2F02000000000049
:10A08000805878000201E8000004E0004220AE00A1
:10A09000F8FF370060C0B300A2FCB70064B1200035
:10A0A000F4E48800C4C8210004E588003A4D0200A9
:10A0B000000000008AFCB7008A5CE20003003A005E
:10A0C00040C0B30000E0B700AA0337000200200040
:10A0D00061B1200002007800CE2F020000000000D5
:10A0E000805878000201E8000004E0004220AE0041
:10A0F000F8FF370060C0B300A2FCB70064B12000D5
:10A10000F4E48800C4C8210004E588003A4D020048
:10A11000000000008AFCB7008A5CE20003003A00FD
:10A1200050C0B30000E0B7009203370002002000E7
:10A1300061B1200002007800E22F02000000000060
:10A14000805878000201E8000004E0004220AE00E0
:10A15000F8FF370060C0B300A2FCB70064B1200074
:10A16000F4E48800C4C8210004E588003A4D0200E8
:10A17000000000008AFCB7008A5CE20003003A009D
:10A1800060C0B30000E0B7007A033700020020008F
:10A1900061B1200002007800F62F020000000000EC
:10A1A000805878000201E8000004E0004220AE0080
:10A1B000F8FF370060C0B300A2FCB70064B1200014
:10A1C000F4E48800C4C8210004E588003A4D020088
:10A1D000000000008AFCB7008A5CE20003003A003D
:10A1E00070C0B30000E0B700620337000200200037
:10A1F00061B12000020078000A3002000000000077
:10A20000805878000201E8000004E0004220AE001F
:10A21000F8FF370060C0B300A2FCB70064B12000B3
:10A22000F4E48800C4C8210004E588003A4D020027
:10A23000000000008AFCB7008A5CE20003003A00DC
:10A2400080C0B30000E0B7004A03370002002000DE
:10A2500061B12000020078001E3002000000000002
:10A26000805878000201E8000004E0004220AE00BF
:10A27000F8FF370050C0B300A2FCB70064B1200063
:10A28000F4E48800C4C8210004E588003A4D0200C7
:10A29000000000008AFCB7008A5CE20003003A007C
:10A2A00090C0B30000E0B700320337000200200086
:10A2B00061B1200002007800303002000000000090
:10A2C000805878000201E8000004E0004220AE005F
:10A2D000F8FF370060C0B300A2FCB70064B12000F3
:10A2E000F4E48800C4C8210004E588003A4D020067
:10A2F000000000008AFCB7008A5CE20003003A001C
:10A30000A0C0B30000E0B7001A033700020020002D
:10A3100061B120000200780044300200000000001B
:10A32000805878000201E8000004E0004220AE00FE
:10A33000F8FF370050C0B300A2FCB70064B12000A2
:10A34000F4E48800C4C8210004E588003A4D020006
:10A35000000000008AFCB7008A5CE20003003A00BB
:10A36000B0C0B30000E0B7000203370002002000D5
:10A3700061B12000020078005630020000000000A9
:10A38000805878000201E8000004E0004220AE009E
:10A39000F8FF370060C0B300A2FCB70064B1200032
:10A3A000F4E48800C4C8210004E588003A4D0200A6
:10A3B000000000008AFCB7008A5CE20003003A005B
:10A3C000C0C0B30000E0B700EA023700020020007E
:10A3D00061B12000020078006A3002000000000035
:10A3E000805878000201E8000004E0004220AE003E
:10A3F000F8FF370060C0B300A2FCB70064B12000D2
:10A40000F4E48800C4C8210004E588003A4D020045
:10A41000000000008AFCB7008A5CE20003003A00FA
:10A42000D0C0B30000E0B700D20237000200200025
:10A4300061B12000020078007E30020000000000C0
:10A44000805878000201E8000004E0004220AE00DD
:10A45000F8FF370060C0B300A2FCB70064B1200071
:10A46000F4E48800C4C8210004E588003A4D0200E5
:10A47000000000008AFCB7008A5CE20003003A009A
:10A48000E0C0B30000E0B700BA02370002002000CD
:10A4900061B120000200780092300200000000004C
:10A4A000805878000201E8000004E0004220AE007D
:10A4B000F8FF370060C0B300A2FCB70064B1200011
:10A4C000F4E48800C4C8210004E588003A4D020085
:10A4D000000000008AFCB7008A5CE20003003A003A
:10A4E000F0C0B30000E0B700A20237000200200075
:10A4F00061B1200002007800A630020000000000D8
:10A50000805878000201E8000004E0004220AE001C
:10A51000F8FF370050C0B300A2FCB70064B12000C0
:10A52000F4E48800C4C8210004E588003A4D020024
:10A53000000000008AFCB7008A5CE20003003A00D9
:10A5400000C1B30000E0B7008A023700020020001B
:10A5500061B1200002007800B83002000000000065
:10A56000805878000201E8000004E0004220AE00BC
:10A57000F8FF370050C0B300A2FCB70064B1200060
:10A58000F4E48800C4C8210004E588003A4D0200C4
:10A59000000000008AFCB7008A5CE20003003A0079
:10A5A00010C1B30000E0B7007202370002002000C3
:10A5B00061B1200002007800CA30020000000000F3
:10A5C000805878000201E8000004E0004220AE005C
:10A5D000F8FF370060C0B300A2FCB70064B12000F0
:10A5E000F4E48800C4C8210004E588003A4D020064
:10A5F000000000008AFCB7008A5CE20003003A0019
:10A6000020C1B30000E0B7005A023700020020006A
:10A6100061B1200002007800DE300200000000007E
:10A62000805878000201E8000004E0004220AE00FB
:10A63000F8FF370060C0B300A2FCB70064B120008F
:10A64000F4E48800C4C8210004E588003A4D020003
:10A65000000000008AFCB7008A5CE20003003A00B8
:10A6600030C1B30000E0B700420237000200200012
:10A6700061B1200002007800F2300200000000000A
:10A68000805878000201E8000004E0004220AE009B
:10A69000F8FF370060C0B300A2FCB70064B120002F
:10A6A000F4E48800C4C8210004E588003A4D0200A3
:10A6B000000000008AFCB7008A5CE20003003A0058
:10A6C00040C1B30000E0B7002A02370002002000BA
:10A6D00061B1200002007800063102000000000095
:10A6E000805878000201E8000004E0004220AE003B
:10A6F000F8FF370060C0B300A2FCB70064B12000CF
:10A70000F4E48800C4C8210004E588003A4D020042
:10A71000000000008AFCB7008A5CE20003003A00F7
:10A7200050C1B30000E0B700120237000200200061
:10A7300061B12000020078001A3102000000000020
:10A74000805878000201E8000004E0004220AE00DA
:10A75000F8FF370050C0B300A2FCB70064B120007E
:10A76000F4E48800C4C8210004E588003A4D0200E2
:10A77000000000008AFCB7008A5CE20003003A0097
:10A7800060C1B30000E0B700FA013700020020000A
:10A7900061B12000020078002C31020000000000AE
:10A7A000805878000201E8000004E0004220AE007A
:10A7B000F8FF370050C0B300A2FCB70064B120001E
:10A7C000F4E48800C4C8210004E588003A4D020082
:10A7D000000000008AFCB7008A5CE20003003A0037
:10A7E00070C1B30000E0B700E201370002002000B2
:10A7F00061B12000020078003E310200000000003C
:10A80000805878000201E8000004E0004220AE0019
:10A81000F8FF370050C0B300A2FCB70064B12000BD
:10A82000F4E48800C4C8210004E588003A4D020021
:10A83000000000008AFCB7008A5CE20003003A00D6
:10A8400080C1B30000E0B700CA0137000200200059
:10A8500061B12000020078005031020000000000C9
:10A86000805878000201E8000004E0004220AE00B9
:10A87000F8FF370050C0B300A2FCB70064B120005D
:10A88000F4E48800C4C8210004E588003A4D0200C1
:10A89000000000008AFCB7008A5CE20003003A0076
:10A8A00090C1B30000E0B700B20137000200200001
:10A8B00061B1200002007800623102000000000057
:10A8C000805878000201E8000004E0004220AE0059
:10A8D000F8FF370060C0B300A2FCB70064B12000ED
:10A8E000F4E48800C4C8210004E588003A4D020061
:10A8F000000000008AFCB7008A5CE20003003A0016
:10A90000A0C1B30000E0B7009A01370002002000A8
:10A9100061B12000020078007631020000000000E2
:10A92000805878000201E8000004E0004220AE00F8
:10A93000F8FF370060C0B300A2FCB70064B120008C
:10A94000F4E48800C4C8210004E588003A4D020000
:10A95000000000008AFCB7008A5CE20003003A00B5
:10A96000B0C1B30000E0B700820137000200200050
:10A9700061B12000020078008A310200000000006E
:10A98000805878000201E8000004E0004220AE0098
:10A99000F8FF370060C0B300A2FCB70064B120002C
:10A9A000F4E48800C4C8210004E588003A4D0200A0
:10A9B000000000008AFCB7008A5CE20003003A0055
:10A9C000C0C1B30000E0B7006A01370002002000F8
:10A9D00061B12000020078009E31020000000000FA
:10A9E000805878000201E8000004E0004220AE0038
:10A9F000F8FF370050C0B300A2FCB70064B12000DC
:10AA0000F4E48800C4C8210004E588003A4D02003F
:10AA1000000000008AFCB7008A5CE20003003A00F4
:10AA2000D0C1B30000E0B70052013700020020009F
:10AA300061B1200002007800B03102000000000087
:10AA4000805878000201E8000004E0004220AE00D7
:10AA5000F8FF370060C0B300A2FCB70064B120006B
:10AA6000F4E48800C4C8210004E588003A4D0200DF
:10AA7000000000008AFCB7008A5CE20003003A0094
:10AA8000E0C1B30000E0B7003A0137000200200047
:10AA900061B1200002007800C43102000000000013
:10AAA000805878000201E8000004E0004220AE0077
:10AAB000F8FF370050C0B300A2FCB70064B120001B
:10AAC000F4E48800C4C8210004E588003A4D02007F
:10AAD000000000008AFCB7008A5CE20003003A0034
:10AAE000F0C1B30000E0B7002201370002002000EF
:10AAF00061B1200002007800D631020000000000A1
:10AB0000805878000201E8000004E0004220AE0016
:10AB1000F8FF370050C0B300A2FCB70064B12000BA
:10AB2000F4E48800C4C8210004E588003A4D02001E
:10AB3000000000008AFCB7008A5CE20003003A00D3
:10AB400000C2B30000E0B7000A0137000200200095
:10AB500061B1200002007800E8310200000000002E
:10AB6000805878000201E8000004E0004220AE00B6
:10AB7000F8FF370060C0B300A2FCB70064B120004A
:10AB8000F4E48800C4C8210004E588003A4D0200BE
:10AB9000000000008AFCB7008A5CE20003003A0073
:10ABA00010C2B30000E0B700F2003700020020003E
:10ABB00061B1200002007800FC31020000000000BA
:10ABC000805878000201E8000004E0004220AE0056
:10ABD000F8FF370050C0B300A2FCB70064B12000FA
:10ABE000F4E48800C4C8210004E588003A4D02005E
:10ABF000000000008AFCB7008A5CE20003003A0013
:10AC000020C2B30000E0B700DA00370002002000E5
:10AC100061B12000020078000E3202000000000046
:10AC2000805878000201E8000004E0004220AE00F5
:10AC3000F8FF370060C0B300A2FCB70064B1200089
:10AC4000F4E48800C4C8210004E588003A4D0200FD
:10AC5000000000008AFCB7008A5CE20003003A00B2
:10AC600030C2B30000E0B700C2003700020020008D
:10AC700061B12000020078002232020000000000D2
:10AC8000805878000201E8000004E0004220AE0095
:10AC9000F8FF370060C0B300A2FCB70064B1200029
:10ACA000F4E48800C4C8210004E588003A4D02009D
:10ACB000000000008AFCB7008A5CE20003003A0052
:10ACC00040C2B30000E0B700AA0037000200200035
:10ACD00061B120000200780036320200000000005E
:10ACE000805878000201E8000004E0004220AE0035
:10ACF000F8FF370060C0B300A2FCB70064B12000C9
:10AD0000F4E48800C4C8210004E588003A4D02003C
:10AD1000000000008AFCB7008A5CE20003003A00F1
:10AD200050C2B30000E0B7009200370002002000DC
:10AD300061B12000020078004A32020000000000E9
:10AD4000805878000201E8000004E0004220AE00D4
:10AD5000F8FF370050C0B300A2FCB70064B1200078
:10AD6000F4E48800C4C8210004E588003A4D0200DC
:10AD7000000000008AFCB7008A5CE20003003A0091
:10AD800060C2B30000E0B7007A0037000200200084
:10AD900061B12000020078005C3202000000000077
:10ADA000805878000201E8000004E0004220AE0074
:10ADB000F8FF370050C0B300A2FCB70064B1200018
:10ADC000F4E48800C4C8210004E588003A4D02007C
:10ADD000000000008AFCB7008A5CE20003003A0031
:10ADE00070C2B30000E0B70062003700020020002C
:10ADF00061B12000020078006E3202000000000005
:10AE0000805878000201E8000004E0004220AE0013
:10AE1000F8FF370050C0B300A2FCB70064B12000B7
:10AE2000F4E48800C4C8210004E588003A4D02001B
:10AE3000000000008AFCB7008A5CE20003003A00D0
:10AE400080C2B30000E0B7004A00370002002000D3
:10AE500061B1200002007800803202000000000092
:10AE6000805878000201E8000004E0004220AE00B3
:10AE7000F8FF370050C0B300A2FCB70064B1200057
:10AE8000F4E48800C4C8210004E588003A4D0200BB
:10AE9000000000008AFCB7008A5CE20003003A0070
:10AEA00090C2B30000E0B70032003700020020007B
:10AEB00061B1200002007800923202000000000020
:10AEC000805878000201E8000004E0004220AE0053
:10AED000F8FF370060C0B300A2FCB70064B12000E7
:10AEE000F4E48800C4C8210004E588003A4D02005B
:10AEF000000000008AFCB7008A5CE20003003A0010
:10AF0000A0C2B30000E0B7001A00370030C0B300A1
:10AF1000A2FCB700A4C92100F4E48800C4C8210041
:10AF200004E58800844D020000000000A4C921004F
:10AF3000F4E48800C04D0200000000008BFCB70064
:10AF400054E480004822DE0023032000041CE100BA
:10AF500007003E0054E480004822DE003306200053
:10AF6000041CE100020039008BDCBF000100370047
:10AF700000E0EF0000000600851F7800861F7800C3
:10AF8000871F7800881F78003DC8A9007068AF004F
:10AF90000D0037000100200001007800702402003D
:10AFA000000000008100E8003322AF00FEFF370000
:10AFB000A0118800700020000008E600F6FF3700AE
:10AFC000C0590400000000007068AE00EC003700BB
:10AFD0009E0CF800961EF900A00CF800981EF900CF
:10AFE000740020000960EF00B5F48000C6F4800012
:10AFF0000402E8000402E900030032000603D10065
:10B000008582D300FBFF370005007800760CB40082
:10B0100090F48800C463800004004B00A0F4880012
:10B02000921EF800A21EF900941EF800A41EF9005A
:10B03000E4C8210034F58800B4410200000000009B
:10B04000740020000960EF00B5F48000C6F48000B1
:10B050000402E8000402E900030032000603D10004
:10B060008582D300FBFF3700740020000960EF00E9
:10B0700005007800860078000402E8000402E90078
:10B08000030032000000D0008180D200FBFF3700B7
:10B09000B4F4800080035200C4F4800001045A001C
:10B0A000F7F4880008F588009E3ED400A0BED600C4
:10B0B0009E3ED400A0BED6009E1EF8008E1EF90053
:10B0C000A01EF800901EF90084F480006020E100CA
:10B0D000A9003E000400390074F48000C31F200062
:10B0E0000418E100A400390074F4800063024200F7
:10B0F0008402780084F4800060024A00040378002F
:10B10000E4C821000480420060034B008600780000
:10B1100054E480000042900054E488008ADCBF00C0
:10B120009AFEB7009B7EEF009C3EEF009CDEBF00C6
:10B130009DFEB7009BDEBF009CFEB7009ADEBF00FD
:10B140009BFEB7009A7EEF0074F48000620242001A
:10B150008402780084F4800060024A0004037800CE
:10B16000E4C821000480420060034B0086007800A0
:10B17000104078008BFCB70054E480004822DE00C9
:10B18000D3F4800004804100D0F48800E3F4800010
:10B19000E0814900E3F488009CDEBF009DFEB7001B
:10B1A0009BDEBF009CFEB7009ADEBF009BFEB7008F
:10B1B0009A7EEF0074F480006102420084027800FD
:10B1C00084F4800060024A0004037800E4C821008F
:10B1D0000480420060034B008600780064E4800035
:10B1E0000042900064E4880064E480000960EF009D
:10B1F000D3F4800004804100D0F48800E3F48000A0
:10B20000E0814900E3F488009CDEBF009DFEB700AA
:10B210009BDEBF009CFEB7009ADEBF009BFEB7001E
:10B220009A7EEF00E4C8210073F48000048041009E
:10B2300084F4800060024A008400780010407800A6
:10B240008DFCB70064E480004822DE00D3F4800067
:10B2500004804100D0F48800E3F48000E0814900DC
:10B26000E3F48800D4F48000F3FF2F000418E10019
:10B2700006003A00E4F48000F3FF20000418E10027
:10B2800002003A000060EF003D003700B4F4800097
:10B290006102420004007800C4F4800060024A00A9
:10B2A000840078009A1EE30003003A00E4F4800072
:10B2B0000120E100240032003DC8A8003D88AE0016
:10B2C0001E0037008042EB003DC8AF008502E80059
:10B2D0000100200001007800B826020000000000F4
:10B2E0008100E8003322AF00FEFF3700A011880084
:10B2F000700020000008E600F6FF370005407800E7
:10B300000160EF0021702200303C020000000000CC
:10B31000A100200001007800B82602000000000013
:10B320008100E8003322AF00FEFF3700A011880043
:10B33000D00020000008E600F6FF370010C0B30080
:10B3400000E0B7000E0037009A1EF800961EF900C4
:10B350009C1EF800981EF90074F4800064024200FC
:10B3600074F4880084F4800060024A0084F4880049
:10B370006458040000000000F057040000000000C2
:10B380004F047800CF0378004F037800CF02780095
:10B3900000000600851F7800861F7800871F780050
:10B3A000881F78001D7CEF007C28EF007E28EF00CE
:10B3B0007168EF007268EF000A3CEF000C3CEF0090
:10B3C0007668EF00A4CF80006124E10016003A0007
:10B3D000907CEF0000C7B30091FCB7004636020036
:10B3E0000000000005002000050078004C25020048
:10B3F000000000000040B3004220AF00050037000D
:10B400008502E8008EFCB700B03A020000000000A0
:10B41000F5FF3700907CEF0080C7B30091FCB700C8
:10B4200046360200000000007068AE0008003700D9
:10B43000760CF800061CF900780CF800081CF900DE
:10B44000820CF8000E1CF900840CF800101CF900A6
:10B45000920CF8001E1CF900940CF800201CF90056
:10B46000163CEF00183CEF007068AE000A00370091
:10B47000E45980004822DE00F3E0800004804100AF
:10B4800040E1880003E18000E081490053E1880049
:10B490006E5A0400000000007068AF000F00370013
:10B4A00065638000C52ADD004300A900050078001F
:10B4B00001002000D2638000E36380009C42020010
:10B4C00000000000F4E080000400400040E188003B
:10B4D00004E180000480480050E188001E1CF80050
:10B4E000021CF900201CF800041CF90010E0800088
:10B4F000281CE30003003A0020E080002A1CE3003F
:10B500007107320094E0800004A0B20004003A0009
:10B51000141CE20002003A00163CEF00183CEF0059
:10B52000021CF800A21EF900041CF800A41EF90079
:10B5300024A0210034F58800B4410200000000007E
:10B54000161CF800121CF900181CF800141CF90055
:10B5500094E0800004A0B20002003A00141CE20053
:10B560005407320024A0210093E0800004804100B1
:10B57000A4E0800060024A008400780004082000F3
:10B580001024E10013003E003D88AE000D0037009E
:10B59000050020000500780064250200000000007E
:10B5A0000040B3004220AF00060037008502E800EB
:10B5B0003322AF00FEFF370034E2B7003562EF0000
:10B5C000F4FF37004869040000000000765F0400C3
:10B5D0000000000094E080006B02420084027800CA
:10B5E000A4E0800060024A000403780024A0210047
:10B5F0000480420060034B00860078001040780011
:10B600006C4060006C04E10013003A003D88AE001D
:10B610000D003700050020000500780078250200A5
:10B62000000000000040B3004220AF0006003700D9
:10B630008502E8003322AF00FEFF370034E2B70096
:10B640003562EF00F4FF3700486904000000000095
:10B65000765F04000000000024A0210093E0800039
:10B6600004804100A4E0800060024A008400780069
:10B670001004E00055003A00E4E080004822DE00BB
:10B680006124E100390039003D88AE000D0037002B
:10B6900005002000050078008C2502000000000055
:10B6A0000040B3004220AF00060037008502E800EA
:10B6B0003322AF00FEFF370034E2B7003562EF00FF
:10B6C000F4FF37001D7CED0094438000614242008E
:10B6D0000440780072E8B7001DDCBF000160EF0095
:10B6E0004200DD00A4C321000400400064C1210029
:10B6F000301A7800301A78001DDCBF000160EF00BE
:10B700004200DD0024C6210004004000E4C1210005
:10B71000301A7800301A780004022000B3E080006C
:10B7200004804100B0E08800C4E0800060024A006C
:10B73000C4E08800B4E0800004A0B20007003A0032
:10B74000181CE20005003A001E3CEC004220AF004D
:10B75000203CEC00163CEF00183CEF00345A04008B
:10B7600000000000E25B0400000000001D5CE2003D
:10B7700014003A003D68AE000D00370005002000BF
:10B7800005007800A0250200000000000040B30082
:10B790004220AF00060037008502E8003322AF00E8
:10B7A000FEFF370034E2B7003562EF00F4FF3700E8
:10B7B00000C2B3008AFCB700344A02000000000057
:10B7C000CD083700765F04000000000094E08000A0
:10B7D0006B02420084027800A4E0800060024A000C
:10B7E0000403780024A021000480420060034B0081
:10B7F00086007800104078007C4060007004E10012
:10B80000BA013A0024A0210093E0800004804100A6
:10B81000A4E0800060024A008400780010427800B2
:10B82000E4C2B20002003A004869040000000000CF
:10B83000F459E20003003A007768EC00465C04002B
:10B8400000000000A4CF80006224E1000F003A0055
:10B850007668EC0075C8BF007648E3000B003A003C
:10B86000E44380006102420004448800F443800005
:10B8700060024A00144488003DE8A90010C0B300EB
:10B88000F4F9B700D2590400000000001DDCBF002D
:10B890000160EF004200DD00A4C3210084024000EB
:10B8A00024C12100B41A7800B41A78001DDCBF004E
:10B8B0000160EF004200DD0024C621008402400048
:10B8C00024C02100B41A7800B41A78001D7CEC0062
:10B8D0007168EC00844380004822DE0083CD2000A4
:10B8E000830242001DDCBF00804A78007268EF00CE
:10B8F000A4CF80006324E100EF003A007548E20025
:10B9000002003A0010C0B30075E8B7007668EC009A
:10B9100075C8BF00B44380000024E1009E003900D8
:10B92000E4E080004822DE006124E10022003900CA
:10B9300002002000C1C2210002007800B4250200EC
:10B9400000000000805878000201E8000004E000D8
:10B950004220AE00F8FF3700017AEF0004D08000EB
:10B960004822DE006824E1001300320004D0800089
:10B970004822DE00C3C221008302420004D08000BE
:10B980004822DE0093E0800004834100A3E08000B1
:10B99000E08149008303780024A0210004004300D3
:10B9A000E0834B0087007800904A7800017AEC0031
:10B9B000AE5C0400000000003D88AE0018003700B7
:10B9C0000100200001007800C225020000000000F4
:10B9D0008100E8003322AF00FEFF3700A01188008D
:10B9E000500020000008E600F6FF370088C8BF00BE
:10B9F0000160EF0004002000604A02000000000027
:10BA00003322AF00FEFF370004022000A41188009B
:10BA10003322AF00FEFF370004022000A41188008B
:10BA20003D88AE001A0037003322AF00FEFF37001A
:10BA3000C4052000A4118800C1C221001104E00047
:10BA4000070032003322AF00FEFF370001409000B4
:10BA500034E2B7003562EF008100E800F7FF3700FD
:10BA60003322AF00FEFF370004022000A41188003B
:10BA70003322AF00FEFF3700A4002000A41188008D
:10BA80003322AF00FEFF3700D4002000A41188004D
:10BA900045448000C32ADD00907CEF00054078001B
:10BAA00091FCB70046360200000000008848E20022
:10BAB00003003A00F4FF200024638800622CEF00AA
:10BAC0003D88AE000B003700010020000100780027
:10BAD000DA250200000000008100E8003322AF00F8
:10BAE000FEFF3700A0118800500020000008E6008B
:10BAF000F6FF370075C8BF008848B4000080FB001F
:10BB000024CB200004004000104378000640780059
:10BB10000160EF0021702200124B020000000000C3
:10BB20001DDCBF0022FCB700225CE20007003200EF
:10BB3000E0C2B3008EFCB700B03A02000000000083
:10BB4000227CED00945D040000000000C0C5B3003D
:10BB50008EFCB700B03A020000000000C1C2210014
:10BB60001104E00008003200811F780001409000BD
:10BB70008EFCB700B03A020000000000CF00780051
:10BB80008100E800F6FF3700642CEF00F4FF20008E
:10BB9000146388008868EC00A44380004822DE001B
:10BBA000634242000440780000E0B7007648E300BA
:10BBB0000300320076C8BF007748E3003E003A0039
:10BBC0003D88AE000B003700010020000100780026
:10BBD000EE250200000000008100E8003322AF00E3
:10BBE000FEFF3700A0118800500020000008E6008A
:10BBF000F6FF3700907CEF0000C4B30091FCB70063
:10BC00004636020000000000050020000500780014
:10BC100002260200000000000040B3004220AF00F6
:10BC2000050037008502E8008EFCB700B03A02003C
:10BC300000000000F5FF37003D88AE000B00370024
:10BC4000010020000100780014260200000000001E
:10BC50008100E8003322AF00FEFF3700A01188000A
:10BC6000500020000008E600F6FF3700B2CCBF000D
:10BC70000160EF0021702200124B02000000000062
:10BC80003D88AE000B003700010020000100780065
:10BC900028260200000000008100E8003322AF00E7
:10BCA000FEFF3700A0118800500020000008E600C9
:10BCB000F6FF370090073700A4CF80006124E10031
:10BCC00002003A0071C8BF0075E8B70094E0800038
:10BCD0007502420084027800A4E0800060024A00FD
:10BCE0000403780024A021000480420060034B007C
:10BCF0008600780010407800F5F9B700F5D9BF004C
:10BD000024FCB700257CEF00263CEF0026DCBF00BA
:10BD100027FCB70025DCBF0026FCB70024DCBF00F1
:10BD200025FCB700247CEF0094E080007402420000
:10BD300084027800A4E0800060024A0004037800D6
:10BD400024A021000480420060034B00860078009C
:10BD5000B4CF800000429000B4CF8800B4CF800000
:10BD60000960EF0023E180000480410020E18800A9
:10BD700033E18000E081490033E1880026DCBF0028
:10BD800027FCB70025DCBF0026FCB70024DCBF0081
:10BD900025FCB700247CEF0094E080007B02420089
:10BDA00084027800A4E0800060024A000403780066
:10BDB00024A021000480420060034B00860078002C
:10BDC00010407800F7F9B700B4CF80004822DE00B9
:10BDD00023E180000480410020E1880033E18000FD
:10BDE000E081490033E1880026DCBF0027FCB70072
:10BDF00025DCBF0026FCB70024DCBF0025FCB70013
:10BE0000247CEF0094E080007A02420084027800F3
:10BE1000A4E0800060024A000403780024A021000E
:10BE20000480420060034B0086007800C4CF80008D
:10BE300000429000C4CF8800C4CF80000960EF00AA
:10BE400023E180000480410020E1880033E180008C
:10BE5000E081490033E1880024E180006200520063
:10BE600020E1880034E1800060005A0030E1880061
:10BE70003DCBBF00000178000560EF00030020000B
:10BE800020E1800031E180006C42020000000000EF
:10BE9000F0E0880001E18800F0E08000960CB4003A
:10BEA000F0E08800C464800003E180000480490061
:10BEB00000E188007068AE0008003700E459800097
:10BEC0004822DE00F3E0800004805100F0E08800AA
:10BED00003E180006080590000E18800163CEF001B
:10BEE000183CEF00345A04000000000094E0800089
:10BEF0006802420084027800A4E0800060024A00E8
:10BF00000403780024A021000480420060034B0059
:10BF100086007800D4E0800000429000D4E08800E1
:10BF200094E080006902420084027800A4E080006E
:10BF300060024A000403780024A02100048042002B
:10BF400060034B0086007800104078001BFCB700AF
:10BF500094E080006A02420084027800A4E080003D
:10BF600060024A000403780024A0210004804200FB
:10BF700060034B0086007800E4E0800000429000FF
:10BF8000E4E08800D4E0800074C7B2000900320009
:10BF9000D4E0800074C5B20006003200D4E0800016
:10BFA00044C7B20003003200D4E0800044C5B200B0
:10BFB000B7043A00D4E080004822DE0014C6B20084
:10BFC0000C003200D4E080004822DE0014C4B2002D
:10BFD00008003200D4E080004822DE0084C7B200AE
:10BFE00004003200D4E080004822DE0084C5B200A4
:10BFF000A7043A00E4E0800064C7B2000900320000
:10C00000E4E0800064C5B20006003200E4E0800095
:10C0100044C7B20003003200E4E0800044C5B2002F
:10C020009B043A00F459E20096033A007828EC00A9
:10C030004220AF007A28EC003D88AE0016003700A1
:10C0400005002000050078003C26020000000000EA
:10C050000040B3004220AF00060037008502E80030
:10C060003322AF00FEFF370034E2B7003562EF0045
:10C07000F4FF3700C0438000D1438000040020005B
:10C080008C4B0200000000003322AF00FEFF37009F
:10C0900004022000A41188003D88AE00180037007B
:10C0A00071C8BF00800278000B60EF00060020001E
:10C0B000010020000100780052260200000000006C
:10C0C0008100E8003322AF00FEFF3700A011880096
:10C0D000A00020000008E600F6FF37000500780009
:10C0E00086007800040020008C4B02000000000055
:10C0F0003322AF00FEFF370004022000A4118800A5
:10C100001D5CE2001D0032007248E2000F003200A8
:10C11000844380004822DE009343800003405200A5
:10C120000080FB0084CD2000040040001040780017
:10C13000E4E080004822DE000024E100030031003A
:10C140007268EC00886004000000000084438000F6
:10C150004822DE0093438000034052000080FB0031
:10C1600024CB2000040340001642780061424200C4
:10C1700004439800CA600400000000001D5CE20057
:10C1800004003A0094658000614242000440780057
:10C19000B2ECB7003D68AE0095003700C0438000A8
:10C1A000D1438000040020008C4B020000000000FE
:10C1B0003322AF00FEFF370004022000A4118800E4
:10C1C00024A0210093E0800004804100A4E08000CE
:10C1D00060024A0084007800904278003322AF0069
:10C1E000FEFF37003402F800E5FF9F003402F9003B
:10C1F0003562EF0094E08000610242008402780022
:10C20000A4E0800060024A000403780024A021001A
:10C210000480420060034B00860078009043780061
:10C220003322AF00FEFF37003402F800E7FF9F0023
:10C230003402F9003562EF0094E0800062024200AF
:10C2400084027800A4E0800060024A0004037800C1
:10C2500024A021000480420060034B008600780087
:10C26000904378003322AF00FEFF37003402F8001D
:10C27000E7FF9F003402F9003562EF0094E0800090
:10C280006302420084027800A4E0800060024A0059
:10C290000403780024A021000480420060034B00C6
:10C2A00086007800904378003322AF00FEFF37000D
:10C2B0003402F800E7FF9F003402F9003562EF0016
:10C2C00094E080006402420084027800A4E08000D0
:10C2D00060024A000403780024A021000480420088
:10C2E00060034B0086007800904378003322AF0053
:10C2F000FEFF37003402F800E7FF9F003402F90028
:10C300003562EF0094E0800065024200840278000C
:10C31000A4E0800060024A000403780024A0210009
:10C320000480420060034B00860078009043780050
:10C330003322AF00FEFF37003402F800E7FF9F0012
:10C340003402F9003562EF0094E08000660242009A
:10C3500084027800A4E0800060024A0004037800B0
:10C3600024A021000480420060034B008600780076
:10C37000904378003322AF00FEFF37003402F8000C
:10C38000E7FF9F003402F9003562EF0094E080007F
:10C390006702420084027800A4E0800060024A0044
:10C3A0000403780024A021000480420060034B00B5
:10C3B00086007800904378003322AF00FEFF3700FC
:10C3C0003402F800E7FF9F003402F9003562EF0005
:10C3D0003322AF00FEFF370004022000A4118800C2
:10C3E0003322AF00FEFF370004022000A4118800B2
:10C3F0007048AE00A102370024A0210093E0800025
:10C4000004804100A4E0800060024A0084007800BB
:10C4100010407800F5F9B700F5D9BF009CF8B700D7
:10C420009D78EF009E38EF009ED8BF009FF8B700C0
:10C430009DD8BF009EF8B7009CD8BF009DF8B700FC
:10C440009C78EF0094E08000610242008402780052
:10C45000A4E0800060024A000403780024A02100C8
:10C460000480420060034B0086007800B4CF800057
:10C4700000429000B4CF8800B4CF80000960EF0084
:10C48000E3C4800004804100E0C48800F3C480005D
:10C49000E0814900F3C488009ED8BF009FF8B70030
:10C4A0009DD8BF009EF8B7009CD8BF009DF8B7008C
:10C4B0009C78EF0094E080006202420084027800E1
:10C4C000A4E0800060024A000403780024A0210058
:10C4D0000480420060034B00860078001040780022
:10C4E000F7F9B700B4CF80004822DE00E3C4800033
:10C4F00004804100E0C48800F3C48000E08149006A
:10C50000F3C488009ED8BF009FF8B7009DD8BF0035
:10C510009EF8B7009CD8BF009DF8B7009C78EF004C
:10C5200094E080006302420084027800A4E080006E
:10C5300060024A000403780024A021000480420025
:10C5400060034B0086007800C4CF8000004290005A
:10C55000C4CF8800C4CF80000960EF00E3C480002E
:10C5600004804100E0C48800F3C48000E0814900F9
:10C57000F3C4880094E080006402420084027800E2
:10C58000A4E0800060024A000403780024A0210097
:10C590000480420060034B00860078001040780061
:10C5A000F9F9B700F9D9BF00A0F8B700A178EF00FA
:10C5B000A238EF00A2D8BF00A3F8B700A1D8BF00EF
:10C5C000A2F8B700A0D8BF00A1F8B700A078EF008C
:10C5D00094E080006502420084027800A4E08000BC
:10C5E00060024A000403780024A021000480420075
:10C5F00060034B0086007800D4CF8000004290009A
:10C60000D4CF8800D4CF80000960EF0003C580003C
:10C610000480410000C5880013C58000E081490006
:10C6200013C58800A2D8BF00A3F8B700A1D8BF00E7
:10C63000A2F8B700A0D8BF00A1F8B700A078EF001B
:10C6400094E080006602420084027800A4E080004A
:10C6500060024A000403780024A021000480420004
:10C6600060034B008600780010407800FBF9B700AB
:10C67000D4CF80004822DE0003C580000480410042
:10C6800000C5880013C58000E081490013C58800FB
:10C69000A2D8BF00A3F8B700A1D8BF00A2F8B70086
:10C6A000A0D8BF00A1F8B700A078EF0094E0800008
:10C6B0006702420084027800A4E0800060024A0021
:10C6C0000403780024A021000480420060034B0092
:10C6D00086007800E4CF800000429000E4CF88001C
:10C6E000E4CF80000960EF0003C5800004804100B2
:10C6F00000C5880013C58000E081490013C588008B
:10C7000094E080006802420084027800A4E0800087
:10C7100060024A000403780024A021000480420043
:10C7200060034B008600780010407800FDF9B700E8
:10C73000FDD9BF00A4F8B700A578EF00A638EF0038
:10C74000A6D8BF00A7F8B700A5D8BF00A6F8B700C5
:10C75000A4D8BF00A5F8B700A478EF0094E080004B
:10C760006902420084027800A4E0800060024A006E
:10C770000403780024A021000480420060034B00E1
:10C7800086007800F4CF800000429000F4CF88004B
:10C79000F4CF80000960EF0023C5800004804100D1
:10C7A00020C5880033C58000E081490033C588007A
:10C7B000A6D8BF00A7F8B700A5D8BF00A6F8B70055
:10C7C000A4D8BF00A5F8B700A478EF0094E08000DB
:10C7D0006A02420084027800A4E0800060024A00FD
:10C7E0000403780024A021000480420060034B0071
:10C7F0008600780010407800FFF9B700F4CF800081
:10C800004822DE0023C580000480410020C5880046
:10C8100033C58000E081490033C58800A6D8BF0039
:10C82000A7F8B700A5D8BF00A6F8B700A4D8BF00E6
:10C83000A5F8B700A478EF0094E080006B024200F6
:10C8400084027800A4E0800060024A0004037800BB
:10C8500024A021000480420060034B008600780081
:10C8600004D080000042900004D0880004D08000F2
:10C870000960EF0023C580000480410020C58800C6
:10C8800033C58000E081490033C5880004AC200036
:10C8900084C58800F5D9BF00664C02000000000086
:10C8A000F6D9BF00664C020000000000F7D9BF00B7
:10C8B000664C020000000000F8D9BF00664C020080
:10C8C00000000000F9D9BF00664C02000000000023
:10C8D000FAD9BF00664C020000000000FBD9BF007F
:10C8E000664C020000000000FCD9BF00664C02004C
:10C8F00000000000E0C2B300664C0200000000002F
:10C90000FDD9BF00664C020000000000FED9BF0048
:10C91000664C020000000000FFD9BF00664C020018
:10C920000000000000DABF00664C020000000000BA
:10C930003D68AE001500370001AC20001104E00096
:10C94000070032003322AF00FEFF370001409000A5
:10C9500034E2B7003562EF008100E800F7FF3700EE
:10C9600021002000010078006E2602000000000077
:10C970008100E8003322AF00FEFF3700A0118800DD
:10C98000500020000008E600F6FF3700644F020068
:10C9900000000000BEEAB700F45580004306200006
:10C9A000041CE10002003900BECABF00BDEAB700A6
:10C9B000BDCABF000160EF004200DD00843E2100DF
:10C9C00084024000C4892100B41A7800B41A7800A7
:10C9D000BDCABF000160EF004200DD0084572100A6
:10C9E00084024000048A2100B41A7800B41A780046
:10C9F000BDCABF000160EF004200DD00847021006D
:10CA000084024000448A2100B41A7800B41A7800E5
:10CA100094E080007502420084027800A4E0800067
:10CA200060024A000403780024A021000480420030
:10CA300060034B008600780010407800F5F9B700DD
:10CA4000F5D9BF0098F8B7009978EF009A38EF0051
:10CA50009AD8BF009BF8B70099D8BF009AF8B700E2
:10CA600098D8BF0099F8B7009878EF0094E080005C
:10CA70007402420084027800A4E0800060024A0050
:10CA80000403780024A021000480420060034B00CE
:10CA900086007800B4CF800000429000B4CF8800B8
:10CAA000B4CF80000960EF00C3C48000048041005F
:10CAB000C0C48800D3C48000E0814900D3C488008A
:10CAC0009AD8BF009BF8B70099D8BF009AF8B70072
:10CAD00098D8BF0099F8B7009878EF0094E08000EC
:10CAE0007B02420084027800A4E0800060024A00D9
:10CAF0000403780024A021000480420060034B005E
:10CB00008600780010407800F7F9B700B4CF8000B5
:10CB10004822DE00C3C4800004804100C0C48800F5
:10CB2000D3C48000E0814900D3C488009AD8BF00F4
:10CB30009BF8B70099D8BF009AF8B70098D8BF0003
:10CB400099F8B7009878EF0094E080007A024200EC
:10CB500084027800A4E0800060024A0004037800A8
:10CB600024A021000480420060034B00860078006E
:10CB7000C4CF800000429000C4CF8800C4CF8000A2
:10CB80000960EF00C3C4800004804100C0C4880075
:10CB9000D3C48000E0814900D3C48800BDCABF006F
:10CBA0000160EF004200DD0084DA200084024000D2
:10CBB00084892100B41A7800B41A7800BDCABF0075
:10CBC0000160EF004200DD0084DA20000400400034
:10CBD000C48A2100301A7800301A780064C58000B9
:10CBE000E202520074C5800060035A003DCBBF00D2
:10CBF000000178000560EF000300200005007800C8
:10CC0000860078006C4202000000000040C58800E9
:10CC100051C5880040C58000960CB40040C588000E
:10CC2000C464800053C580000480490050C588005A
:10CC30007068AE0008003700E45980004822DE002A
:10CC400043C580000480510040C5880053C5800062
:10CC50006080590050C58800BDCABF000160EF0068
:10CC60004200DD0084F3200084024000848A210019
:10CC7000B41A7800B41A780094E080007F02420071
:10CC800084027800A4E0800060024A000403780077
:10CC900024A021000480420060034B00860078003D
:10CCA00010407800F5F9B700F5D9BF0098F8B70043
:10CCB0009978EF009A38EF009AD8BF009BF8B70038
:10CCC00099D8BF009AF8B70098D8BF0099F8B70074
:10CCD0009878EF0094E080007E02420084027800A1
:10CCE000A4E0800060024A000403780024A0210030
:10CCF0000480420060034B0086007800B4CF8000BF
:10CD000000429000B4CF8800B4CF80000960EF00EB
:10CD1000C3C4800004804100C0C48800D3C4800024
:10CD2000E0814900D3C488009AD8BF009BF8B700BF
:10CD300099D8BF009AF8B70098D8BF0099F8B70003
:10CD40009878EF0094E080007D0242008402780031
:10CD5000A4E0800060024A000403780024A02100BF
:10CD60000480420060034B00860078001040780089
:10CD7000F7F9B700B4CF80004822DE00C3C48000BA
:10CD800004804100C0C48800D3C48000E081490011
:10CD9000D3C488009AD8BF009BF8B70099D8BF00C9
:10CDA0009AF8B70098D8BF0099F8B7009878EF00C4
:10CDB00094E080007C02420084027800A4E08000BD
:10CDC00060024A000403780024A02100048042008D
:10CDD00060034B0086007800C4CF800000429000C2
:10CDE000C4CF8800C4CF80000960EF00C3C48000B6
:10CDF00004804100C0C48800D3C48000E0814900A1
:10CE0000D3C48800BDCABF000160EF004200DD004E
:10CE1000840C21008402400084892100B41A780027
:10CE2000B41A7800BDCABF000160EF004200DD0007
:10CE300084DA200004004000E4C92000301A7800A1
:10CE4000301A7800BC57020000000000BDCABF00C5
:10CE50000160EF004200DD008425210084024000D3
:10CE60000000EB003DC8AF000000E800010020001A
:10CE700004002000B41A7800B41A7800486904004D
:10CE800000000000A4CF80006124E100FA003A0015
:10CE90007C28EC004220AF007E28EC00004480009B
:10CEA0007C08E300F2003A00104480007E08E300B2
:10CEB000EF003A0080C2B3008AFCB700344A020097
:10CEC0000000000094E080007502420084027800B7
:10CED000A4E0800060024A000403780024A021003E
:10CEE0000480420060034B00860078001040780008
:10CEF000F5F9B700F5D9BF009EECB7009F6CEF00C5
:10CF0000A02CEF00A0CCBF00A1ECB7009FCCBF00CD
:10CF1000A0ECB7009ECCBF009FECB7009E6CEF006A
:10CF200094E080007402420084027800A4E0800053
:10CF300060024A000403780024A02100048042001B
:10CF400060034B0086007800B4CF80000042900060
:10CF5000B4CF8800B4CF80000960EF00F364800094
:10CF600004804100F064880003658000E08149008E
:10CF700003658800A0CCBF00A1ECB7009FCCBF0028
:10CF8000A0ECB7009ECCBF009FECB7009E6CEF00FA
:10CF900094E080007B02420084027800A4E08000DC
:10CFA00060024A000403780024A0210004804200AB
:10CFB00060034B008600780010407800F7F9B70056
:10CFC000B4CF80004822DE00F3648000048041007A
:10CFD000F064880003658000E081490003658800F3
:10CFE000A0CCBF00A1ECB7009FCCBF00A0ECB70065
:10CFF0009ECCBF009FECB7009E6CEF0094E08000D9
:10D000007A02420084027800A4E0800060024A00B4
:10D010000403780024A021000480420060034B0038
:10D0200086007800C4CF800000429000C4CF880002
:10D03000C4CF80000960EF00F364800004804100E9
:10D04000F064880003658000E08149000365880082
:10D05000F4648000E20252000465800060035A001C
:10D060003DCBBF000160EF0001002000000178000F
:10D070008101780005007800860078006C4202008B
:10D0800000000000F067880001688800F0678000F9
:10D09000960CB400F0678800C464800003688000C8
:10D0A00004804900006888007068AE0008003700FE
:10D0B000E45980004822DE00F367800004805100BC
:10D0C000F06788000368800060805900006888006D
:10D0D00094E080007F02420084027800A4E0800097
:10D0E00060024A000403780024A02100048042006A
:10D0F00060034B008600780010407800F5F9B70017
:10D10000F5D9BF00A6ECB700A76CEF00A82CEF0084
:10D11000A8CCBF00A9ECB700A7CCBF00A8ECB70013
:10D12000A6CCBF00A7ECB700A66CEF0094E080008F
:10D130007E02420084027800A4E0800060024A007F
:10D140000403780024A021000480420060034B0007
:10D1500086007800B4CF800000429000B4CF8800F1
:10D16000B4CF80000960EF00336580000480410087
:10D170003065880043658000E08149004365880090
:10D18000A8CCBF00A9ECB700A7CCBF00A8ECB700A3
:10D19000A6CCBF00A7ECB700A66CEF0094E080001F
:10D1A0007D02420084027800A4E0800060024A0010
:10D1B0000403780024A021000480420060034B0097
:10D1C0008600780010407800F7F9B700B4CF8000EF
:10D1D0004822DE003365800004804100306588000D
:10D1E00043658000E081490043658800A8CCBF000A
:10D1F000A9ECB700A7CCBF00A8ECB700A6CCBF0035
:10D20000A7ECB700A66CEF0094E080007C0242001F
:10D2100084027800A4E0800060024A0004037800E1
:10D2200024A021000480420060034B0086007800A7
:10D23000C4CF800000429000C4CF8800C4CF8000DB
:10D240000960EF003365800004804100306588008C
:10D2500043658000E08149004365880000C2B30057
:10D260008AFCB700344A02000000000022023700A6
:10D270004869040000000000A4CF80006224E1009F
:10D2800003003A007C28EC004220AF007E28EC002E
:10D290000402200093E080000480410090E08800B8
:10D2A000A4E0800060024A00A4E08800A85A0400BC
:10D2B00000000000023CEC004220AF00043CEC0007
:10D2C000765A040000000000F4E0800073648000DF
:10D2D0008302520004E180008364800003035A004B
:10D2E0003DCBBF000160EF000100200014002000D2
:10D2F0000960EF000402E8000402E90003003200C4
:10D300000000D0008180D200FBFF37008503400081
:10D31000068448003DCBBF000160EF000100200003
:10D320004300A9000001780081017800070078001F
:10D33000880078009C4202000000000070E0880035
:10D3400081E088007068AF001B00370014002000E7
:10D350000960EF00D0638000E16380000402E80010
:10D360000402E900030032008100D1000080D300F4
:10D37000FBFF37004300A90000017800810178001D
:10D3800070E0800081E080009C420200000000000C
:10D39000800278000103780005007800760CB40064
:10D3A00030E08800C463800004004B0040E0880047
:10D3B000126A0400000000007068AE001900370017
:10D3C000240020000960EF00D0638000E16380004A
:10D3D0000402E8000402E900030032008100D100E9
:10D3E0000080D300FBFF37004300A9000001780054
:10D3F0008101780070E0800081E080009C420200A2
:10D400000000000080027800010378000500780029
:10D41000760CB40030E08800C463800004004B0048
:10D4200040E088007068AF00B900370001002000BC
:10D430000100780070240200000000008100E80074
:10D440003322AF00FEFF3700A011880070002000DB
:10D450000008E600F6FF3700061CF800A21EF900DF
:10D46000081CF800A41EF90024A0210034F588004F
:10D47000B4410200000000000FDCBF008002780011
:10D4800010DCBF000BE0B70011DCBF000003780028
:10D490000D60EF000640780003E0B7000BC0BF004E
:10D4A000804078000540780001E0B7000040EB00C4
:10D4B00074E080008003520084E0800001045A0080
:10D4C00097E08800A8E08800123CD40014BCD60085
:10D4D00094E080006102420084027800A4E08000B1
:10D4E00060024A000403780024A021000480420066
:10D4F00060034B008600780010407800F5F9B70013
:10D50000F5D9BF000AFCB7000B7CEF000C3CEF0024
:10D510000CDCBF000DFCB7000BDCBF000CFCB7003F
:10D520000ADCBF000BFCB7000A7CEF0024A021003E
:10D5300093E0800004804100A4E0800060024A0083
:10D5400084007800B4CF800000429000B4CF8800FF
:10D55000B4CF80000960EF0053E0800004804100F8
:10D5600050E0880063E08000E081490063E08800CB
:10D5700064E080006020E1006500390004003E00A6
:10D5800054E0800003FF2F000418E10060003E001B
:10D590003D88AE001F003700010020000100780028
:10D5A00082260200000000008100E8003322AF0064
:10D5B000FEFF3700A0118800B00020000008E60040
:10D5C000F6FF370060E0800041702200303C02002E
:10D5D0000000000050E0800041702200303C02005A
:10D5E000000000003322AF00FEFF370004022000DD
:10D5F000A41188003322AF00FEFF3700A4002000F2
:10D60000A41188003322AF00FEFF3700D4002000B1
:10D61000A4118800140020000960EF00D06380008E
:10D62000E16380000402E8000402E9000300320024
:10D630008100D1000080D300FBFF37004300A90028
:10D64000000178008101780050E0800061E08000F6
:10D650009C42020000000000800278000103780074
:10D6600005007800760CB40030E08800C4638000C8
:10D6700004004B0040E088000A1CF8000E1CF90072
:10D680000C1CF800101CF9003DCBBF000160EF003E
:10D6900001002000000178008101780070E0800026
:10D6A00081E080006C4202000000000080027800EF
:10D6B00001037800050078008E0CB4008003780028
:10D6C00006007800908CB400000478003DCBBF00C9
:10D6D0000160EF0001002000140020000960EF004D
:10D6E0000402E8000402E900030032000000D00058
:10D6F0008180D200FBFF370000805300F0E08800FB
:10D7000001005C0000E18800345A040000000000C1
:10D710007068AE00F80037000100200001007800BA
:10D72000A2260200000000008100E8003322AF00C2
:10D73000FEFF3700A0118800700020000008E600FE
:10D74000F6FF3700061CF800A21EF900081CF800BE
:10D75000A41EF90024A0210034F58800B441020081
:10D7600000000000740020000960EF0075E08000F8
:10D7700086E080000402E8000402E90003003200B1
:10D780000603D1008582D300FBFF37007400200020
:10D790000960EF0005007800860078000402E800C8
:10D7A0000402E900030032000000D0008180D200B2
:10D7B000FBFF370074E080008003520084E08000AB
:10D7C00001045A0097E08800A8E08800123CD400C9
:10D7D00014BCD600123CD40014BCD60094E08000E7
:10D7E0006302420084027800A4E0800060024A00E4
:10D7F0000403780024A021000480420060034B0051
:10D800008600780010407800F5F9B700F5D9BF0020
:10D810000AFCB7000B7CEF000C3CEF000CDCBF00F7
:10D820000DFCB7000BDCBF000CFCB7000ADCBF002E
:10D830000BFCB7000A7CEF0094E08000620242001B
:10D8400084027800A4E0800060024A0004037800AB
:10D8500024A021000480420060034B008600780071
:10D86000B4CF800000429000B4CF8800B4CF8000D5
:10D870000960EF0053E080000480410050E0880020
:10D8800063E08000E081490063E088000CDCBF00B9
:10D890000DFCB7000BDCBF000CFCB7000ADCBF00BE
:10D8A0000BFCB7000A7CEF0094E0800061024200AC
:10D8B00084027800A4E0800060024A00040378003B
:10D8C00024A021000480420060034B008600780001
:10D8D00010407800F7F9B700B4CF80004822DE008E
:10D8E00053E080000480410050E0880063E0800045
:10D8F000E081490063E088000CDCBF000DFCB7004C
:10D900000BDCBF000CFCB7000ADCBF000BFCB7004F
:10D910000A7CEF0024A0210093E0800004804100F5
:10D92000A4E0800060024A0084007800C4CF800038
:10D9300000429000C4CF8800C4CF80000960EF008F
:10D9400053E080000480410050E0880063E08000E4
:10D95000E081490063E0880054E08000F3FF2F007D
:10D960000418E10004003A0064E08000F3FF2000A6
:10D970000418E100600032003D88AE001F0037004F
:10D980000100200001007800822602000000000053
:10D990008100E8003322AF00FEFF3700A0118800AD
:10D9A000B00020000008E600F6FF370060E08000CD
:10D9B00041702200303C02000000000050E0800076
:10D9C00041702200303C0200000000003322AF0012
:10D9D000FEFF370004022000A41188003322AF00AC
:10D9E000FEFF3700A4002000A41188003322AF00FE
:10D9F000FEFF3700D4002000A4118800240020007E
:10DA00000960EF00D0638000E16380000402E80059
:10DA10000402E900030032008100D1000080D3003D
:10DA2000FBFF37004300A900000178008101780066
:10DA300050E0800061E080009C4202000000000095
:10DA4000800278000103780005007800760CB400AD
:10DA500030E08800C463800004004B0040E0880090
:10DA60000A1CF8000E1CF9000C1CF800101CF90030
:10DA70003DCBBF000160EF000100200000017800F5
:10DA80008101780070E0800081E080006C4202003B
:10DA90000000000080027800010378000500780093
:10DAA0008E0CB4008003780006007800908CB400DF
:10DAB000000478003DCBBF000160EF0001002000B2
:10DAC000140020000960EF000402E8000402E900ED
:10DAD000030032000000D0008180D200FBFF37003D
:10DAE00000805300F0E0880001005C0000E1880045
:10DAF000345A0400000000004F047800CF0378007F
:10DB00004F037800CF02780000000600851F7800E0
:10DB1000861F78000500200005007800222A0200F8
:10DB2000000000000040B3004220AF0006003700B4
:10DB30008502E8003322AF00FEFF370034E2B70071
:10DB40003562EF00F4FF37007828EF007A28EF0005
:10DB500014002000044488008228EF007368EF005E
:10DB60007568EF007768EF007048A800F479EF005F
:10DB7000CA590200000000003D68AE008600370070
:10DB80000100200001007800482A02000000000087
:10DB90008100E8003322AF00FEFF3700A0118800AB
:10DBA000D00020000008E600F6FF3700C0438000E8
:10DBB000D1438000040020008C4B020000000000D4
:10DBC0003322AF00FEFF370004022000A4118800BA
:10DBD0003322AF00FEFF3700A4002000A41188000C
:10DBE0003322AF00FEFF3700D4002000A4118800CC
:10DBF00077C8BF00800278000B60EF0006002000AD
:10DC000001002000010078006A2A020000000000E4
:10DC10008100E8003322AF00FEFF3700A01188002A
:10DC2000300120000008E600F6FF3700050078000C
:10DC300086007800040020008C4B020000000000E9
:10DC40003322AF00FEFF370004022000A411880039
:10DC50003322AF00FEFF3700A4002000A41188008B
:10DC60003322AF00FEFF3700D4002000A41188004B
:10DC70007468EF0074C8BF00844380004822DE004F
:10DC80000024E100440039007448E2000D003A002D
:10DC90000100200001007800922A0200000000002C
:10DCA0008100E8003322AF00FEFF3700A01188009A
:10DCB000E00020000008E600F6FF3700986E040040
:10DCC00000000000A54380000B60EF00060020006C
:10DCD0000100200001007800AE2A020000000000D0
:10DCE0008100E8003322AF00FEFF3700A01188005A
:10DCF000900020000008E600F6FF370005007800DD
:10DD000086007800040020008C4B02000000000018
:10DD10003322AF00FEFF3700A4032000A4118800C7
:10DD20003322AF00FEFF370004022000A411880058
:10DD3000A44380000960EF0023CB200003004200D1
:10DD4000904278000B60EF0006002000050078008C
:10DD500086007800040020008C4B020000000000C8
:10DD60003100200001007800CA2A020000000000F3
:10DD70008100E8003322AF00FEFF3700A0118800C9
:10DD8000B00020000008E600F6FF37007468EC00E1
:10DD90003A6E04000000000001002000010078003D
:10DDA000E42A0200000000008100E8003322AF00F6
:10DDB000FEFF3700A0118800900120000008E60057
:10DDC000F6FF37003D68AE004A013700BD6AEF003C
:10DDD000E45580004822DE0044C6B200450132000E
:10DDE000BDCABF00800278000B60EF000600200073
:10DDF00001002000010078000C2B02000000000050
:10DE00008100E8003322AF00FEFF3700A011880038
:10DE1000900020000008E600F6FF370005007800BB
:10DE200086007800440020008C4B020000000000B7
:10DE30003322AF00FEFF370004022000A411880047
:10DE4000BDCABF000160EF004200DD00843E21003A
:10DE500004004000C4892100301A7800301A78008C
:10DE6000E4C4800004407800EAF9B7009DD8BF0000
:10DE70009CF8B7009ED8BF009DF8B7009FD8BF00A0
:10DE80009EF8B7009F78EF00E4C48000044078005B
:10DE9000E9F9B7009DD8BF009CF8B7009ED8BF0035
:10DEA0009DF8B7009FD8BF009EF8B7009F78EF009D
:10DEB000E4C4800004407800E8F9B7009DD8BF00B2
:10DEC0009CF8B7009ED8BF009DF8B7009FD8BF0050
:10DED0009EF8B7009F78EF00E4C48000044078000B
:10DEE000E7F9B700BDCABF000160EF004200DD00E6
:10DEF0008457210004004000048A2100301A780071
:10DF0000301A780004C5800004407800EEF9B700AC
:10DF1000A1D8BF00A0F8B700A2D8BF00A1F8B700F1
:10DF2000A3D8BF00A2F8B700A378EF0004C5800013
:10DF300004407800EDF9B700A1D8BF00A0F8B70001
:10DF4000A2D8BF00A1F8B700A3D8BF00A2F8B700BD
:10DF5000A378EF0004C5800004407800ECF9B70016
:10DF6000A1D8BF00A0F8B700A2D8BF00A1F8B700A1
:10DF7000A3D8BF00A2F8B700A378EF0004C58000C3
:10DF800004407800EBF9B700BDCABF000160EF00A4
:10DF90004200DD008470210004004000448A21001A
:10DFA000301A7800301A780024C5800004407800C8
:10DFB000F2F9B700A5D8BF00A4F8B700A6D8BF00F3
:10DFC000A5F8B700A7D8BF00A6F8B700A778EF005C
:10DFD00024C5800004407800F1F9B700A5D8BF003F
:10DFE000A4F8B700A6D8BF00A5F8B700A7D8BF000F
:10DFF000A6F8B700A778EF0024C580000440780099
:10E00000F0F9B700A5D8BF00A4F8B700A6D8BF00A4
:10E01000A5F8B700A7D8BF00A6F8B700A778EF000B
:10E0200024C5800004407800EFF9B70004AC20005C
:10E0300084C58800E7D9BF00664C020000000000DC
:10E04000E8D9BF00664C020000000000E9D9BF001B
:10E05000664C020000000000EAD9BF00664C0200D6
:10E0600000000000EBD9BF00664C02000000000079
:10E07000ECD9BF00664C020000000000EDD9BF00E3
:10E08000664C020000000000EED9BF00664C0200A2
:10E0900000000000E0C2B300664C02000000000077
:10E0A000EFD9BF00664C020000000000F0D9BF00AD
:10E0B000664C020000000000F1D9BF00664C02006F
:10E0C00000000000F2D9BF00664C02000000000012
:10E0D0003322AF00FEFF370004022000A4118800A5
:10E0E0003322AF00FEFF370004022000A411880095
:10E0F00001AC20001104E000070032003322AF0021
:10E10000FEFF37000140900034E2B7003562EF00B7
:10E110008100E800F7FF37003322AF00FEFF370031
:10E1200004022000A4118800BDCABF000160EF00F6
:10E130004200DD0084DA200004004000A40020003A
:10E14000301A7800301A78000100200001007800B1
:10E15000282B0200000000008100E8003322AF00FD
:10E16000FEFF3700A0118800400020000008E600F4
:10E17000F6FF370005007800860078008400200054
:10E180008C4B0200000000003322AF00FEFF37007E
:10E1900004022000A4118800BDCABF000160EF0086
:10E1A0004200DD0084F3200004004000A4002000B1
:10E1B000301A7800301A7800010020000100780041
:10E1C000402B0200000000008100E8003322AF0075
:10E1D000FEFF3700A0118800400020000008E60084
:10E1E000F6FF3700050078008600780084002000E4
:10E1F0008C4B0200000000003322AF00FEFF37000E
:10E2000004022000A4118800BDCABF000160EF0015
:10E210004200DD00840C210004004000A400200026
:10E22000301A7800301A78000100200001007800D0
:10E23000582B0200000000008100E8003322AF00EC
:10E24000FEFF3700A0118800400020000008E60013
:10E25000F6FF370005007800860078008400200073
:10E260008C4B0200000000003322AF00FEFF37009D
:10E2700004022000A4118800BDCABF000160EF00A5
:10E280004200DD008425210004004000A40020009D
:10E29000301A7800301A7800010020000100780060
:10E2A000702B0200000000008100E8003322AF0064
:10E2B000FEFF3700A0118800500020000008E60093
:10E2C000F6FF370005007800860078000400200083
:10E2D0008C4B0200000000003322AF00FEFF37002D
:10E2E00004022000A4118800BD6AEC00E86E04005E
:10E2F000000000004F037800CF0278000000060005
:10E30000851F7800101AF800121AF90090D08000CA
:10E310001004E00003003200123AEC0086710400A1
:10E320000000000094D0800083D0800003005200E1
:10E33000CF02780000000600851F7800101AF80050
:10E34000161AF900121AF800101AF900123AEF0022
:10E35000101AF800141AF900CA82A900C682A9008E
:10E36000C4FEEF00923B02000000000000C5B300B5
:10E37000B6FEB700B83EEF0014002000D4F58800C8
:10E38000F0CFB300B7FEB700D43B0200000000009E
:10E390000004E00002003200B07104000000000040
:10E3A000C4FEEF00923B020000000000C4FEEF003C
:10E3B000923B020000000000CA82A800C682A900A9
:10E3C000CA82A900C682A90010C5B300B6FEB70074
:10E3D000F0CFB300B7FEB700141AF800B81EF9006A
:10E3E000161AF800BA1EF900684102000000000089
:10E3F000C4FEEF00923B02000000000019FAB700D3
:10E40000195AE20002003200F87104000000000016
:10E41000C4FEEF00923B020000000000E40F200069
:10E420000024E10002003200087204000000000035
:10E43000C4FEEF00923B02000000000018FAB70093
:10E44000C4FEEF00923B020000000000CA82A80058
:10E45000C682A90018DABF000160EF0001002000A9
:10E460000000BE00CF02780000000600851F780083
:10E47000861F78007088A9007068AF00120037000E
:10E48000140020000960EF00506580006165800085
:10E490000402E8000402E900030032000000D0009A
:10E4A0008180D200FBFF370034648000040040000C
:10E4B00010D08800446480000480480020D0880088
:10E4C00088720400000000007068AE001000370081
:10E4D000240020000960EF00506580006165800025
:10E4E0000402E8000402E900030032000000D0004A
:10E4F0008180D200FBFF37003464800004004000BC
:10E5000010D08800446480000480480020D0880037
:10E510003DC8AE00C90037007068AF004900370041
:10E5200014D08000610242008402780024D0800070
:10E5300060024A000403780085D0880096D08800E5
:10E540009C7102000000000006FAB70006DABF0066
:10E55000AEECB700AF6CEF00B02CEF00B0CCBF005A
:10E56000B1ECB700AFCCBF00B0ECB700AECCBF0091
:10E57000AFECB700AE6CEF00021AF800101AF90009
:10E58000041AF800121AF9009C7102000000000041
:10E5900007FAB70034D080004822DE00736580009F
:10E5A000048041007065880083658000E081490037
:10E5B00083658800B02CEF00846580006020E10056
:10E5C0001A003E00040039007465800003FF2F002C
:10E5D0000418E10015003600140020000960EF0067
:10E5E00070658000816580000402E8000402E90093
:10E5F000030032000000D0008180D200FBFF370012
:10E60000346480000400400010D08800446480001E
:10E610000480480020D08800022DEC004220AF008A
:10E62000042DEC001E730400000000007088A80098
:10E6300010C0B30000E0B700930037001A74040064
:10E64000000000007068AE007A00370014D080002F
:10E65000630242008402780024D0800060024A00F5
:10E660000403780085D0880096D088009C71020051
:10E670000000000006FAB70006DABF00AEECB700F3
:10E68000AF6CEF00B02CEF00B0CCBF00B1ECB70026
:10E69000AFCCBF00B0ECB700AECCBF00AFECB70062
:10E6A000AE6CEF0014D08000620242008402780059
:10E6B00024D0800060024A000403780085D08800DE
:10E6C00096D088009C7102000000000007FAB70095
:10E6D00034D080004822DE00736580000480410051
:10E6E0007065880083658000E0814900836588004B
:10E6F000B0CCBF00B1ECB700AFCCBF00B0ECB700FE
:10E70000AECCBF00AFECB700AE6CEF0014D0800011
:10E71000610242008402780024D0800060024A0036
:10E720000403780085D0880096D088009C71020090
:10E730000000000008FAB70044D080000960EF0034
:10E7400073658000048041007065880083658000E7
:10E75000E081490083658800B0CCBF00B1ECB70010
:10E76000AFCCBF00B0ECB700AECCBF00AFECB70091
:10E77000AE6CEF00021AF800101AF900041AF80043
:10E78000121AF9009C7102000000000009FAB7009B
:10E7900044D080004822DE00736580000480410080
:10E7A0007065880083658000E0814900836588008A
:10E7B00074658000F3FF2F000418E10004003A00A4
:10E7C00084658000F3FF20000418E100150032008A
:10E7D000240020000960EF007065800081658000E2
:10E7E0000402E8000402E900030032000000D00047
:10E7F0008180D200FBFF37003464800004004000B9
:10E8000010D08800446480000480480020D0880034
:10E81000022DEC004220AF00042DEC001A7404001D
:10E82000000000007088A80010C0B30000E0B7002E
:10E830001500370042740400000000003DC8AF001E
:10E840001000370054658000610242007465880042
:10E850006465800060024A0084658800022DEC0037
:10E860004220AF00042DEC00106880009C0DE300F6
:10E8700004003A00206880009E0DE30001003A0089
:10E880007088A8000060EF004F037800CF02780086
:10E8900000000600851F7800861F780014DABF008C
:10E8A00017FAB700B4D080004822DE006A24E100E5
:10E8B00009003A007D6BEF009D6BEF00A0C0B30034
:10E8C00075EBB7000879EF000060EF00D600370065
:10E8D000D874040000000000A45B80004822DE0021
:10E8E0006A24E10012003A00B4D080004822DE0021
:10E8F00004C2B2000E003A009D6BEC00A45B8000E5
:10E900004822DE006A24E10005003A009DCBBF00EA
:10E91000155AE30002003A0010C0B30075EBB700CF
:10E920000060EF00C0003700D87404000000000051
:10E93000A45B80004822DE006A24E10006003A0061
:10E94000155AE20004003A0010C0B30075EBB7009E
:10E95000D874040000000000A45B80004822DE00A0
:10E960006124E10008003A00B4D080004822DE00B3
:10E9700004C2B20004003A0020C0B30075EBB70037
:10E98000D874040000000000A45B80004822DE0070
:10E990006324E10006003A00B4D080004822DE0083
:10E9A0006D24E10002003A0040C0B30075EBB700EF
:10E9B000A45B80004822DE006124E1000E003A00E2
:10E9C000E45B80004822DE00A39321008302420022
:10E9D00017DABF00804A7800BD4AE20003003A001F
:10E9E000B4D080006124E10000003A007D6BEC00AF
:10E9F0001276040000000000A45B80004822DE00C4
:10EA00006224E1005C003A00E45B80004822DE0002
:10EA1000A393210083024200804AEB007D6BEF004C
:10EA2000B5CBBF00A2FCB700648D2100F4E48800E0
:10EA3000A493210004E588003A4D02000000000084
:10EA400018FAB700C4D08000F4CFB2000200320040
:10EA5000185AE2000D003A00BD4AE2000B003A00ED
:10EA6000B4D080006524E10008003A0030C0B30053
:10EA700075EBB700856BEF0020C0B30000E0B70076
:10EA8000690037009A75040000000000C4D08000BF
:10EA9000F4CFB2000C003A00E45580004822DE00BA
:10EAA0006124E10008003A00B4D080006124E10054
:10EAB00005003A0030C0B30075EBB700856BEF007E
:10EAC0009A75040000000000185AE20005003A00A0
:10EAD00030C0B30075EBB700856BEF009A7504008A
:10EAE00000000000C4D08000F4CFB20010003A0053
:10EAF00030C0B30075EBB700856BEF00010020005C
:10EB000001007800EC290200000000008100E8000C
:10EB10003322AF00FEFF3700A011880070022000F2
:10EB20000008E600F6FF37009A75040000000000B8
:10EB3000756BEF00B4D080006524E1000C003A0052
:10EB400070E8A80094C680006102420094C6880064
:10EB5000A4C6800060024A00A4C68800645D8000EC
:10EB60004822DE006142420004407800ADEBB7006D
:10EB70001276040000000000A45B80004822DE0042
:10EB80006324E10009003A00245C80004822DE0092
:10EB9000839021008302420017DABF00804A780088
:10EBA000856BEC001276040000000000A45B80007E
:10EBB0004822DE006424E1001A003A00245C800050
:10EBC0004822DE00614052000080FB00849021005A
:10EBD0000400400010427800B4C3B20007003A00BD
:10EBE000245C80004822DE00614052000080FB006F
:10EBF0008490210004034000004BEB00245C800063
:10EC00004822DE008390210083024200804AEB000C
:10EC1000756BEF00856BEF0010C0B30000E0B7002C
:10EC2000010037000060EF004F037800CF0278004A
:10EC300000000600851F7800861F78008A08F8000B
:10EC4000041AF9008C08F800061AF900041AF800F2
:10EC50000A1AF900061AF800041AF900063AEF0039
:10EC6000041AF800081AF90070E8A900117AEF00F8
:10EC700070C8AF000400370014D080004822DE00C6
:10EC80006524E10050003A00CA82A900C682A900AA
:10EC9000C4FEEF00923B02000000000010C5B3006C
:10ECA000B6FEB700F0CFB300B7FEB700081AF80001
:10ECB000B81EF9000A1AF800BA1EF90068410200ED
:10ECC00000000000C4FEEF00923B020000000000C4
:10ECD0000FFAB7000F5AE20018003200117AEC0068
:10ECE00084D080004822DE007424E1001300390043
:10ECF0000100200001007800C82902000000000087
:10ED00008100E8003322AF00FEFF3700A011880029
:10ED1000400020000008E600F6FF3700117AEF00FF
:10ED2000CA82A800C682A900400620006E330200F5
:10ED3000000000004476040000000000C4FEEF0064
:10ED4000923B020000000000E40F20000024E100DC
:10ED50001B003200117AEC0084D080004822DE00D3
:10ED600023032000041CE10013003E0001002000EA
:10ED700001007800DA290200000000008100E800AC
:10ED80003322AF00FEFF3700A011880030002000C2
:10ED90000008E600F6FF3700117AEF00CA82A800EB
:10EDA000C682A900400620006E3302000000000069
:10EDB00044760400000000009E760400000000007D
:10EDC000E8C2A800E902A8000C3AEF0064D0800075
:10EDD00004A0B20056003200107AEF007088AE0036
:10EDE00007003700060DE20002003A00080DE200BD
:10EDF00003003200062DED004200AE00082DED00AC
:10EE000070C0B3000EFAB70074D08000F4CFB20027
:10EE10000F003200E8C2A900E8C2A800E6E2AE0096
:10EE20000800370001A121000EDABF000160EF00E9
:10EE300012002000821F78004F017800803B020002
:10EE4000000000000E7AED000477040000000000CE
:10EE50007088AE0006003700060DE20004003A009C
:10EE6000080DE20002003A00927704000000000062
:10EE700070E8AF0006003700645C80004822DE00C6
:10EE80006124E10002003200950BAE00040037005F
:10EE90009277040000000000927704000000000058
:10EEA00014D080004822DE006124E1000E003A0008
:10EEB00010DABF0014FAB70002DABF0015FAB70083
:10EEC00010C0B30016FAB7004A7402000000000038
:10EED0006104E10002003A0010C0B3008DEBB700FE
:10EEE000927704000000000014D080004822DE0069
:10EEF0006524E1000B003A0010DABF0014FAB700F5
:10EF000002DABF0015FAB70050C0B30016FAB70016
:10EF10004A740200000000006204E10001003900B0
:10EF2000950BA8000C3AEC00E67604000000000007
:10EF3000C4FEEF00923B020000000000C4FEEF00A0
:10EF4000923B02000000000070C8AF000C003700C8
:10EF500014D080004822DE006124E10008003A005D
:10EF6000C4FEEF00923B020000000000E40F20000E
:10EF70000024E10002003200B0770400000000002D
:10EF800070C8AF000400370014D080004822DE00B3
:10EF90006524E10002003A00CA82A800C682A900E6
:10EFA000645C80004822DE006124E10003003A0036
:10EFB00010C0B30000E0B70008003700060DE20003
:10EFC00005003A00080DE20003003A0010C0B3004B
:10EFD00000E0B700010037000060EF004F03780049
:10EFE000CF02780000000600851F7800861F780099
:10EFF000871F7800881F7800F4D9BF00BDEAB700EA
:10F00000BD4AE20018003A00B4CF80006524E10058
:10F0100015003A0084C680006020E100120039002B
:10F0200003003E0074C680006120E1000E0039003C
:10F0300074C680006100520070C6880084C68000DB
:10F0400060005A0080C68800E45980004822DE0033
:10F0500093C680000480510090C68800A3C680003B
:10F0600060805900A0C68800BD4AE2003F003A0017
:10F07000B4CF80006124E1003C003A00645D800070
:10F080004822DE006824E100210039003D68AE001E
:10F090000B00370001002000010078001628020054
:10F0A000000000008100E8003322AF00FEFF3700BF
:10F0B000A0118800300020000008E600F6FF3700AD
:10F0C000E45980004822DE0061424200044078009A
:10F0D00000E0B7000080FB0094C6800000005200F2
:10F0E00090C68800A4C6800060005A00A0C68800B0
:10F0F00074C680006100520070C6880084C680001B
:10F1000060005A0080C68800B67804000000000045
:10F11000645D80004822DE006124E10013003900B4
:10F120003D68AE000B0037000100200001007800B0
:10F1300028280200000000008100E8003322AF0010
:10F14000FEFF3700A0118800300020000008E60014
:10F15000F6FF370094C680006100520090C6880018
:10F16000A4C6800060005A00A0C688003D68AE00BA
:10F170001400370001002000010078003A28020046
:10F18000000000008100E8003322AF00FEFF3700DE
:10F19000A0118800A00020000008E600F6FF37005C
:10F1A00070C6800081C68000040020008C4B0200E5
:10F1B000000000003322AF00FEFF370004022000F1
:10F1C000A41188003D68AE00140037000100200043
:10F1D0000100780056280200000000008100E800CD
:10F1E0003322AF00FEFF3700A0118800A0002000EE
:10F1F0000008E600F6FF370090C68000A1C6800038
:10F20000040020008C4B0200000000003322AF00FD
:10F21000FEFF370004022000A4118800BDCABF0011
:10F220000160EF004200DD0084DA200004004000AD
:10F23000A4002000301A7800301A78000500780009
:10F24000CE18B400F064880084C6800004004B002F
:10F2500000658800BDCABF000160EF004200DD000C
:10F2600084F3200004004000A4002000301A78003D
:10F27000301A780005007800D218B400F0678800D2
:10F28000A4C6800004004B0000688800BDCABF000F
:10F290000160EF004200DD00840C2100040040000A
:10F2A00064CA2000301A7800301A7800BDCABF0046
:10F2B0000160EF004200DD008425210004004000D1
:10F2C000A4002000301A7800301A78006030E10085
:10F2D0000600390002003E006128E1000300390009
:10F2E00070C8A800787904000000000070C8A90068
:10F2F0003D68AE00640037003322AF00FEFF3700E8
:10F30000A4022000A41188003322AF00FEFF3700C2
:10F3100064062000A41188003322AF00FEFF3700EE
:10F32000D4032000A4118800BDCABF000160EF0013
:10F3300004002000604A02000000000001002000DC
:10F340000100780072280200000000008100E8003F
:10F350003322AF00FEFF3700A011880040002000DC
:10F360000008E600F6FF3700F064800001658000C9
:10F37000040020008C4B0200000000003322AF008C
:10F38000FEFF370004022000A411880001002000C5
:10F390000100780088280200000000008100E800D9
:10F3A0003322AF00FEFF3700A0118800400020008C
:10F3B0000008E600F6FF3700F06780000168800073
:10F3C000040020008C4B0200000000003322AF003C
:10F3D000FEFF370004022000A41188000100200075
:10F3E000010078009E280200000000008100E80073
:10F3F0003322AF00FEFF3700A0118800400020003C
:10F400000008E600F6FF37003065800041658000A7
:10F41000040020008C4B0200000000003322AF00EB
:10F42000FEFF370004022000A41188008042EB0098
:10F4300070C8AF008502E8000100200001007800DC
:10F44000B4280200000000008100E8003322AF0071
:10F45000FEFF3700A0118800300020000008E60001
:10F46000F6FF3700054078000160EF00040020003F
:10F47000604A0200000000003322AF00FEFF3700A8
:10F4800004022000A4118800F879EF001400200085
:10F49000E46C88009E2DEF00E5598000C82ADE004C
:10F4A000C92ADD000500780001002000E26C800020
:10F4B000F36C80006C420200000000004465800094
:10F4C0000120E1000900390003003E00346580009E
:10F4D0000020E100050036009C2DEC004220AF002A
:10F4E0009E2DEC004C7A0400000000003D68AE0048
:10F4F000140037000100200001007800CA28020033
:10F50000000000008100E8003322AF00FEFF37005A
:10F51000A0118800500020000008E600F6FF370028
:10F520001068800021688000040020008C4B0200DD
:10F53000000000003322AF00FEFF3700040220006D
:10F54000A41188003D68AE001400370001002000BF
:10F5500001007800E2280200000000008100E800BD
:10F560003322AF00FEFF3700A011880050002000BA
:10F570000008E600F6FF3700E06C8000F16C8000C8
:10F58000040020008C4B0200000000003322AF007A
:10F59000FEFF370004022000A4118800B4CF8000D1
:10F5A0006524E10003003200B4CF80006924E1004B
:10F5B00008003A00F46C80006020E10005003E0085
:10F5C00003003900E46C80006220E100010031009A
:10F5D000DC013700E46C8000E1025200F46C800032
:10F5E00060035A003DCBBF00000178000560EF00CA
:10F5F0000300200005007800860078006C420200BD
:10F6000000000000800378000104780094002000CE
:10F6100007007800880078000402E8000402E9008E
:10F62000030032000000D0008180D200FBFF3700D1
:10F630003465800000005200306888004465800016
:10F6400001005A00406888003D68AE001B0037008A
:10F650000100200001007800FA28020000000000EC
:10F660008100E8003322AF00FEFF3700A0118800C0
:10F67000900020000008E600F6FF370030688000A8
:10F6800041688000040020008C4B02000000000054
:10F69000D100200001007800FA28020000000000DC
:10F6A0008100E8003322AF00FEFF3700A011880080
:10F6B000000120000008E600F6FF3700022DEF00F1
:10F6C000042DEF009E0CF800AA0CF900A00CF80025
:10F6D000AC0CF900FE0CF800A608F900000DF800CB
:10F6E000A808F900756BEF007D6BEF008D6BEF00E4
:10F6F00070C8AF0074003700B4CF80006124E1000F
:10F7000071003A003D68AE000B0037000100200098
:10F710000100780018290200000000008100E800C4
:10F720003322AF00FEFF3700A011880080002000C8
:10F730000008E600F6FF370094002000A608F80055
:10F740008A08F900A808F8008C08F9000402E8000B
:10F750000402E900030032008A28D4008CA8D600F5
:10F76000FBFF37008A08F800FC19F9008C08F80044
:10F770008A08F9008C28EF008A08F800FA19F900C5
:10F780003D68AE000B00370001002000010078004A
:10F790002E290200000000008100E8003322AF00A3
:10F7A000FEFF3700A0118800800020000008E6005E
:10F7B000F6FF3700CA82A900C682A900C4FEEF0086
:10F7C000923B02000000000020C5B300B6FEB70067
:10F7D00010C0B300B7FEB700FA19F800B81EF90060
:10F7E000FC19F800BA1EF900684102000000000090
:10F7F000C4FEEF00923B020000000000F7F9B700E2
:10F80000F759E2000F0032003D68AE000B003700F0
:10F810000100200001007800F02602000000000036
:10F820008100E8003322AF00FEFF3700A0118800FE
:10F83000500020000008E600F6FF3700F87B0400C7
:10F8400000000000C4FEEF00923B02000000000038
:10F85000E40F20000024E10019003200F879EC00E8
:10F86000C4CF800023032000041CE10012003E00EE
:10F8700001002000010078000427020000000000C1
:10F880008100E8003322AF00FEFF3700A01188009E
:10F89000300020000008E600F6FF3700CA82A8000A
:10F8A000C682A900A00020006E3302000000000004
:10F8B000DA7B040000000000227C0400000000004D
:10F8C000E8C2A800E902A800950BA900A56BEF000B
:10F8D0003D68AE000B0037000100200001007800F9
:10F8E00044290200000000008100E8003322AF003C
:10F8F000FEFF3700A0118800800020000008E6000D
:10F90000F6FF370020688000F46C80000020E100E2
:10F91000CC00390004003E0010688000E46C8000D8
:10F920000020E100C700390070E8A9003DC8A90027
:10F9300070C8AF003DC8A800367202000000000089
:10F94000B4CF80006524E10015003A0024688000EF
:10F950006020E1001200390003003E0014688000BE
:10F960006120E1000E00360074C680006102420092
:10F9700074C6880084C6800060024A0084C688007D
:10F98000E45980004822DE0093C6800004804100D4
:10F9900090C68800A3C68000E0814900A3C6880005
:10F9A00070C8AF0003003700B4CF80006524E100C9
:10F9B0005E003A003D68AE000B00370001002000F9
:10F9C000010078005A290200000000008100E800D0
:10F9D0003322AF00FEFF3700A0118800A0002000F6
:10F9E0000008E600F6FF3700CA82A900C682A90017
:10F9F000C4FEEF00923B02000000000000C5B3000F
:10FA0000B6FEB700B83EEF00F0CFB300B7FEB700C8
:10FA100004202000D4F58800D43B02000000000040
:10FA20000004E0000F0032003D68AE000B0037001C
:10FA3000010020000100780072290200000000008F
:10FA40008100E8003322AF00FEFF3700A0118800DC
:10FA5000600020000008E600F6FF3700F87C040094
:10FA600000000000C4FEEF00923B02000000000016
:10FA7000C4FEEF00923B020000000000CA82A80012
:10FA8000C682A90054658000E202520064658000CD
:10FA900060035A003DCBBF00000178000560EF0015
:10FAA0000300200005007800860078006C42020008
:10FAB0000000000030458800414588003045800046
:10FAC000960CB40030458800C46480004345800033
:10FAD00004804900404588007068AE000800370087
:10FAE000E45980004822DE00334580000480510044
:10FAF00030458800434580006080590040458800BB
:10FB000094002000A608F8009E08F900A808F80054
:10FB1000A008F9000402E8000402E9000300320032
:10FB20009E28D400A0A8D600FBFF37009E08F8004E
:10FB30008A08F900A008F8008C08F900F044800059
:10FB40008A0CB4006464800003458000848049000E
:10FB50008A08E30003003A00644480000120E100C9
:10FB600020003200F5D9BF0002FAB700F6D9BF0075
:10FB700003FAB7001A760200000000006104E100F9
:10FB80000F003A003D68AE000B0037000100200076
:10FB90000100780086290200000000008100E800D2
:10FBA0003322AF00FEFF3700A01188007000200054
:10FBB0000008E600F6FF3700F27D040000000000B8
:10FBC00004202000534480000480410050448800F9
:10FBD0006444800060024A00644488009E7D040002
:10FBE00000000000645C80004822DE006124E10027
:10FBF00002003A00227E040000000000950BAE00D7
:10FC000002003700227E0400000000007088AF0070
:10FC100006003700AE0CF800AA0CF900B00CF80092
:10FC2000AC0CF9001E7E0400000000007088AE00DD
:10FC300002003700227E040000000000827C0400E5
:10FC4000000000003D68AE000B00370001002000FE
:10FC5000010078009C290200000000008100E800FB
:10FC60003322AF00FEFF3700A01188008000200083
:10FC70000008E600F6FF370070C8AF002400370028
:10FC8000B4CF80006124E10021003A00CA82A900BB
:10FC9000C682A900C0C4B300B6FEB700B83EEF00EC
:10FCA000BA3EEF00F0CFB300B7FEB700D43B02007E
:10FCB000000000000004E0000D0032000100200000
:10FCC0000100780016270200000000008100E80013
:10FCD0003322AF00FEFF3700A01188007000200023
:10FCE0000008E600F6FF37004A7E0400000000002E
:10FCF000C4FEEF00923B020000000000C4FEEF00D3
:10FD0000923B020000000000CA82A800C682A9003F
:10FD10003D68AE000B0037000100200001007800B4
:10FD2000B2290200000000008100E8003322AF0089
:10FD3000FEFF3700A0118800800020000008E600C8
:10FD4000F6FF37004F047800CF0378004F037800A8
:10FD5000CF02780000000600851F7800C500200053
:10FD600003000900B51F78000202B80003F0A600E6
:10FD7000020037000383B900010037000303B80015
:10FD80004200A9008502430060844B0001F0A600F8
:10FD900002003700028BB90001003700020BB800E7
:10FDA00085024B0008844B000980B000038BB9002A
:10FDB00008044B0087834C00870178000801780015
:10FDC0008500780004007800250120000300090068
:10FDD000CF127800CF02780000000600851F78005F
:10FDE000861F7800871F7800FE39EF00FA39EF0090
:10FDF000A4002000E4CF8800F639EF00F839EF00C6
:10FE0000F419E20003003A00000020000100200085
:10FE1000E4003700F0CF8000FE39EC00800278006B
:10FE200005007800F419B40004D08000004290006E
:10FE300004D0880004D08000D4C2B2000C003A0084
:10FE400014002000D4CF8800F0CF8000FE39EC00F1
:10FE50008002780005007800F419B40004D0800016
:10FE60000042900004D088004E7F04000000000093
:10FE700004D08000B4C2B20008003A00F0CF800085
:10FE8000FE39EC008002780005007800F419B40017
:10FE900004D080000042900004D0880004D080008C
:10FEA00003032000041CE100AE003E0004D08000EB
:10FEB00093032000041CE100AA00390004D0800054
:10FEC00004C3B20015003A00F0CF8000F419B4006A
:10FED0001042780084C7B20005003200F0CF8000E5
:10FEE000F419B4001042780084C5B2000B003A0047
:10FEF00004012000E4CF8800FE39EC00F0CF800040
:10FF0000FE39EC008002780005007800F419B40096
:10FF100004D080000042900004D08800E4CF80002C
:10FF20006A20E10026003A0004D08000030320008C
:10FF3000041CE10020003E0004D080009303200058
:10FF4000041CE1001C003900A0002000010020007A
:10FF5000B2CF8000C3CF8000AC7E02000000000062
:10FF6000800278000103780004D080000443B100CF
:10FF70000440780000E0B7000080FB00050040006E
:10FF8000B0CF88000400200006004A00C0CF8800DF
:10FF9000F0CF8000FE39EC00800278000500780088
:10FFA000F419B40004D080000042900004D088000E
:10FFB000947F040000000000B280040000000000F4
:10FFC000E4CF80007020E10066003A0004D0800099
:10FFD00013062000041CE10007003E0004D080004E
:10FFE000A3072000041CE1000300390000DABF0071
:10FFF000F04DB2000100370000DABF0000FAB70090
:020000040001F9
:1000000004D0800003032000041CE10005003E0032
:1000100004D0800093032000041CE100010039009B
:100020000800370004D0800013042000041CE10005
:100030004C003E0004D0800063042000041CE1005A
:100040004800390004D0800003032000041CE100B4
:1000500019003E0004D0800093032000041CE1003E
:100060001500390044002000B5CF8000C6CF8000C5
:100070000402E8000402E900030032008502D00017
:100080000683D200FBFF370004D080000443B10098
:100090000440780000E0B7000080FB00050040004D
:1000A000B0CF88000400200006004A00C0CF8800BE
:1000B000848004000000000044002000B5CF8000D0
:1000C000C6CF80000402E8000402E9000300320009
:1000D0008502D0000683D200FBFF370004D08000E9
:1000E0001444B1000440780000E0B7006A404000CA
:1000F0000080FB0005004000B0CF88000400200015
:1001000006004A00C0CF8800F0CF8000FE39EC0026
:100110008002780005007800F419B40004D0800053
:100120000042900004D0880004D080001306200014
:10013000041CE10007003E0004D08000A30720005B
:10014000041CE1000300390000DABF00F04DB200EA
:100150000100370000DABF0000FAB7000080040099
:1001600000000000E4CF80006A20E1000B003A00AC
:10017000D4CF80006120E10008003A000400200094
:10018000B3CF800003005200B0CF880004002000ED
:10019000C3CF800003005A00C0CF8800B0CF8000DA
:1001A000C1CF8000CF0378004F037800CF027800E2
:1001B00000000600851F7800AD6BEF00CE38EF0021
:1001C000D038EF00D238EF00D438EF003D68AE00F1
:1001D0000B00370001002000010078006C270200AE
:1001E000000000008100E8003322AF00FEFF37006E
:1001F000A0118800300120000008E600F6FF37005B
:10020000648D210084D0880080710200000000000D
:10021000B5EBB70010C0B300F4F9B700F579EF0003
:1002200010C0B300F6F9B700F47702000000000038
:100230003D68AE002000370001002000010078007A
:100240008E270200000000008100E8003322AF008A
:10025000FEFF3700A0118800300020000008E600F3
:10026000F6FF3700819021001104E0000700320002
:100270003322AF00FEFF37000140900034E2B700A8
:100280003562EF008100E800F7FF370061002000D1
:10029000010078008E270200000000008100E800C5
:1002A0003322AF00FEFF3700A0118800B00020000D
:1002B0000008E600F6FF370084902100A4CF8800F4
:1002C000EE7E02000000000070C6880081C6880033
:1002D0003DCBBF00000178000560EF000300200067
:1002E00070C6800081C680006C42020000000000E1
:1002F00090C68800A1C68800CE18E20012003A001D
:10030000D018E20010003A00D218E2000E003A00C5
:10031000D418E2000C003A0001002000010078002F
:10032000A8270200000000008100E8003322AF008F
:10033000FEFF3700A0118800A00120000008E600A1
:10034000F6FF3700480037003D68AE000B0037006D
:100350000100200001007800D0270200000000000A
:100360008100E8003322AF00FEFF3700A0118800B3
:10037000300120000008E600F6FF3700F479EF00B6
:10038000F579EF0050C0B300F6F9B700F47702003A
:10039000000000003D68AE000B00370001002000A7
:1003A00001007800F2270200000000008100E80050
:1003B0003322AF00FEFF3700A0118800500120005B
:1003C0000008E600F6FF3700F479EF00F579EF005A
:1003D00010C0B300F6F9B700F47702000000000087
:1003E0003D68AE00200037000100200001007800C9
:1003F0008E270200000000008100E8003322AF00D9
:10040000FEFF3700A0118800300020000008E60041
:10041000F6FF3700819021001104E0000700320050
:100420003322AF00FEFF37000140900034E2B700F6
:100430003562EF008100E800F7FF3700610020001F
:10044000010078008E270200000000008100E80013
:100450003322AF00FEFF3700A0118800B00020005B
:100460000008E600F6FF3700CF0278000000060023
:10047000851F78001C1AF800201AF90000D18000AE
:100480001004E000190032001E1AF800221AF900C8
:1004900010D180001004E00006003A0004D1800072
:1004A000E3D0800003005200130037006A8204008A
:1004B0000000000000D180009042780010D1800040
:1004C00010407800002CE10002003A007082040025
:1004D00000000000223AEC00488204000000000006
:1004E000203AEC003E8204000000000004D18000AD
:1004F000E3D0800003005200CF0278000000060025
:10050000851F7800101AE2000300320080D08000BE
:100510008E8204000000000000408000A0D088000F
:10052000141AF8001C1AF900121AF8001E1AF90021
:100530003882020000000000804278008582FB00C3
:1005400005407800143AB400A0D080001004E00008
:1005500005003A000540800000C2B300804A7800E0
:100560000020EF0011003700141AF800A81CF90051
:10057000121AF800AA1CF900744C020000000000D6
:10058000B0D08800B0D080001004E000030032003A
:10059000B5D08000804AEB00163AEC00161AF8003D
:1005A0000008F900141AF8000000F900CF027800E2
:1005B00000000600851F7800861F7800277AEF006C
:1005C00014002000D4D088001C3AEF007088A900E5
:1005D000141AF8009E08F900161AF800A008F9008D
:1005E000141AF800201AF900161AF800141AF90063
:1005F000163AEF00141AF8001E1AF900CA82A90070
:10060000C682A900C4FEEF00923B02000000000079
:1006100020C5B300B6FEB70010C0B300B7FEB700E8
:100620001E1AF800B81EF900201AF800BA1EF900C8
:100630006841020000000000C4FEEF00923B02008F
:100640000000000026FAB700265AE2000F00320030
:100650003D68AE000B00370001002000010078006B
:10066000F0260200000000008100E8003322AF0005
:10067000FEFF3700A0118800500020000008E600AF
:10068000F6FF37001C83040000000000C4FEEF00EA
:10069000923B020000000000E40F20000024E10073
:1006A0001A003200277AEC0034D180004822DE00A4
:1006B00023032000041CE10012003E000100200082
:1006C0000100780004270200000000008100E8001B
:1006D0003322AF00FEFF3700A01188003000200059
:1006E0000008E600F6FF3700CA82A800C682A9000B
:1006F000A00020006E33020000000000FE82040013
:10070000000000004683040000000000E8C2A800CA
:10071000E902A800223AEF0014D1800004A0B20040
:10072000EB003200D4D080006120E10013003A00D9
:100730001C1AE20011003A0014D18000C30220000C
:100740000418E1000D00360070C0B30019FAB700BC
:10075000C4D080004822DE00F4CFB2000500320091
:10076000E8C2A900E8C2A800197AED00A883040035
:100770000000000062850400000000007088AE00E8
:1007800020003700446880006020E10013003E0034
:1007900003003900346880006120E1000F003E0052
:1007A00070C0B30019FAB700C4D080004822DE0040
:1007B000F4CFB20005003200E8C2A900E8C2A800E8
:1007C000197AED00D4830400000000006285040063
:1007D0000000000002840400000000004468800063
:1007E0006020E1000700390003003E00346880000B
:1007F0006220E10003003900062DED004200AE004A
:10080000082DED00D1C2A800E842A800E842A900E6
:10081000D1C2A90010C0B30019FAB700C4D080003B
:100820004822DE00F4CFB20006003200D1A2A900B7
:10083000E842A800E842A900197AED000E840400FD
:1008400000000000247AEF0070C0B30019FAB7006E
:10085000C4D080004822DE00F4CFB2000F00320086
:10086000E8C2A900E8C2A800E6E2AE00080037002E
:1008700041A2210019DABF000160EF001200200040
:10088000821F78004F017800803B020000000000CA
:10089000197AED002884040000000000185AE200D4
:1008A00021003A0024D1800003082000041CE1004C
:1008B0000A0036000408200023D1800003405200C3
:1008C0000160EF004100DE000408200000405200FB
:1008D00025FAB700908404000000000024D18000B5
:1008E00003082000041CE1000B00310024D180002B
:1008F0000448B1000440780000E0B7000160EF0058
:100900004100DE00040820000440400025FAB70042
:10091000908404000000000000C8B30025FAB7006E
:100920001C85040000000000C4D080006124E100A8
:100930001D003A0024D1800003082000041CE100BF
:10094000080036000408200023D180000340520034
:10095000040820000040520025FAB700D0840400AB
:100960000000000024D1800003082000041CE100E6
:100970000900310024D180000448B100044078000F
:1009800000E0B700040820000440400025FAB7004A
:10099000D08404000000000000C8B30025FAB700AE
:1009A0001C85040000000000C4D080006224E10027
:1009B0001F003A0024D1800003082000041CE1003D
:1009C000090036000408200023D1800003405200B3
:1009D0004100DD00040820000040520025FAB70065
:1009E000148504000000000024D1800003082000CA
:1009F000041CE1000A00310024D180000448B10049
:100A00000440780000E0B7004100DD000408200049
:100A10000440400025FAB7001485040000000000DF
:100A200000C8B30025FAB7001C85040000000000D0
:100A300024DABF0025FAB70024DABF0025FAB70090
:100A400070C0B30019FAB700C4D080004822DE009D
:100A5000F4CFB2000E00320025DABF00800078002B
:100A600019DABF000100A50003003900D1A2A800D7
:100A70003E85040000000000D1A2A900E842A800C1
:100A8000E842A900197AED00248504000000000066
:100A900050C0B30019FAB700C4D080004822DE006D
:100AA000F4CFB20006003200D1A2A900E842A800AB
:100AB000E842A900197AED004C850400000000000E
:100AC000D1C2A800223AEC008C8304000000000090
:100AD000C4FEEF00923B020000000000C4FEEF00E5
:100AE000923B020000000000C4FEEF00923B0200B7
:100AF00000000000E40F20000024E10002003200AA
:100B0000748504000000000004202000F3448000ED
:100B100004804100F04488000445800060024A00DF
:100B2000044588001A3AEC004220AF001C3AEC0061
:100B300070448000A60CB4004465800083448000AB
:100B400084804900044580000120E1001B003E0034
:100B500003003900F44480000020E1001700310058
:100B6000E45980004822DE00D3D080008482410016
:100B7000E3D08000E0814900030378003DCBBF0053
:100B8000000178000560EF0003002000E06C8000A9
:100B9000F16C80006C420200000000000608E100D9
:100BA00004003E00020039000500E10001003100B0
:100BB0007088A8008A83040000000000CA82A9008F
:100BC000C682A900C0C4B300B6FEB700B83EEF00AD
:100BD000BA3EEF00F0CFB300B7FEB700D43B02003F
:100BE000000000000004E0000D00320001002000C1
:100BF0000100780016270200000000008100E800D4
:100C00003322AF00FEFF3700A011880070002000E3
:100C10000008E600F6FF3700E2850400000000004F
:100C2000C4FEEF00923B020000000000C4FEEF0093
:100C3000923B020000000000CA82A800C682A90000
:100C40000060EF004F037800CF027800000006003C
:100C5000851F7800861F7800871F7800881F78001E
:100C600010DABF000160EF004200DD00840C2100BB
:100C70000400400064CA2000301A7800301A78005E
:100C80004D4BE20013003A0010DABF000160EF00A4
:100C90004200DD0084F3200004004000A400200096
:100CA000301A7800301A78009400200075448800CB
:100CB000864488000402E8000402E90003003200D0
:100CC0008E28D40090A8D600FBFF3700828604004F
:100CD00000000000645A80004822DE006124E10028
:100CE00008003A0010DABF000160EF004200DD00AA
:100CF00084F3200004004000E4882000301A7800CB
:100D0000301A780010DABF000160EF004200DD0009
:100D100084DA200004004000E4C92000301A780082
:100D2000301A78003D68AE004D00370085D0800055
:100D30000B60EF0006002000010020000100780099
:100D4000A6320200000000008100E8003322AF005C
:100D5000FEFF3700A0118800C00020000008E60058
:100D6000F6FF3700050078008600780004002000B8
:100D70008C4B0200000000003322AF00FEFF370062
:100D800004022000A4118800010020000100780066
:100D9000D4260200000000008100E8003322AF00EA
:100DA000FEFF3700A0118800900020000008E60038
:100DB000F6FF37008044800041702200303C020082
:100DC000000000007044800041702200303C0200AE
:100DD000000000003322AF00FEFF370004022000B5
:100DE000A41188000100200001007800C432020034
:100DF000000000008100E8003322AF00FEFF370052
:100E0000A0118800F00020000008E600F6FF37007F
:100E10004065800041702200303C0200000000006C
:100E20003065800041702200303C0200000000006C
:100E30003322AF00FEFF370004022000A411880017
:100E40003322AF00FEFF3700A4002000A411880069
:100E50003322AF00FEFF3700D4002000A411880029
:100E6000A60CE20003003A00A80CE20001003A00E0
:100E700088003700FE0CF800B218F900000DF800E9
:100E8000B418F90014002000E46C88009E2DEF00D7
:100E9000E5598000C82ADE00C92ADD000500780077
:100EA00001002000E26C8000F36C80006C420200C4
:100EB00000000000446580000120E10009003900C5
:100EC00003003E00346580000020E100050036008C
:100ED0009C2DEC004220AF009E2DEC0048870400C2
:100EE000000000003D68AE00170037000100200040
:100EF00001007800E8320200000000008100E800F4
:100F00003322AF00FEFF3700A011880060012000EF
:100F10000008E600F6FF3700F06C80004170220008
:100F2000303C020000000000E06C800041702200B4
:100F3000303C0200000000003322AF00FEFF37000B
:100F400004022000A4118800E46C8000E102520039
:100F5000F46C800060035A003DCBBF0000017800B4
:100F60000560EF000300200005007800860078008F
:100F70006C42020000000000800378000104780049
:100F80009400200007007800880078000402E80040
:100F90000402E900030032000000D0008180D2008A
:100FA000FBFF370034658000000052003068880085
:100FB0004465800001005A00406888003D68AE002A
:100FC00017003700010020000100780010330200F4
:100FD000000000008100E8003322AF00FEFF370070
:100FE000A0118800900020000008E600F6FF3700FE
:100FF0004068800041702200303C02000000000088
:101000003068800041702200303C02000000000087
:101010003322AF00FEFF370004022000A411880035
:10102000022DEF00042DEF009E0CF800AA0CF90031
:10103000A00CF800AC0CF9003D68AE000D003700C4
:1010400005002000050078002C330200000000009D
:101050000040B3004220AF00060037008502E800E0
:101060003322AF00FEFF370034E2B7003562EF00F5
:10107000F4FF370011DABF0018FAB7008E08F80045
:10108000141AF9009008F800161AF900DA82020022
:10109000000000004F047800CF0378004F03780071
:1010A000CF02780000000600851F7800861F7800B8
:1010B000871F7800881F7800FB79EF00020020006E
:1010C00021A0210002007800862B02000000000011
:1010D000805878000201E8000004E0004220AE00E1
:1010E000F8FF370084AC200084D0880024A02100C1
:1010F00094D08800808202000000000070D0880038
:101100000E1AE2007F043200F579EF00017AEF0059
:10111000087AEF00097AEF00619F210072D0800009
:10112000B24878003104E0004220AE00FCFF3700F6
:10113000649F210084D088008071020000000000BC
:101140006104E1000D00360020C0B300A2FCB7002E
:1011500084A02100F4E48800849F210004E5880035
:10116000844D02000000000084A02100F4E4880007
:10117000C04D02000000000001FAB700020020008C
:10118000C19F210002007800982B0200000000009F
:10119000805878000201E8000004E0004220AE0020
:1011A000F8FF370020C0B300A2FCB700649F210005
:1011B000F4E48800C49F210004E588003A4D020051
:1011C00000000000F4F9B700F459E20004003A000E
:1011D00020C0B300F5F9B700C09004000000000083
:1011E00002002000C19F210002007800A82B02000D
:1011F00000000000805878000201E8000004E000D0
:101200004220AE00F8FF370020C0B300A2FCB700B8
:10121000649F2100F4E48800C49F210004E5880055
:101220003A4D020000000000F4F9B700F459E20062
:1012300004003A0030C0B300F5F9B700C0900400D4
:101240000000000002002000C19F21000200780081
:10125000B82B020000000000805878000201E8006E
:101260000004E0004220AE00F8FF370020C0B300C9
:10127000A2FCB700649F2100F4E48800C49F210011
:1012800004E588003A4D020000000000F4F9B700C0
:10129000F459E20004003A0040C0B300F5F9B70089
:1012A000C09004000000000002002000C19F210047
:1012B00002007800C82B020000000000805878006F
:1012C0000201E8000004E0004220AE00F8FF370011
:1012D00020C0B300A2FCB700649F2100F4E48800A2
:1012E000C49F210004E588003A4D02000000000080
:1012F000F4F9B700F459E20004003A0050C0B3001A
:10130000F5F9B700C09004000000000002002000C2
:10131000C19F210002007800D82B020000000000CD
:10132000805878000201E8000004E0004220AE008E
:10133000F8FF370020C0B300A2FCB700649F210073
:10134000F4E48800C49F210004E588003A4D0200BF
:1013500000000000F4F9B700F459E20004003A007C
:1013600060C0B300F5F9B700C090040000000000B1
:1013700002002000C19F210002007800E82B02003B
:1013800000000000805878000201E8000004E0003E
:101390004220AE00F8FF370020C0B300A2FCB70027
:1013A000649F2100F4E48800C49F210004E58800C4
:1013B0003A4D020000000000F4F9B700F459E200D1
:1013C00004003A0070C0B300F5F9B700C090040003
:1013D0000000000002002000C19F210002007800F0
:1013E000F82B020000000000805878000201E8009D
:1013F0000004E0004220AE00F8FF370020C0B30038
:10140000A2FCB700649F2100F4E48800C49F21007F
:1014100004E588003A4D020000000000F4F9B7002E
:10142000F459E20004003A0080C0B300F5F9B700B7
:10143000C09004000000000002002000C19F2100B5
:1014400002007800082C020000000000805878009C
:101450000201E8000004E0004220AE00F8FF37007F
:1014600010C0B300A2FCB700649F2100F4E4880020
:10147000C49F210004E588003A4D020000000000EE
:10148000F4F9B700F459E20004003A0090C0B30048
:10149000F5F9B700C0900400000000000200200031
:1014A000C19F210002007800162C020000000000FD
:1014B000805878000201E8000004E0004220AE00FD
:1014C000F8FF370020C0B300A2FCB700649F2100E2
:1014D000F4E48800C49F210004E588003A4D02002E
:1014E00000000000F4F9B700F459E20004003A00EB
:1014F000A0C0B300F5F9B700C090040000000000E0
:1015000002002000C19F210002007800262C02006A
:1015100000000000805878000201E8000004E000AC
:101520004220AE00F8FF370020C0B300A2FCB70095
:10153000649F2100F4E48800C49F210004E5880032
:101540003A4D020000000000F4F9B700F459E2003F
:1015500004003A00C0C0B300F5F9B700C090040021
:101560000000000002002000C19F2100020078005E
:10157000362C020000000000805878000201E800CC
:101580000004E0004220AE00F8FF370010C0B300B6
:10159000A2FCB700649F2100F4E48800C49F2100EE
:1015A00004E588003A4D020000000000F4F9B7009D
:1015B000F459E20004003A00B0C0B300F5F9B700F6
:1015C000C09004000000000002002000C19F210024
:1015D00002007800442C02000000000080587800CF
:1015E0000201E8000004E0004220AE00F8FF3700EE
:1015F00020C0B300A2FCB700649F2100F4E488007F
:10160000C49F210004E588003A4D0200000000005C
:10161000F4F9B700F459E20004003A00D0C0B30076
:10162000F5F9B700C090040000000000020020009F
:10163000C19F210002007800542C0200000000002D
:10164000805878000201E8000004E0004220AE006B
:10165000F8FF370020C0B300A2FCB700649F210050
:10166000F4E48800C49F210004E588003A4D02009C
:1016700000000000F4F9B700F459E20004003A0059
:10168000E0C0B300F5F9B700C0900400000000000E
:1016900002002000C19F210002007800642C02009B
:1016A00000000000805878000201E8000004E0001B
:1016B0004220AE00F8FF370020C0B300A2FCB70004
:1016C000649F2100F4E48800C49F210004E58800A1
:1016D0003A4D020000000000F4F9B700F459E200AE
:1016E00004003A00F0C0B300F5F9B700C090040060
:1016F0000000000002002000C19F210002007800CD
:10170000742C020000000000805878000201E800FC
:101710000004E0004220AE00F8FF370010C0B30024
:10172000A2FCB700649F2100F4E48800C49F21005C
:1017300004E588003A4D020000000000F4F9B7000B
:10174000F459E20004003A0000C1B300F5F9B70013
:10175000C09004000000000002002000C19F210092
:1017600002007800822C02000000000080587800FF
:101770000201E8000004E0004220AE00F8FF37005C
:1017800010C0B300A2FCB700649F2100F4E48800FD
:10179000C49F210004E588003A4D020000000000CB
:1017A000F4F9B700F459E20004003A0010C1B300A4
:1017B000F5F9B700C090040000000000020020000E
:1017C000C19F210002007800902C02000000000060
:1017D000805878000201E8000004E0004220AE00DA
:1017E000F8FF370020C0B300A2FCB700649F2100BF
:1017F000F4E48800C49F210004E588003A4D02000B
:1018000000000000F4F9B700F459E20004003A00C7
:1018100020C1B300F5F9B700C0900400000000003B
:1018200002002000C19F210002007800A02C0200CD
:1018300000000000805878000201E8000004E00089
:101840004220AE00F8FF370020C0B300A2FCB70072
:10185000649F2100F4E48800C49F210004E588000F
:101860003A4D020000000000F4F9B700F459E2001C
:1018700004003A0030C1B300F5F9B700C09004008D
:101880000000000002002000C19F2100020078003B
:10189000B02C020000000000805878000201E8002F
:1018A0000004E0004220AE00F8FF370020C0B30083
:1018B000A2FCB700649F2100F4E48800C49F2100CB
:1018C00004E588003A4D020000000000F4F9B7007A
:1018D000F459E20004003A0040C1B300F5F9B70042
:1018E000C09004000000000002002000C19F210001
:1018F00002007800C02C0200000000008058780030
:101900000201E8000004E0004220AE00F8FF3700CA
:1019100020C0B300A2FCB700649F2100F4E488005B
:10192000C49F210004E588003A4D02000000000039
:10193000F4F9B700F459E20004003A0050C1B300D2
:10194000F5F9B700C090040000000000020020007C
:10195000C19F210002007800D02C0200000000008E
:10196000805878000201E8000004E0004220AE0048
:10197000F8FF370010C0B300A2FCB700649F21003D
:10198000F4E48800C49F210004E588003A4D020079
:1019900000000000F4F9B700F459E20004003A0036
:1019A00060C1B300F5F9B700C0900400000000006A
:1019B00002002000C19F210002007800DE2C0200FE
:1019C00000000000805878000201E8000004E000F8
:1019D0004220AE00F8FF370010C0B300A2FCB700F1
:1019E000649F2100F4E48800C49F210004E588007E
:1019F0003A4D020000000000F4F9B700F459E2008B
:101A000004003A0070C1B300F5F9B700C0900400BB
:101A10000000000002002000C19F210002007800A9
:101A2000EC2C020000000000805878000201E80061
:101A30000004E0004220AE00F8FF370010C0B30001
:101A4000A2FCB700649F2100F4E48800C49F210039
:101A500004E588003A4D020000000000F4F9B700E8
:101A6000F459E20004003A0080C1B300F5F9B70070
:101A7000C09004000000000002002000C19F21006F
:101A800002007800FA2C0200000000008058780064
:101A90000201E8000004E0004220AE00F8FF370039
:101AA00020C0B300A2FCB700649F2100F4E48800CA
:101AB000C49F210004E588003A4D020000000000A8
:101AC000F4F9B700F459E20004003A00A0C1B300F1
:101AD000F5F9B700C09004000000000002002000EB
:101AE000C19F2100020078000A2D020000000000C2
:101AF000805878000201E8000004E0004220AE00B7
:101B0000F8FF370010C0B300A2FCB700649F2100AB
:101B1000F4E48800C49F210004E588003A4D0200E7
:101B200000000000F4F9B700F459E20004003A00A4
:101B300090C1B300F5F9B700C090040000000000A8
:101B400002002000C19F210002007800182D020031
:101B500000000000805878000201E8000004E00066
:101B60004220AE00F8FF370020C0B300A2FCB7004F
:101B7000649F2100F4E48800C49F210004E58800EC
:101B80003A4D020000000000F4F9B700F459E200F9
:101B900004003A00B0C1B300F5F9B700C0900400EA
:101BA0000000000002002000C19F21000200780018
:101BB000282D020000000000805878000201E80093
:101BC0000004E0004220AE00F8FF370020C0B30060
:101BD000A2FCB700649F2100F4E48800C49F2100A8
:101BE00004E588003A4D020000000000F4F9B70057
:101BF000F459E20004003A00C0C1B300F5F9B7009F
:101C0000C09004000000000002002000C19F2100DD
:101C100002007800382D0200000000008058780093
:101C20000201E8000004E0004220AE00F8FF3700A7
:101C300030C0B300A2FCB700649F2100F4E4880028
:101C4000C49F210004E588003A4D02000000000016
:101C5000F4F9B700F459E20004003A00E0C1B3001F
:101C6000F5F9B700C0900400000000000200200059
:101C7000C19F210002007800482D020000000000F2
:101C8000805878000201E8000004E0004220AE0025
:101C9000F8FF370010C0B300A2FCB700649F21001A
:101CA000F4E48800C49F210004E588003A4D020056
:101CB00000000000F4F9B700F459E20004003A0013
:101CC000D0C1B300F5F9B700C090040000000000D7
:101CD00002002000C19F210002007800562D020062
:101CE00000000000805878000201E8000004E000D5
:101CF0004220AE00F8FF370010C0B300A2FCB700CE
:101D0000649F2100F4E48800C49F210004E588005A
:101D10003A4D020000000000F4F9B700F459E20067
:101D200004003A00F0C1B300F5F9B700C090040018
:101D30000000000002002000C19F21000200780086
:101D4000642D020000000000805878000201E800C5
:101D50000004E0004220AE00F8FF370020C0B300CE
:101D6000A2FCB700649F2100F4E48800C49F210016
:101D700004E588003A4D020000000000F4F9B700C5
:101D8000F459E20004003A0010C2B300F5F9B700BC
:101D9000C09004000000000002002000C19F21004C
:101DA00002007800742D02000000000080587800C6
:101DB0000201E8000004E0004220AE00F8FF370016
:101DC00010C0B300A2FCB700649F2100F4E48800B7
:101DD000C49F210004E588003A4D02000000000085
:101DE000F4F9B700F459E20004003A0000C2B3006D
:101DF000F5F9B700C09004000000000002002000C8
:101E0000C19F210002007800822D02000000000026
:101E1000805878000201E8000004E0004220AE0093
:101E2000F8FF370020C0B300A2FCB700649F210078
:101E3000F4E48800C49F210004E588003A4D0200C4
:101E400000000000F4F9B700F459E20004003A0081
:101E500030C2B300F5F9B700C090040000000000E4
:101E600002002000C19F210002007800922D020094
:101E700000000000805878000201E8000004E00043
:101E80004220AE00F8FF370010C0B300A2FCB7003C
:101E9000649F2100F4E48800C49F210004E58800C9
:101EA0003A4D020000000000F4F9B700F459E200D6
:101EB00004003A0020C2B300F5F9B700C090040056
:101EC0000000000002002000C19F210002007800F5
:101ED000A02D020000000000805878000201E800F8
:101EE0000004E0004220AE00F8FF370020C0B3003D
:101EF000A2FCB700649F2100F4E48800C49F210085
:101F000004E588003A4D020000000000F4F9B70033
:101F1000F459E20004003A0040C2B300F5F9B700FA
:101F2000C09004000000000002002000C19F2100BA
:101F300002007800B02D02000000000080587800F8
:101F40000201E8000004E0004220AE00F8FF370084
:101F500020C0B300A2FCB700649F2100F4E4880015
:101F6000C49F210004E588003A4D020000000000F3
:101F7000F4F9B700F459E20004003A0050C2B3008B
:101F8000F5F9B700C0900400000000000200200036
:101F9000C19F210002007800C02D02000000000057
:101FA000805878000201E8000004E0004220AE0002
:101FB000F8FF370010C0B300A2FCB700649F2100F7
:101FC000F4E48800C49F210004E588003A4D020033
:101FD00000000000F4F9B700F459E20004003A00F0
:101FE00060C2B300F5F9B700C09004000000000023
:101FF00002002000C19F210002007800CE2D0200C7
:1020000000000000805878000201E8000004E000B1
:102010004220AE00F8FF370010C0B300A2FCB700AA
:10202000649F2100F4E48800C49F210004E5880037
:102030003A4D020000000000F4F9B700F459E20044
:1020400004003A0070C2B300F5F9B700C090040074
:102050000000000002002000C19F21000200780063
:10206000DC2D020000000000805878000201E8002A
:102070000004E0004220AE00F8FF370010C0B300BB
:10208000A2FCB700649F2100F4E48800C49F2100F3
:1020900004E588003A4D020000000000F4F9B700A2
:1020A000F459E20004003A0080C2B300F5F9B70029
:1020B000C09004000000000002002000C19F210029
:1020C00002007800EA2D020000000000805878002D
:1020D0000201E8000004E0004220AE00F8FF3700F3
:1020E00020C0B300A2FCB700649F2100F4E4880084
:1020F000C49F210004E588003A4D02000000000062
:10210000F4F9B700F459E20004003A00A0C2B300A9
:10211000F5F9B700C09004000000000002002000A4
:10212000C19F210002007800FA2D0200000000008B
:10213000805878000201E8000004E0004220AE0070
:10214000F8FF370020C0B300A2FCB700649F210055
:10215000F4E48800C49F210004E588003A4D0200A1
:1021600000000000F4F9B700F459E20004003A005E
:1021700090C2B300F5F9B700C09004000000000061
:10218000FBD9BF00800278000B60EF000600200042
:10219000F5D9BF00800378000F60EF000800200031
:1021A0003322AF00FEFF3700A4002000A4118800F6
:1021B0003322AF00FEFF3700D4002000A4118800B6
:1021C0003322AF00FEFF370004022000A411880074
:1021D0000500780086007800040020008C4B020087
:1021E000000000003322AF00FEFF37000402200091
:1021F000A41188003322AF00FEFF3700D403200073
:10220000A41188003322AF00FEFF37000402200033
:10221000A4118800619F21001104E0000700320032
:102220003322AF00FEFF37000140900034E2B700D8
:102230003562EF008100E800F7FF37003322AF007E
:10224000FEFF370004022000A41188000700780078
:1022500088007800040020008C4B02000000000081
:102260003322AF00FEFF370004022000A4118800D3
:1022700001DABF000160EF0021702200303C020053
:10228000000000003322AF00FEFF370004022000F0
:10229000A41188003322AF00FEFF3700A402200003
:1022A000A4118800A4CF80004822DE006224E1004F
:1022B0000B003900A4CF80004822DE00A3022000DA
:1022C000041CE10006003900F5D9BF0010FAB70080
:1022D00001DABF0011FAB7002886020000000000F2
:1022E000103AEF0024A0210094D0880080820200E0
:1022F0000000000070D08800FB79EC0080880400AA
:10230000000000004F047800CF0378004F037800EE
:10231000CF02780000000600DA8002000000000012
:1023200020C3B300A2FCB70084AC2000F4E4880012
:102330008490210004E58800844D02000000000024
:10234000548802000000000000000600851F78008D
:1023500038C8BF003948E300FDFF3200C4418000A7
:102360004822DE0063802000030042001040780015
:102370003BE8B700C44180004822DE0061424200D1
:102380000440780000E0B7000160EF002403200063
:10239000110009000480D8000140780039E8B70036
:1023A0003BC8BF00CF02780000000600851F780000
:1023B000F419E20003003200A0CF8000E491040091
:1023C0000000000020CF8000C0CF8800F819F8007E
:1023D0001C1AF900F619F8001E1AF90038820200DA
:1023E00000000000804278008582FB0005407800F4
:1023F000F839B400C0CF80001004E00005003A00B6
:1024000025CF800000C2B300804A78000020EF0092
:1024100011003700F819F800A81CF900F619F800A7
:10242000AA1CF900744C020000000000D0CF880004
:10243000D0CF80001004E00003003200D5CF800030
:10244000804AEB00FA39EC00FA19F800E419F900B7
:10245000F819F8000000F900CF027800000006002B
:10246000851F780002002000819E21000200780074
:102470002C27020000000000805878000201E800CC
:102480000004E0004220AE00F8FF3700049821006D
:10249000A4CF8800849E2100B4CF8800D69102008A
:1024A0000000000090CF8800F219E2003A003200EC
:1024B0003D68AE000D0037000500200005007800E3
:1024C00042270200000000000040B3004220AF009D
:1024D000060037008502E8003322AF00FEFF370018
:1024E00034E2B7003562EF00F4FF3700010020004E
:1024F0000100780058270200000000008100E80079
:102500003322AF00FEFF3700A0118800300020000A
:102510000008E600F6FF370091CF80001104E000CC
:10252000070032003322AF00FEFF37000140900069
:1025300034E2B7003562EF008100E800F7FF3700B2
:10254000648D210084C5880091CF80001104E000D3
:1025500007003200811F780011407800664C0200AD
:1025600000000000CF0078008100E800F7FF37008E
:102570008C91020000000000F439EF00849E2100DD
:10258000B4CF8800D69102000000000090CF8800F0
:102590005492040000000000CF0278000000060002
:1025A000851F7800A691020000000000804278009C
:1025B000140620000524E10006003E00A4072000C8
:1025C0000524E1000300390005407800F04DB20019
:1025D0000100370005407800E6F9B70034CF8000ED
:1025E000F4C3B2000900320034CF8000E4C2B2006C
:1025F0000600320034CF800014C2B2000300320063
:1026000034CF80006D24E10028003A00E4418000CE
:102610000960EF00E383200083024200804AEB0060
:102620000100200001007800583302000000000083
:102630008100E8003322AF00FEFF3700A0118800C0
:10264000400020000008E600F6FF3700E18320008C
:102650001104E000070032003322AF00FEFF370014
:102660000140900034E2B7003562EF008100E800DD
:10267000F7FF37003322AF00FEFF370004022000CF
:10268000A411880001982100E2832000B24878005C
:102690003104E0004220AE00FCFF3700309202001F
:1026A000000000005C9404000000000034CF8000B3
:1026B00034C2B20029003A00E44180000960EF0012
:1026C000E383200083024200804AEB003322AF0004
:1026D000FEFF370004022000A41188003322AF005F
:1026E000FEFF3700A4002000A41188003322AF00B1
:1026F000FEFF3700D4002000A4118800E1832000F1
:102700001104E000070032003322AF00FEFF370063
:102710000140900034E2B7003562EF008100E8002C
:10272000F7FF37003322AF00FEFF3700040220001E
:10273000A411880081AC2000E2832000B248780018
:102740003104E0004220AE00FCFF37005488020054
:10275000000000005C9404000000000034CF800002
:10276000C4C5B2003F003A00E44180000960EF00B8
:10277000E383200083024200804AEB003322AF0053
:10278000FEFF370004022000A41188003322AF00AE
:10279000FEFF3700A4002000A41188003322AF0000
:1027A000FEFF3700D4002000A4118800E183200040
:1027B0001104E000070032003322AF00FEFF3700B3
:1027C0000140900034E2B7003562EF008100E8007C
:1027D000F7FF37003322AF00FEFF3700040220006E
:1027E000A4118800E4832000F4E48800C04D0200B6
:1027F00000000000800278000500E00003003A00BD
:10280000380037001894040000000000E483200022
:10281000F4E48800C04D020000000000800278004F
:10282000440620000520E10001003C002D00370097
:10283000E4832000F4E48800C04D020000000000A2
:1028400080027800101AF800E5FF9F00101AF900C6
:10285000117AEF0028860200000000005C9404005A
:102860000000000034CF8000E4C7B20003003A004B
:102870000000FE005C94040000000000E4418000C1
:102880000960EF00E383200083024200E6D9BF0025
:1028900080429800E441800023022000041CE100F3
:1028A00003003E003C68EF005A9404000000000062
:1028B0003C68EC000B00370002002000E1832000A0
:1028C00002007800B4250200000000008058780063
:1028D0000201E8000004E0004220AE00F8FF3700EB
:0C28E0003C68EF00CF027800000006000A
:0200000401F009
:10000000CF000000CF00000007000000A2000000A9
:10001000C60000000F000000E7000000C200000062
:00000001FF
